:020000022000DC
:10600000000004207D860200F9610700F3670700A5
:10601000F9610700F9610700F9610700000000005D
:10602000000000000000000000000000F96107000F
:10603000F961070000000000F9610700F96107003D
:1060400071850200F9610700D1890200AD88020064
:10605000BD880200F9610700ED810200F9610700C7
:10606000F9610700B1890200C18902004D86020072
:10607000F9610700F9610700F9610700F96107009C
:10608000218E02005D860200F9610700F9610700B8
:10609000F9610700F96107001D890200F961070035
:1060A000F9610700F9610700F9610700F96107006C
:1060B000F9610700F961070000000000000000001E
:1060C000F9610700F9610700F9610700CD88020056
:1060D0006D860200F9610700F9610700F18902008D
:1060E000E1890200F9610700F9610700F588020003
:0860F00000000000F961070047
:1070000040F8044B40F8045B40F8046B40F8047B04
:1070100040F8048B40F8049B40F804AB40F804BBF4
:1070200040F804CB40F804DB6846704781F000412B
:1070300002E000BF83F0004330B54FEA41044FEA5D
:10704000430594EA050F08BF90EA020F1FBF54EAF8
:10705000000C55EA020C7FEA645C7FEA655C00F094
:10706000E2804FEA5454D4EB5555B8BF6D420CDD65
:107070002C4480EA020281EA030382EA000083EAE8
:10708000010180EA020281EA0303362D88BF30BD88
:1070900011F0004F4FEA01314FF4801C4CEA1131DE
:1070A00002D0404261EB410113F0004F4FEA03333D
:1070B0004CEA133302D0524263EB430394EA050FC8
:1070C00000F0A780A4F10104D5F1200E0DDB02FA37
:1070D0000EFC22FA05F2801841F1000103FA0EF2CB
:1070E000801843FA05F359410EE0A5F120050EF191
:1070F000200E012A03FA0EFC28BF4CF0020C43FAC2
:1071000005F3C01851EBE37101F0004507D54FF0CE
:10711000000EDCF1000C7EEB00006EEB0101B1F51E
:10712000801F1BD3B1F5001F0CD349085FEA300064
:107130004FEA3C0C04F101044FEA445212F5800F6F
:1071400080F09A80BCF1004F08BF5FEA500C50F10C
:10715000000041EB045141EA050130BD5FEA4C0CEF
:10716000404141EB0101013C28BFB1F5801FE9D24C
:1071700091F0000F04BF01460020B1FA81F308BF6F
:107180002033A3F10B03B3F120020CDA0C3208DD3B
:1071900002F1140CC2F10C0201FA0CF021FA02F116
:1071A0000CE002F11402D8BFC2F1200C01FA02F186
:1071B00020FA0CFCDCBF41EA0C019040E41AA2BFAB
:1071C00001EB0451294330BD6FEA04041F3C1CDA73
:1071D0000C340EDC04F11404C4F1200220FA04F093
:1071E00001FA02F340EA030021FA04F345EA03013D
:1071F00030BDC4F10C04C4F1200220FA02F001FAFF
:1072000004F340EA0300294630BD21FA04F0294680
:1072100030BD94F0000F83F4801306BF81F4801119
:107220000134013D4EE77FEA645C18BF7FEA655C8C
:1072300029D094EA050F08BF90EA020F05D054EA5E
:10724000000C04BF1946104630BD91EA030F1EBF63
:107250000021002030BD5FEA545C05D14000494167
:1072600028BF41F0004130BD14F580043CBF01F55A
:10727000801130BD01F0004545F0FE4141F4700140
:107280004FF0000030BD7FEA645C1ABF194610461B
:107290007FEA655C1CBF0B46024650EA013406BF1C
:1072A00052EA033591EA030F41F4002130BD00BFDB
:1072B00090F0000F04BF0021704730B54FF4806498
:1072C00004F132044FF000054FF0000150E700BF19
:1072D00090F0000F04BF0021704730B54FF4806478
:1072E00004F1320410F0004548BF40424FF0000165
:1072F0003EE700BF42004FEAE2014FEA31014FEAA8
:1073000002701FBF12F07F4393F07F4F81F06051F6
:10731000704732F07F4208BF704793F07F4F04BF41
:1073200041F40021704730B54FF4607401F000451E
:1073300021F000411CE700BF50EA010208BF70477E
:1073400030B54FF000050AE050EA010208BF70476F
:1073500030B511F0004502D5404261EB41014FF4D8
:10736000806404F132045FEA915C3FF4D8AE4FF0E0
:1073700003025FEADC0C18BF03325FEADC0C18BFC3
:10738000033202EBDC02C2F1200300FA03FC20FA14
:1073900002F001FA03FE40EA0E0021FA02F1144461
:1073A000BDE600BF4FEA4102B2F1E04324BFB3F5AE
:1073B000001CDCF1FE5C0DD901F0004C4FEAC0026C
:1073C0004CEA5070B2F1004F40EB830008BF20F050
:1073D0000100704711F0804F21D113F13872BCBF0A
:1073E00001F00040704741F480114FEA5252C2F15F
:1073F0001802C2F1200C10FA0CF320FA02F018BFA8
:1074000040F001004FEAC1234FEAD32303FA0CFCFA
:1074100040EA0C0023FA02F34FEA4303CCE77FEA89
:10742000625307D150EA01331EBF4FF0FE4040F4D3
:107430004000704701F0004040F0FE4040F4000082
:10744000704700BF80F0004002E000BF81F00041C3
:1074500042001FBF5FEA410392EA030F7FEA226CFA
:107460007FEA236C6AD04FEA1262D2EB1363C1BF8A
:10747000D218414048404140B8BF5B42192B88BFF9
:10748000704710F0004F40F4000020F07F4018BF1C
:10749000404211F0004F41F4000121F07F4118BF3C
:1074A000494292EA030F3FD0A2F1010241FA03FCE4
:1074B00010EB0C00C3F1200301FA03F100F00043CC
:1074C00002D5494260EB4000B0F5000F13D3B0F194
:1074D000807F06D340084FEA310102F10102FE2A03
:1074E00051D2B1F1004F40EBC25008BF20F0010073
:1074F00040EA03007047490040EB0000013A28BF12
:10750000B0F5000FEDD2B0FA80FCACF1080CB2EB94
:107510000C0200FA0CF0AABF00EBC2505242184312
:10752000BCBFD0401843704792F0000F81F40001B7
:1075300006BF80F400000132013BB5E74FEA41038A
:107540007FEA226C18BF7FEA236C21D092EA030FF6
:1075500004D092F0000F08BF0846704790EA010F70
:107560001CBF0020704712F07F4F04D1400028BF9D
:1075700040F00040704712F100723CBF00F500007F
:10758000704700F0004343F0FE4040F400007047B5
:107590007FEA226216BF08467FEA23630146420261
:1075A00006BF5FEA412390EA010F40F48000704774
:1075B0004FF0000304E000BF10F0004348BF40421A
:1075C0005FEA000C08BF704743F0964301464FF056
:1075D00000001CE050EA010208BF70474FF00003B2
:1075E0000AE000BF50EA010208BF704711F00043F3
:1075F00002D5404261EB41015FEA010C02BF8446C3
:107600000146002043F0B64308BFA3F18053A3F521
:107610000003BCFA8CF2083AA3EBC25310DB01FA68
:1076200002FC634400FA02FCC2F12002BCF1004FEC
:1076300020FA02F243EB020008BF20F0010070477D
:1076400002F1200201FA02FCC2F1200250EA4C00D1
:1076500021FA02F243EB020008BF20EADC70704717
:107660007BB972B90029BEBF00204FF0004106E08F
:1076700008BF00281CBF6FF000414FF0FF3000F042
:1076800081B9ADF1080C6DE904CE002909DB002BAE
:107690001ADB02F045FDDDF804E0DDE9022304B069
:1076A0007047404261EB4101002B1BDB02F038FDCB
:1076B000DDF804E0DDE9022304B0404261EB410162
:1076C000524263EB43037047524263EB430302F0C1
:1076D00027FDDDF804E0DDE9022304B0404261EB60
:1076E00041017047524263EB430302F019FDDDF89C
:1076F00004E0DDE9022304B0524263EB4303704728
:1077000053B94AB9002908BF00281CBF4FF0FF3108
:107710004FF0FF3000F036B9ADF1080C6DE904CE42
:1077200002F0FEFCDDF804E0DDE9022304B070475E
:1077300070B54FF0FF0C4CF4E06C1CEA11541DBF07
:107740001CEA135594EA0C0F95EA0C0F00F0DEF8D2
:107750002C4481EA030621EA4C5123EA4C5350EAB7
:10776000013518BF52EA033541F4801143F4801308
:1077700038D0A0FB02CE4FF00005E1FB02E506F099
:107780000042E0FB03E54FF00006E1FB03569CF0EE
:10779000000F18BF4EF0010EA4F1FF04B6F5007FF4
:1077A00064F5407404D25FEA4E0E6D4146EB060666
:1077B00042EAC62141EA55514FEAC52040EA5E50EF
:1077C0004FEACE2EB4F1FD0C88BFBCF5E06F1ED899
:1077D000BEF1004F08BF5FEA500E50F1000041EBD0
:1077E000045170BD06F0004646EA010140EA02007D
:1077F00081EA0301B4EB5C04C2BFD4EB0C0541EA9F
:10780000045170BD41F480114FF0000E013C00F3B3
:10781000AB8014F1360FDEBF002001F0004170BDD7
:10782000C4F10004203C35DA0C341BDC04F11404F0
:10783000C4F1200500FA05F320FA04F001FA05F27C
:1078400040EA020001F0004221F0004110EBD37049
:1078500021FA04F642EB06015EEA430E08BF20EA75
:10786000D37070BDC4F10C04C4F1200500FA04F318
:1078700020FA05F001FA04F240EA020001F00041AA
:1078800010EBD37041F100015EEA430E08BF20EA1D
:10789000D37070BDC4F1200500FA05F24EEA020E65
:1078A00020FA04F301FA05F243EA020321FA04F094
:1078B00001F0004121FA04F220EA020000EBD3704B
:1078C0005EEA430E08BF20EAD37070BD94F0000F4B
:1078D0000FD101F00046400041EB010111F4801F7F
:1078E00008BF013CF7D041EA060195F0000F18BF30
:1078F000704703F00046520043EB030313F4801F6C
:1079000008BF013DF7D043EA0603704794EA0C0F25
:107910000CEA135518BF95EA0C0F0CD050EA41063B
:1079200018BF52EA4306D1D181EA030101F00041B8
:107930004FF0000070BD50EA410606BF10461946E0
:1079400052EA430619D094EA0C0F02D150EA0136EC
:1079500013D195EA0C0F05D152EA03361CBF10462D
:1079600019460AD181EA030101F0004141F0FE41CC
:1079700041F470014FF0000070BD41F0FE4141F450
:10798000780170BD704700BF4A0011D212F5001295
:1079900011D20DD56FF47873B3EB62520ED44FEA67
:1079A000C12343F0004343EA505323FA02F07047E7
:1079B0004FF00000704750EA013002D14FF0FF3025
:1079C00070474FF00000704730B5144685B017A3DC
:1079D000D3E90023FFF744FE054601A9284647F0F6
:1079E00093F99DF807309DF806200F491B0443EAE0
:1079F00042539DF8082043EAC2239DF8092043EA38
:107A000042139DF80A2043EA5203BDF8042025F0F2
:107A10000105A2F2BC7243EA4263A5FB01012360A7
:107A200005B030BDAFF3008000CA9A3B00CA9A3B54
:107A300000000000182A2DE9F74F054621D0202A22
:107A400022D00A200423C5F8002185F8040185F816
:107A50000531284600F0A0FC0022034695F80541B8
:107A6000A24214D3DFF8DCC0DFF8DCE000EB8403D3
:107A700095F804210132B4EB820F1AD303B0BDE8AC
:107A8000F08F0C200623DEE70E200823DBE711F839
:107A9000044B03F8044B11F8034C03F8034C11F8A2
:107AA000024C03F8024C11F8014C03F8014C01326E
:107AB000D4E795F80521B4FBF2FA02FB1A4913F852
:107AC000041C13F8038C13F8027C13F8016C019268
:107AD000B9F1000F0BD11CF808B01CF807801CF896
:107AE00006701CF801601EF80A108BEA0101D5F837
:107AF0000021202A0CD1B9F1040F09D1DFF84490FC
:107B000019F8011019F8088019F8077019F80660BB
:107B1000019AA21A043310F8229000EB820281EA43
:107B2000090103F8041C517888EA010803F8038C62
:107B300091784F4003F8027CD278564003F8016CEC
:107B4000013495E773370A0068370A002DE9F04FD2
:107B5000044685B0084600F01FFC89460246804670
:107B6000214600204EF025FB231D019304F1100354
:107B70000125029322462146002311F82300324EAC
:107B8000305C01F823000133042BF6D1019B013155
:107B90008B42F1D1617963786170617A6171617B47
:107BA0006172A17A6373A378A170A17BA372A37998
:107BB000A171E17BA373E378E170E17AE173E1798C
:107BC000E172E37199F80431AB4234D092F800B01D
:107BD0005678917892F803A08BEA060081EA0A03AE
:107BE00080EA0307039366F007F88BEA0000784009
:107BF000107086EA010065F0FFFF46407E40567037
:107C0000039865F0F9FF4140794091708BEA0A00D2
:107C100065F0F2FF8AEA000A029B87EA0A07D7703A
:107C200004329342D2D128464246214601354EF0D5
:107C3000C0FAEDB29EE742462146284605B0BDE8AF
:107C4000F04F4EF0B6BA00BF73370A002DE9F04F7F
:107C5000504C904603F003029B101F2B04EB821440
:107C600089469E464C49A8BF4FF01F0E1C2B1D464F
:107C7000A8BF1C2551F822206168033587B025EA8A
:107C8000E575294101920391E268A1688446294182
:107C900000202A410290049105925CF8045B3F4A5F
:107CA000154225F0004111D106AA02EB810151F8DD
:107CB000102C002D40EA0200B8BF5242B8F1010872
:107CC00049F8042BE9D107B0BDE8F08F344A1542DA
:107CD00009D154F82120002BBABFCEF100018A400F
:107CE00042FA0EF2E5E72F4A154214D110392E4A16
:107CF000019E52F8212082FB0616AEF10302002AF3
:107D000044DA51426FF0004242FA01F7B742D0DB49
:107D100006FA01F2CDE74A04B2F1006FB6BF4A0598
:107D200000210421B2F1005FB8BF92001F4EB8BF1E
:107D30000231B2F1804FBCBF52000131B242C7BF25
:107D40001B4F1C4E1C4F1D4E924687FB0ABA77688C
:107D50005744924687FB0ABAB7685744924687FB56
:107D60000ABAF768BA448AFB027236691644144AA2
:107D700052F8212086FB0272019ED20082FB067619
:107D8000104A52F82120AEEB0202B8E746FA02F29E
:107D90008FE700BF98710A0088710A00FCFFFF7F1F
:107DA000F0FFFF7FC0FFFF7FC8700A009979825AF9
:107DB0006321851060700A00A9BDA02974700A00B3
:107DC000A8700A0088700A002DE9F74F00F5A04856
:107DD0004FF0000A476D88F8B4AD88F8AEADB1F148
:107DE000000B816DC0F820A04FF0FF3304464362C2
:107DF0000CBFFF220C22CB1BD019013B04F5DA7615
:107E00008842C8BF1A46236C0092314604F15400E0
:107E10009847009A8242054613D1002F68D1A549A0
:107E20000522304659F0C7F878B1A34905223046FB
:107E300059F0C1F848B10823E361002003B0BDE860
:107E4000F08F0623F8E70123F6E7B4F8BA31236090
:107E5000A360B4F8BC316360E36094F8BE31C3F34F
:107E600002120132A261BBF1000F40F0BB8194F815
:107E7000BF2188F8B02D180688F8AFBD4BD503F0A8
:107E8000070B0BF1010B4FF0030A05F5DA710AFA43
:107E90000BFA236C5246214404F1540098470544E0
:107EA00098F8B50D01282DD804F58D520221123213
:107EB00001FA0BF1A44611449CF8C1319CF8C2E1CF
:107EC000DB084FEA9E0EDB0243EA4E139CF8C3E147
:107ED00043EADE0300B15BBA22F8023F91420CF1A3
:107EE000030CE9D14FF0030A0AFA0BFA0AF10D0A62
:107EF00016F80A302C2B00F0E3803B2B0ED1072321
:107F0000E3616FE104F58D50524604F2C111143063
:107F100059F065F8EAE74FF00D0AE9E7212B40F048
:107F20009B8006EB0A020AF102015378FE2B68D00F
:107F3000FF2B21D0012B5ED0F92B84D1735C042B55
:107F400013D1D17888F8AF1D5079137903EB002352
:107F50000A204343012BD8BF64232362C90744BFCF
:107F6000937988F8B13D0AF108018A46C0E70AEB27
:107F70000301BAF1000FF8D016F801A04B1CA5EBD5
:107F8000030B0AF11F025A4515DB01F2B5115A46DF
:107F900021443046009359F04DF8009B0BF5DA71FF
:107FA0001F440AF12002236C214404F15400984735
:107FB00000230BEB0005BAF10B0FD8D106EB030B36
:107FC0003E4900935246584658F0F5FF009B03F196
:107FD0000B010028D0D19BF80B30032BCCD19BF8A0
:107FE0000C30012BC8D19BF80E209BF80D3003EB11
:107FF00002236362C0E7735C4A1C9918002BFAD114
:10800000B3E716F801A04B1CA5EB030B0AF11F0206
:108010005A4515DB01F2B5115A462144304600930A
:1080200059F008F8009B0BF5DA711F440AF12002A1
:10803000236C214404F15400984700230BEB000506
:10804000A26B1AB9DA19A263A4F83CA00AEB0301E7
:10805000BAF1000FD5D188E7A36DDB1B202BB4BF8D
:1080600007230123E8E604F5A55006EB0B011430C5
:10807000009258F0B4FF009A93447EE0009258F0CA
:10808000AEFF009A616B236C114461635144ABEB0A
:108090000202214404F1540000929847636B009A55
:1080A00029461A4494E0636C394404F1540098471B
:1080B00098E000BFC5200900CB200900BD1E0900C3
:1080C00006EB0A030AF10A0B99785A7802EB0122AF
:1080D00022611979DA7802EB0122626199795A7981
:1080E00002EB01222260197ADA7902EB0122626046
:1080F0005B7A88F8B33D1A0644D503F007030133D1
:1081000005F5DA7103229A4001932144236C009211
:1081100004F15400984798F8B51D009A01290544C8
:10812000A1D8019B04F5A5524FF0020C12324FF07A
:10813000010B0CFA03FC04EB0A000BFA03FB94445A
:1081400090F8BE3190F8BFE1DB084FEA9E0EDB02EB
:1081500043EA4E1390F8C0E143EADE0301B15BBA93
:1081600022F8023F944500F10300E9D10BF1FF3BF7
:108170000BEB4B0B0AF10D0AD34404F5A04301228B
:1081800083F8B42D16F80B30174A04F5A0480BF10C
:10819000010188F8B23DD35CA3610023636341F21F
:1081A000B47A8D421EDD16F801B0606B4B1CEA1AE2
:1081B00050449345204406EB03013FF75FAF5A4616
:1081C000009358F00CFF626B009B5A440BEB0301C9
:1081D0006263BBF1000FE4D101238D4288F8AE3D0C
:1081E0003FF761AF012029E6A86D0A002DE9F047AD
:1081F000002486B0CDE90044614A624E624D0121FF
:1082000013684BB1D6F804330B4205D0A2F5C04039
:1082100080B260F0F5F80C430432AA424FEA410103
:10822000EED1584BD3F87C3173B14FF4BE7060F08F
:10823000E7F84FF0A04344F00044D3F81035009322
:10824000524BD3F810350193E3B2D3B1504F01260E
:108250000025344210D0AB0003F1804303F5C04346
:10826000D3F81005D3F8101557F8253023B1C1F312
:108270000141C0F3052098470135082D4FEA460615
:10828000E7D1002C78DA04AE0023049373604FF03A
:10829000FF33029300253F4F0393A84617F9012FA0
:1082A000531C4ED002F03F0402A920465FFA82F927
:1082B00060F095F8002844D0354B19194FEA991908
:1082C00091F9281053F821A0BAF1000F0BD1B9F1A0
:1082D000030F36D1E10802F0070001238340705CF0
:1082E0000343735402E0B9F1030FF3D01F2C8BBF8B
:1082F00002F01F022246254B4FF0A04302F5E07228
:10830000694653F822202046C2F3014260F067F824
:1083100030B1022A15D1B9F1030F0CD1494605E05D
:10832000032A0ED1B9F1030F05D10221204637F0FF
:1083300063FB0135EDB2BAF1000F02D04946204689
:10834000D04708F10103022B4FF00108A6D19DB1DF
:108350004FF0A0430099D3F8102503F540739142E4
:10836000D3F8103502D10199994205D00092049AB0
:10837000CDE90132059B8DE706B0BDE8F08700BF6F
:108380000061004000600040206100400003005098
:10839000D45B01202B5C0120D0F80031103B102B66
:1083A00007D8054A22FA03F313F0010F08BF002093
:1083B00070470020704700BF010101002DE9F04F18
:1083C00004468DB00846FFF7E7FF0D4601900246D0
:1083D000214695F804014DF0ECFE95F80461231D4B
:1083E000013E099304F11003F6B20A93627A637BAB
:1083F00062736279627262786271A27A6370A37842
:10840000A270A27BA372A379A271E279A373E3782D
:10841000E270E27AE271E27BE272E3732546224681
:10842000002312F823105148415C02F82310013355
:10843000042BF6D1099B01329342F1D1019A2146D6
:1084400030464DF0B6FE002E00F08C8095F800808E
:10845000AB780093404665F0CFFB029065F0CCFB13
:10846000039065F0C9FB6F780B90384665F0C4FB4C
:10847000024665F0C1FB049065F0BEFB82460098A1
:1084800095F803B065F0B8FB059065F0B5FB069074
:1084900065F0B2FB8146584665F0AEFB079065F08B
:1084A000ABFB089065F0A8FBDDE9023183EA010C23
:1084B0000B9B069983EA0C0C82EA0C0C8AEA0C0CE2
:1084C00081EA0C0C89EA0C0C009980EA0C0C87EA12
:1084D0000C0C81EA0C0C04995A404A4005998AEA2E
:1084E00002024A40089989EA02024A404240009941
:1084F00088EA02024A408BEA02026A70039A0599EE
:108500005A408AEA02024A4006994A40079989EA93
:1085100002024A40424088EA02027A408BEA0C0C8E
:108520008BEA020B85F800C085F802B0029A53402E
:10853000049A53408AEA030A089A89EA0A0981EAF6
:1085400009035340584000990A9B88EA000887EACB
:1085500008077940E9700435AB427FF477AF013EFC
:10856000F6B243E70DB0BDE8F08F00BF68360A00F1
:1085700010B54FF08043D3F80443620707D54FF49A
:1085800084705FF049FF10B11E4B1B689847A3062B
:1085900008D54FF48A705FF03FFF18B11A4B0020E6
:1085A0001B689847600608D54FF48C705FF034FF65
:1085B00018B1154B01201B689847210608D54FF4C8
:1085C0008E705FF029FF18B1104B00201B68984790
:1085D000E20508D54FF490705FF01EFF18B10B4B09
:1085E00001201B689847A3050AD54FF492705FF0ED
:1085F00013FF28B1054BBDE810401B680220184747
:1086000010BD00BF645D0120685D01206C5D01202C
:10861000DFED0A7A9FED0A7ADFED0A6AA0EE277A8B
:10862000DFED097AE7EE007AB7EE007AA0EE267A5F
:1086300067EE807A87EE870A704700BF6BD30DBC68
:10864000BA132FBDAEE534BF75AA2A3E02480322F5
:10865000002122F0A3BA00BF00B00040024804226B
:10866000012122F09BBA00BF001001400248042201
:10867000022122F093BA00BF0040024008B57E4AB2
:108680007E4B7F498B42C0F0BF807E4B7E4A0021EB
:108690009342C0F0BE804FF08053D3F83021082AB7
:1086A0004ED14FF080420021C2F80C11C2F81011D7
:1086B000C2F8381502F54042D3F80414C2F8201568
:1086C000D3F80814C2F82415D3F80C14C2F82815EE
:1086D000D3F81014C2F82C15D3F81414C2F83015BE
:1086E000D3F81814C2F83415D3F81C14C2F8401586
:1086F000D3F82014C2F84415D3F82414C2F848154E
:10870000D3F82814C2F84C15D3F82C14C2F850151D
:10871000D3F83014C2F85415D3F83414C2F86015E5
:10872000D3F83814C2F86415D3F83C14C2F86815AD
:10873000D3F84014C2F86C15D3F84434C2F870353D
:1087400055F088FC18B1514B514AC3F88C2655F0AE
:1087500081FC18B14F4BFB22C3F8182555F07AFC69
:1087600058B14FF080424FF08051D2F8E43ED1F83A
:10877000581261F30303C2F8E43E55F06BFC20B1DC
:10878000454B4FF40072C3F840264FF08053D3F8A6
:108790003031082B09D14FF08043D3F80024D107A2
:1087A00044BF6FF00102C3F800243C4AD2F888307D
:1087B00043F47003C2F88830BFF34F8FBFF36F8F5D
:1087C0004FF01023D3F80C22D20725D5344B0122C9
:1087D000C3F80425D3F80024002AFBD04FF0102260
:1087E000D2F80C3223F00103C2F80C322C4BD3F830
:1087F0000024002AFBD00022C3F80425D3F800246B
:10880000002AFBD000F0ACFC52F8040B43F8040B38
:1088100038E743F8041B3BE7D3F80022002A03DBC8
:10882000D3F80432002B22DA1D4B0122C3F80425B1
:10883000D3F80024002AFBD04FF010221221C2F8F6
:108840000012D3F80024002AFBD04FF0102312228C
:10885000C3F80422124BD3F80024002AFBD00022D4
:10886000C3F80425D3F80024002AFBD0CAE70D4B37
:108870000D4A1A6040F0BCFF2C7B0A00000001206A
:10888000E805012000060120946901200050004005
:108890004881030000F000400090024000ED00E03D
:1088A00000E00140000001200090D003014902488F
:1088B00047F03ABB985C01200030004002494FF07D
:1088C000402047F031BB00BFCC5C012008B5074811
:1088D000D0F8183143B14FF48C715FF089FDBDE8D9
:1088E0000840034856F06CBF08BD00BF003002408E
:1088F000385C012008B50748D0F8183143B14FF46F
:108900008C715FF075FDBDE80840034856F058BF14
:1089100008BD00BF00F002405C5C012073B51F4C35
:10892000022501A861F020FB052812D11C4D4FF44F
:108930000C741C48ADF802400DF1020161F0A0FA80
:1089400008B30C2803D1184918485AF052FA02B05B
:1089500070BD019B032B14D004D8022BE1D100235E
:108960002370DEE7A3F10902022ADAD80A2B06D027
:10897000092B14BF0120022047F09CF9D1E7002009
:10898000FAE72570CDE7D5F8B030002BD1D01E68BE
:108990000448D3E9011290473346F6E77569012090
:1089A000745D0120A4590120B81C090098600900D9
:1089B0000149024857F09BBE805C012000900040B6
:1089C0000149024857F093BE8C5C012000A0004092
:1089D0000149024864F068B8005D012000200040B1
:1089E0000149024864F060B8245D01200080024023
:1089F0002DE9F04FBC4BBD4AD3F80013002385B0DE
:108A00001C4601201D4621FA03F6F6070BD552F845
:108A1000236046B100FA03F6344342F82350BFF313
:108A20006F8FBFF34F8F0133192BECD1E10738D58E
:108A3000AD4B0122C3F81425C3F8102500221546BA
:108A4000930003F1804303F51C330132082A5D6073
:108A50009D62F5D1A44BA6485D629D64C3F8585150
:108A6000D3F80024D3F800140A43C3F80024D3F841
:108A70000023C3F808239F4AC3F8042300214FF4BE
:108A8000927258F0EDFA9A4A8DF8085040231383F9
:108A9000138101214FF4807301A8ADF8043017F061
:108AA000BFFE14F4006F924D07D08F4BD3F8A83659
:108AB000A5F81631012385F81C31A20204F48006C2
:108AC00035D5894AD2F8143513F4807308D01EB115
:108AD000D2F80034DB0702D408204BF0A5FA0123BA
:108AE000814AD2F81015CF0540F14A8195F81C3122
:108AF0008BB1002385F81C31B5F816319BB24FF4C9
:108B0000E06203930121882301A8ADF80420ADF8A9
:108B1000083017F085FE744B4FF44072D3F82035BF
:108B20000293012101A8ADF8042017F079FE7EB36D
:108B30006D4BD3F8006440F201723240F005C3F887
:108B4000002409D50121C3F82C1501A84FF4806336
:108B5000ADF8043017F064FE71050FD5624B0122A9
:108B6000C3F808259A65D3F8002312F4001208BF51
:108B7000C3F854214FF40012C3F80423B20507D5FB
:108B80004FF4A063012101A8ADF8043017F048FEAE
:108B900023022ED5544BD3F88014D3F88424D3F871
:108BA00088E4D3F88CC4D3F89074D3F89464D3F8E1
:108BB0009804D3F89C3411F07F0FD2B201D1052A6A
:108BC00017D04FF4C0688DF808108DF80E00012101
:108BD00001A8ADF804808DF809208DF80AE08DF821
:108BE0000BC08DF80C708DF80D608DF80F3017F0FC
:108BF00017FE414B23403BB1BFF35B8F3F4B4FF020
:108C000000021A70BFF35B8F394FDFF8DCB000262B
:108C1000B8464FF0140AB14606F10C0324FA03F3E8
:108C2000D80726D50AFB06B305EB4611D3F808276B
:108C3000D8F8003013FA82F3C8F80030B1F806C053
:108C400090B2082E1CFA82F24FEA4613CA8000F056
:108C5000A480B8F80820824240F09F80CA88B8F803
:108C6000041092B2914240F2988016B924481AF04A
:108C7000C5FD0136092E08F12008CDD1214B234036
:108C8000002B00F09480184BD3F86C84C3F86C84EC
:108C9000BFF36F8FBFF34F8F14F480641CBFD3F802
:108CA0008044D3F88064DFF848A01DBFC6F3C01627
:108CB000C4F3C01486F0010626464FF000094FF4B5
:108CC000E06B28FA09F1CA0703D4B9F1000F31D1DA
:108CD00084B3054B142202FB09315FFA89F0D1F805
:108CE0000836DAF810100FE0007002400071024000
:108CF000E82101200514C001FCFB1F00082301200E
:108D00004C7002400004000151FA83F1CAF81010BF
:108D100005EB4911B1F816E05EFA83FCA1F816C024
:108D2000B1F816C0BAF814E01FFA8CFCE6455ED91B
:108D30004BF05AF909F10109B9F1080F0AF1200ABB
:108D4000BFD100244FF0010904F1100328FA03F306
:108D5000DB0701D474B96EB105EB44126301D17A1B
:108D6000002955D0D288B98892B2914250D9E0B248
:108D70004BF05AF90134082C07F12007E4D116E032
:108D8000002B7FF4C8AE95F82131002B7FF4C3AEE1
:108D90004FF40013C2F80833BDE62B44DA7A8AB9DF
:108DA0004FF0E023D3F8F03DD90700D500BE1A4AB2
:108DB0001A4B136010460023536005B0BDE8F04F16
:108DC00007F014BDDA88A8F8042083F80B90DB883C
:108DD0008DF808609BB24FF4E062012101A8ADF864
:108DE000042003938DF8099017F01AFD41E7C98A12
:108DF000ADF804B089B260F07F00039100218DF8D6
:108E000008008DF8091001A8012117F009FD91E76C
:108E10002B4483F80A90ADE73863012055CD080054
:108E200010B5074CD4F800314BB1064B5B6898473E
:108E300020464FF48071BDE810405FF0D9BA10BDF4
:108E400000000140485D0120022A2DE9F04159D17E
:108E50003B4B826883FB02423A4D846985FB046484
:108E600022440A60DFF8F0C042688CFB0242364EB2
:108E7000C46986FB047422444A60026883FB024290
:108E8000046A85FB046422448A60304E026886FBD3
:108E900002422F4C056A84FB05752A44CA604FF0D4
:108EA0006045426885FB0272C76985FB07E73A4463
:108EB0000A61826884FB0272876986FB07E73A448D
:108EC0004A61426983FB02728A6102698CFB027209
:108ED000CA61C26883FB02720A62C36886FB03230D
:108EE0004B62036985FB03238B62436984FB032385
:108EF000CB620023C1E91033C1E90E33C1E90C3361
:108F0000BDE8F081134B902404FB023202F1480EBD
:108F100002F18C0501F14406683250F8043B55F823
:108F200004795EF804CB1C468CFB048441F8044BA6
:108F300087FB0343AA4246F80439EED1E0E700BFBD
:108F4000D8E3CEB8281C3107CD3C410D9A615FC9EA
:108F5000669EA0F6206E0A0033C3BEB22DE9F84328
:108F60001C4E04468846914600254FF4004746F0C3
:108F70000106B4F85E20ABB29A4205D894F83400EA
:108F8000BDE8F84336F04CBD03F00F0347FA03F396
:108F900013EA090F14BF0121002120464DF06CFF98
:108FA000B4F85E30AAB2A3EB08039A4203DD94F84A
:108FB000340036F063FD94F8610036F05FFD402028
:108FC000B04794F8610036F02BFD4020B0470135E2
:108FD000CFE700BF401D0A00F8B590F86530013BAF
:108FE00080F86B3090F866305A1E80F86C20012BA8
:108FF00088BF90F86C304FF000058CBF03F1FF3351
:10900000012380F86D30044680F86E500127856595
:1090100040F2033694F86330EAB293423CD82368B6
:10902000314A934257D002F58052934255D002F50F
:109030008052934253D002F58032934251D002F5D0
:10904000805293421ED10423284850F8332000EB6D
:10905000C300002590F9043001215160002BC2F8B3
:109060000455D160C2F80855C2F810554FF4803548
:10907000C2F8045306DB5A0903F01F0399401C4B46
:1090800043F82210236801224FF47A715A60DA60A3
:10909000C3F840151A60F8BDA36C03EB02131B7BE9
:1090A0001F2B86BF03F01F0312494FF0A04103F5A9
:1090B000E07341F82360A36C94F86D1003EB021386
:1090C0003942187B04D036F0D9FC7F000135A1E786
:1090D00036F0A6FCF9E70023B6E70123B4E7022344
:1090E000B2E70323B0E700BF008000407C680A00BD
:1090F00000E100E00003005000280CDB43090649B2
:1091000000F01F0020330122824041F82320BFF3EA
:109110004F8FBFF36F8F704700E100E043090649AE
:1091200000F01F0020330122824041F82320BFF3CA
:109130004F8FBFF36F8F704700E100E00028ABBF97
:1091400000F16040054B00F5614000F00F004FEA70
:109150004111B4BF195480F80013704714ED00E0BA
:10916000BFF34F8F0549064BCA6802F4E062134310
:10917000CB60BFF34F8F00BFFDE700BF00ED00E005
:109180000400FA05014B1868704700BF5400012025
:1091900007EE900AF5EEC07AF1EE10FA01D400F075
:1091A00009B808B580F0004000F004F8404261EBD7
:1091B000410108BD70B5FEF79DF80C4B0022044636
:1091C0000D46FEF7B5FAFEF7DFFB0646FEF770F830
:1091D000074B0022FEF7ACFA02460B462046294612
:1091E000FDF728FFFEF7D0FB314670BD0000F03DD3
:1091F0000000F04170B510EE105A25F00044012334
:10920000B4F1FF4FB0EE403A0646036004D320EEBF
:10921000003AB0EE430A70BD34B9DFEDD07AB7EE54
:10922000007A87EE273AF4E7B4F1E45F0BD2002D21
:10923000BEBF4FF0FF330360B1EE400A24F048F99F
:10924000B1EE403AE5E7002D80F2C682B4F1964FC8
:10925000E3D2B4F17A5F9FEDC25A78D2DFEDBF0A54
:1092600020EE050A002000F015FEF0EE402AF5EE93
:10927000402AF1EE10FAD0D023EE220AB0EEC00A56
:1092800085EE000A24F024F9F5EEC02AF1EE10FA7A
:10929000B0EE402A40F1B9804FF0FF33B4F17E5F69
:1092A000336000F09382B4F1804F00F08F82B1EE12
:1092B000433A6B0000F1DE81AA4B9C4200F2F5803C
:1092C000B0EE430A24F004F9A74B9C42B1EE400AE9
:1092D00040F29D80B7EE007A37EE437A67EE077A68
:1092E000DFEDA26A9FEDA26A9FEDA23AA7EEA66A01
:1092F000DFEDA16AE6EE276A9FEDA06AA6EEA76AF7
:10930000DFED9F6AE6EE276A9FED9E6AA6EEA73A1A
:10931000DFED9D6AE7EE866A9FED9C6AA6EEA76A7E
:10932000DFED9B6AE6EE276A9FED9A6AA6EEA76AD2
:10933000DFED996AE6EE276A23EE073AA6EEA73A32
:10934000F6EE007AA7EE673A33EE003AFFE0B1EEB0
:10935000407AB0EE470A1DF071F9B4EE407AF1EEB2
:1093600010FA19D0F6EE007A27EE277AB0EE470A07
:109370001DF064F937EE400A30EE000AF0EE407A54
:10938000FEEECF7A17EE903A062B39D8DFE803F0DD
:109390002312121F1F2B2B00DFED807A77EEC37A8A
:1093A00017EE903A03F0010307EE903A9B00B8EEF7
:1093B000E70AE9E7F6EE007A37EEC00ADFED670A62
:1093C00020EE050A00F036FBF1EE402A4FE7F7EEFB
:1093D000007A37EEC00ADFED610A20EE050A0020B0
:1093E00000F058FDF0E7F7EE087A30EE670ADFED9F
:1093F0005B0A20EE050A00F01DFBB1EE400AE3E730
:10940000F0EE007A30EE670AE5E7012346E7644BA9
:109410009C4264D99FED637A33EE477A67EE074A40
:109420009FED616ADFED616ADFED615A9FED615A80
:109430009FED613A64EE877AE7EE866A9FED5F6A98
:10944000A6EEA76ADFED5E6AE6EE276A9FED5D6A2B
:10945000A6EEA76ADFED5C6AE7EEA65ADFED5B6A6F
:10946000E5EEA76ADFED5A5AE6EEA75ADFED596A34
:10947000E5EEA76ADFED585AA7EEA55ADFED575A79
:10948000E5EE275A9FED565AA5EEA75ADFED555A3D
:10949000E5EE275AE5EE876AA6EEE73ADFED527A67
:1094A00094EE863A33EE673A4EE7504B9C4206D92B
:1094B000B0EE007A37EE437A9FED280A0EE74C4B68
:1094C0009C4206D99FED4B7A9FED240A33EE477AF2
:1094D000A4E7F7EE007A33EE673A9FED200A9FED9E
:1094E000467ADFED467ADFED466AE3EE077A9FEDD6
:1094F000457AA7EE837ADFED447AE7EE037A9FEDB3
:10950000437AA7EE837ADFED4D7AE7EE037A9FED9B
:10951000407AE3EE076A9FED3F7AA6EE837ADFEDAD
:109520003E6AE7EE036A9FED3D7AA6EE837AF7EE98
:10953000006AE7EE036A67EE837A87EEA67AFEEEAC
:10954000006AF0EE477AE3EE267A37EE803A002D95
:10955000BFF65FAE32EE433A5BE600BF00000000AC
:10956000DB0F49406666663F1F4A3B3FA283D33705
:10957000679767393F239E3DA1549C3A7E02F23B98
:1095800001F0893D752C3C384584E23834B6053A03
:10959000C66E3D3B1599A83C661AA53E0000004BDF
:1095A00007336D3E0C5BEC3E6B7BA53976F4B7BAA6
:1095B00067F8663A85300DBA521CE63107E7C73BBB
:1095C000474D06BD5EB9F73E27F9A3B9FE7771BBDB
:1095D0003D37933C3C2117BEF7E9AF399916143B50
:1095E000FEFC28BC155A843DCDCDF83D17A6DD3FC5
:1095F0001FA69D3FC316BB3F5E3C5B3C78756A3E31
:10960000AF72D53DB24B7A3FE73ABA3FF400223F02
:10961000DBD5523BDFEF443F2D390840BE2E1D40C5
:1096200067FF0538B435F13ABDD7F536E440DA3C8A
:10963000E6DC153E7ACCA63E5A245C3E3F239EBD16
:10964000D6EE4B3A54BF983C6E0F303EC5D0383FF3
:109650003B2DB23FE8C4D5BAD23D5B3A5C061CBA9A
:10966000FD0C503A610B36BBABAAAA3D1D7FD63E1E
:1096700000000000B4F1824FF7EE002A75D2FDEE33
:10968000C35A1FED197A5FED196A1FED196AF8EEDA
:10969000E57A15EE903A73EE677A033BE7EE876A58
:1096A0001FED1E7AA6EEA77A5FED1F6AE7EE276A26
:1096B0001FED207AA6EEA77A5FED216AE7EE276A12
:1096C0001FED227AA6EEA77A5FED236AE7EE866A9F
:1096D0001FED246AA6EEA76A5FED256AE6EE276A0B
:1096E0001FED266AA6EEA76A5FED276AE6EE276AF7
:1096F00027EE277AE6EEA72A87EE223AB6EE007A20
:10970000A7EE873A042B3FF622AFDFE803F02B28C1
:1097100025220300B1EE087A37EE877AF1EE046A6B
:1097200077EEA66A66EE876AB1EE007A37EE877A40
:1097300027EE267AB0EE080A37EE800A20EE070AF6
:10974000B0EE007A77EE877A27EE800A23F0C0FE2B
:10975000FAE5B7EE007AE1E7F7EE006AE4E7B7EE84
:10976000007AE7E7B7EE000AEAE7B0EE430A23F033
:10977000AFFEB4F1B94F30EE620A24D2C2EE836A72
:109780005FED4C5A1FED4C6A66EEA67AB6EE007A93
:10979000A7EEA56A5FED4F5AE6EE275A1FED506A15
:1097A000A5EEA76A5FED515AE6EE275A1FED526A01
:1097B000A5EEA76A33EE477A1FED543AA6EE263A95
:1097C000A7EE003AC3E623EE003AC0E61FED583A92
:1097D000C0E61FED593A1CE5B4F17E5FF9D0B4F153
:1097E000804FF6D01FED5E2A63E500BF7FB510EE17
:1097F000105A834A25F000439342044605D80023BB
:1098000080ED000A4360002022E07E4A93423AD86D
:1098100025F00043002DDFED7C7A7C4A23F00F0316
:1098200018DD934230EE670A09BFDFED797A9FEDCC
:10983000797A9FED797A30EE670A70EE477A30EEEA
:10984000670AC0ED007A30EE470A80ED010A012078
:1098500004B070BD934230EE270A09BFDFED6C7A89
:109860009FED6C7A9FED6C7A30EE270A70EE077AE6
:1098700030EE670AC0ED007A30EE070A80ED010A8B
:109880004FF0FF30E4E7654A93426DD89FED647A6C
:10989000B0EEC00AF6EE007AE0EE077AFDEEE77A67
:1098A000F8EEE76A17EE900ADFED577AA6EEE70AC0
:1098B0001F28DFED587A66EEA77A30EE677A09DC6A
:1098C0005849461E25F0004251F8261022F0FF02AA
:1098D0008A4207D117EE102AC2F3C752C2EBD35205
:1098E000082A02DC84ED007A1BE09FED497AB0EE95
:1098F000406AA6EEC76A70EE467AE6EEC77A9FED3A
:10990000467AD6EE877A36EE677A17EE102AC2F3D9
:10991000C752C2EBE353192B15DC84ED007AB0EE8D
:10992000460A30EE470A002D30EE670A84ED010A40
:109930008EDAB1EE477AB1EE400A84ED007A84ED1A
:10994000010A404284E79FED387AB0EE460AA6EE5F
:10995000C70A76EE407AE6EEC77A9FED347AD6EE05
:10996000877A30EE677ABDE7B3F1FF4F06D330EE6A
:10997000400A80ED010A80ED000A44E7DA15863AD4
:10998000A3EBC25307EE903ABDEEE77ADFED286A0B
:10999000B8EEC77A77EEC77A8DED017A67EEA67AD0
:1099A000BDEEE77AB8EEC77A77EEC77A8DED027A28
:1099B00067EEA67AF5EE407AF1EE10FACDED037A75
:1099C00019D1B5EE407AF1EE10FA16D002232146F5
:1099D00001A800F089F8002DBFF63AAFD4ED007A67
:1099E000F1EE677AC4ED007AD4ED017AF1EE677A90
:1099F000C4ED017AA5E70323E9E70123E7E700BF08
:109A0000D80F493FE3CB1640800FC93FD00FC93F65
:109A1000004435374344353708A3852E800F49432A
:109A200084F9223F14620A0000A3852E32318D246E
:109A30000000804310EE103A23F00043B3F1485F7A
:109A4000B7EE007A04D2FDEEC07A17EE902ABAB3D0
:109A500060EE006ADFED1C5A9FED1C6A1C4AA6EE00
:109A6000A56A9342DFED1B5AE6EE265A9FED1A6A6D
:109A7000A5EEA66ADFED195AE6EE265A9FED186AA2
:109A8000A5EEA66A60EEC00A26EE266AF6EE007A19
:109A9000E6EE860A66EEA77A04D877EEE07A37EE2D
:109AA000670A70470F4A93429ABF03F17F4306EE5D
:109AB000903AF5EE026A37EE667A77EEE67AECE7F0
:109AC000B0EE470A704700BF4ED747ADF6740F316E
:109AD0009999993E7CF293B4010DD037610BB6BAD7
:109AE000ABAA2A3D0000483F2DE9F04F9246033AC9
:109AF00048BF0AF10402D7B0D2109B46551C2DB2C4
:109B000002910BF1FF31EB0080460DF16809501A0C
:109B10000BF1090CC24F0393AAEBC50500EB0C0631
:109B20004C460028AABF3B5CDFEDC17A07EE903AB5
:109B300000F10100A8BFF8EE677AB042E4EC017AC8
:109B4000EFD142AF08EB8B0309EB8B040193BE46C8
:109B5000DFEDB77A26464046F0EC016A019B36ED10
:109B6000017A9842E6EE877AF6D101318C45EEEC27
:109B7000017A04F10404EBD1A949DFEDAA6A9FED53
:109B8000AA6A531809240593A300049356AB03EB68
:109B9000840212ED140A07EB840006A92246002A6B
:109BA00045DC28463DF05AFFB0EE407AB4EE000A9C
:109BB00027EE000A1CF042FDF2EE007AA0EE677A72
:109BC000002DFDEEC77A17EE906AF8EEE77A37EED1
:109BD000677A3EDD06AA601EC5F1080E52F82030F5
:109BE00043FA0EF10E4401FA0EF1591A42F8201010
:109BF000C5F10702114100293ADD002201360DF1BD
:109C0000180E1346944255DC002D03DD012D62D061
:109C1000022D6AD002292BD1B7EE000A30EE477A26
:109C200033B328463DF01AFF37EE407A20E060EE6D
:109C3000267A013AFDEEE77AF8EEE77AA7EEC60A51
:109C4000BDEEC00AA1EC010A30ED010A37EE800A30
:109C5000A5E705D1621E06A951F822100912CAE72C
:109C6000F6EE007AB4EEE77AF1EE10FA20DA00218F
:109C7000B5EE407AF1EE10FA40F08480601E0023C9
:109C80000DF1180E082838DC002B56D10FA901223F
:109C900051F8040DB0B3049B3E1D04EB0B01601C96
:109CA0001E4409EB8101224490422DDD14466BE7EE
:109CB0000221A2E7DEF8000053B920B1C0F58070A0
:109CC000CEF80000012001320EF1040E034699E7A0
:109CD000C0F1FF00F4E704F1FF3E06A850F82E2083
:109CE00002F07F0240F82E2094E704F1FF3E06A820
:109CF00050F82E2002F03F02F4E75EF820200138F1
:109D00001343BFE70132C3E7059B1B5C07EE903AA4
:109D1000F8EE677A4446E1EC017ADFED457A8C464D
:109D2000F4EC015A019B3CED017A9C42E5EE877A06
:109D3000F6D1E6EC017A0130B6E7013C083D06AA0F
:109D400052F82430DBB12846B7EE000A3DF086FE1B
:109D50009FED347A381D4FEA840800EB84002346D7
:109D600006AD002B3CDA2346002B63DBDFF8BCE0BA
:109D7000DFED2F7A07EB830C0025E01A47E0013C6A
:109D8000083DDDE7039BB0EE470AA3EB0A003DF078
:109D900065FE9FED257AB4EEC70AF1EE10FA19DBE5
:109DA000DFED207A60EE277A06AAFDEEE77A083525
:109DB000F8EEE77AA7EEC70AFDEEE77ABDEEC00A35
:109DC00010EE103A42F8243017EE903A013442F87F
:109DD0002430B8E7BDEEC00A06AA10EE103AF6E746
:109DE00055F8232007EE902AF8EEE77A013B67EE5C
:109DF000807A20EE070A60ED017AB2E7FEEC016A94
:109E0000BCEC017A01350A2DE6EE877A01D0854255
:109E1000F4DD56AA02EB800040ED287A013BA3E76F
:109E200094620A000000803B000080435C630A00EB
:109E3000000000002FA81FED027A00EB0803224665
:109E4000002A17DAE1B1F1EE477A029BC3ED007AFE
:109E5000DDED2E7A77EEC77A01239C4213DA09B141
:109E6000F1EE677A029B06F00700C3ED017A57B066
:109E7000BDE8F08F73ED017A013A37EE277ADFE71C
:109E8000F0EE477AE1E7B0EC017A013377EE877ABA
:109E9000E3E700BF10EE103A23F00043B3F1485F50
:109EA00004D2FDEEC07A17EE903A5BB320EE007A52
:109EB000DFED157A9FED156AA7EE276ADFED147ABC
:109EC000E6EE077A9FED136AA7EE876ADFED127A56
:109ED00060EE076AE6EE077A30B99FED106AA7EEEA
:109EE000276AA6EE260A704767EEE67AB6EE006AA3
:109EF000E0EE867AD7EE870ADFED097AE6EEA70A6A
:109F000030EE600A704700BFD3C92E2F342FD7B26E
:109F10001BEF3836010D50B98988083CABAA2ABE20
:109F2000ABAA2A3E10EE103A23F00042B2F1465F8F
:109F3000F0EE407A14D2BDEEC07A17EE101A29BBAB
:109F4000431C134306D1F0EEC07AB7EE007A87EED9
:109F5000270A7047012800F09B80BFEE007AF6E7E1
:109F60004C498A4212D3002B9FED4B7AB8BFF1EED9
:109F7000407A37EE677ADFED497AB8BFF1EE600AD2
:109F800077EEE07ADFED460A77EE877A67EEA76A2A
:109F9000DFED445A9FED446A9FED445A3D4926EE59
:109FA000A67A67EEA64AA7EE256A8A42DFED405AF6
:109FB000E6EE075A9FED3F6AA5EE876ADFED3E5A4F
:109FC000E6EE075A9FED3D6AA5EE876ADFED3C5A43
:109FD000E7EE055A9FED3B5AA5EE875ADFED3A5A58
:109FE000E5EE075A9FED395AA5EE875ADFED385A4C
:109FF000E5EE075AB0EE467AA5EEA67AB0EE606AB4
:10A00000A7EE246A9FED337AE6EE260AE4EE870A8D
:10A0100037EEA00A1DD307EE100AF8EEC76A60EE0D
:10A02000005A30EE260A9B1785EE806A03F0020381
:10A03000C3F1010307EE103A36EE606AB8EEC77A54
:10A0400077EEC67AB0EE006AE7EEC66A26EE870AB9
:10A05000704701281CD010EE103A6FF30B0306EE88
:10A06000903A76EEE77A70EEE70AFFEE007A87EE36
:10A07000807AF7EE007A17EE103A6FF30B0300EEDA
:10A08000103AE6EE807AE0EE807AA7EE870A704713
:10A09000704700BF40A12C3FDA0F493F68212233AF
:10A0A000000000005FAE9BB745F4A3388453D93756
:10A0B000C8261A3A16696B3BA427B33C8988083E28
:10A0C0007AC09538B937813948DEBE3A1F37113C1E
:10A0D000D10D5D3DABAAAA3E42084B0802F05532B5
:10A0E00003F05533801AC91A8A08830801F0333106
:10A0F00000F0333002F0333203F033330344881876
:10A1000003EB131300EB101003F00F3300F00F30CC
:10A11000184400EB002000EB0040000E704700BF29
:10A120002DE9F04782B00646DDF828E00846B4463F
:10A130000D46002B4ED18A4214466DD9B2FA82F2F6
:10A1400042B1C2F12003954026FA03F394401D4327
:10A1500006FA02FC260CA7B2B5FBF6F14FEA1C4347
:10A1600006FB115543EA054301FB07F0984209D964
:10A17000E31801F1FF3580F00381984240F200813D
:10A18000023923441B1A1FFA8CFCB3FBF6F006FBC2
:10A1900010334CEA034C00FB07F363450AD914EB78
:10A1A0000C0C00F1FF3580F0ED80634540F2EA8051
:10A1B000A444023840EA0140ACEB030C0021BEF19C
:10A1C000000F04D02CFA02F30022CEE9003202B0D4
:10A1D000BDE8F0878B4209D9BEF1000F01D0CEE96E
:10A1E00000610021084602B0BDE8F087B3FA83F1B0
:10A1F000174600294DD1834202D3B24200F20F81AB
:10A20000B6EB070C60EB030301201D46BEF1000F07
:10A21000DDD0CEE900C5DAE7002A00F098801A46C2
:10A22000B4FA84F3002B40F0AF800B1B270CA6B2CE
:10A230000121B3FBF7F54FEA1C4007FB153340EA59
:10A24000034306FB05F8984507D9E31805F1FF30ED
:10A2500002D2984500F2E8800546A3EB08031FFAF6
:10A260008CFCB3FBF7F007FB10334CEA034C06FB06
:10A2700000F3634508D914EB0C0C00F1FF3602D251
:10A28000634500F2CE803046ACEB030C40EA05405B
:10A2900095E7C1F120058B4022FA05FC4CEA030C3E
:10A2A00000FA01F426FA05F3E84002FA01F943EA5C
:10A2B00004084FEA1C4206FA01FAB0FBF2F71FFA53
:10A2C0008CF602FB17004FEA184444EA004407FBEF
:10A2D00006F0A0420AD91CEB040407F1FF3380F01A
:10A2E0009C80A04240F29980023F6444241A1FFAE5
:10A2F00088F3B4FBF2F002FB104443EA044300FB92
:10A3000006F69E4209D91CEB030300F1FF3480F0EE
:10A3100082809E427FD90238634440EA0740A0FB16
:10A3200009749B1BA3423E46A04664D361D0BEF194
:10A33000000F0AD0BAEB060263EB080303FA05F537
:10A34000CA401543CB40CEE9005300213FE77308D4
:10A3500043EAC1734A08190C41EA02414FEAC67C3C
:10A360009BB2B2FBF4F02646A04627461F2243EAE2
:10A370000143B1FBF4F1A3EB080341EA004158E7C4
:10A380002946FFE6284615E71A46C3F120019C40FE
:10A3900026FA01F320FA01F190400343270C06FA54
:10A3A00002FCB1FBF7F0A6B207FB1015190C41EA4D
:10A3B000054100FB06F58D423BD9611801D28D4263
:10A3C00020D8491B0138B1FBF7F5019505FB06F8CC
:10A3D000019D9BB207FB151143EA0143434526D279
:10A3E000E31805F1FF31C6D24345C4D2A91E234468
:10A3F000C1E7BA459BD2B7EB090664EB0C04013800
:10A40000A04694E7651B29440238B1FBF7F5019596
:10A4100005FB06F8DCE720467FE71F4666E70846AF
:10A42000F4E6A44402382FE7023D234415E70199DE
:10A43000A1E7491BB1FBF7F5019505FB06F8C7E756
:10A440002DE9F0410D4606464FF029F8294640F225
:10A45000FE4058F0DBFC06F10807044690B1436863
:10A4600028469847A36801219B690546984710B183
:10A47000284846F055F9A368394628469B68BDE848
:10A48000F04118472449284657F0FAFD18B390F8D0
:10A490005030D906ECD443F0100380F850303946E0
:10A4A00053F0D2FB96F82A3003F00C03002B90F8FF
:10A4B000513014BF0122002223F0060343EA420375
:10A4C00080F8513005D190F8503043F0020380F805
:10A4D0005030BDE8F0811149284657F0D1FD0446BF
:10A4E000B0B190F82A309A07C2D443F0020339463B
:10A4F00080F82A3053F04BF996F82A1001F00C013D
:10A500000039204618BF0121BDE8F04153F026B9BB
:10A510000348AEE7AE460900FCC1090060C209006D
:10A52000A04609002DE9F7430746002608466A467B
:10A5300001A9019658F0EEF90199022902D82348A1
:10A5400046F0DAF87868012289001DF0C7FB7E60CA
:10A5500080463E81019BB4B2A34206D85B00C7F897
:10A5600004803B8103B0BDE8F083009B184953F899
:10A57000245040F2E942284625F040FC686840F249
:10A58000E942022125F0F8FBA86840F27A6125F043
:10A5900063FC40F27A6347F6FF720E49814656F03B
:10A5A000DEFEE8684FF4D06125F056FC09494FF40F
:10A5B000D06347F6FF72054656F0D1FE28F8249086
:10A5C00008EB840401366580C4E700BF47440900F6
:10A5D0005C2509000080FFFF2DE9F04F2DED028B77
:10A5E00091468DB0C268BDF864B0DDF86880BDF8F2
:10A5F0006C501D9C07468A461E46B0EE408A2AB122
:10A6000043689A4200F0B8800FF0DCFC4BEA050387
:10A610001F2B09D8BAF1000F7BD1002D00F0A580C7
:10A6200054464FF0040A09E0BAF1000F40F092805E
:10A63000002D00F0938054464FF0080AB9F1000F46
:10A6400000F0978040F20122ADF81820721CADF89E
:10A650001A200022079206A85FF03EFC81460028DF
:10A6600051D1182201460DEB020056F0F9FCDFED46
:10A67000447A9FED447A444B8DF818A028EE278A3F
:10A680005E43C8EE077A42F210734D4508BFC846D4
:10A69000B6FBF3F64846189BADF8246001260794F4
:10A6A0008DF82D600293ADF80CB0CDF81080ADF8A8
:10A6B0001450B6EE007A77EE877AFCEEE77ACDEDAD
:10A6C000087A4DF0EFF98146E8B9304C06AA02A9A4
:10A6D00020465FF0DBFB8146A8B92D493A4607F1D9
:10A6E00028000AF05DFE9DF97020217830465FF069
:10A6F000FDFB814638B9207831465FF0C9FB8146C1
:10A7000008B9189BFB6048460DB0BDEC028BBDE854
:10A71000F08F3CB3F0EE0C7AB4EEE78AF1EE10FA6B
:10A720006946204610D807EE906A9FED1A7AF8EE37
:10A73000677AF4EEC77AF1EE10FA05D84CF06EFEA7
:10A740006C464FF0020A79E74CF068FE6C464FF019
:10A75000030A73E700244FF0060A6FE72C464FF018
:10A760000A0A6BE74FF0010A68E72C464FF0050A2A
:10A7700064E7CDE906996EE74FF01109C3E700BF22
:10A780000024744900401C4440420F00B7050120DA
:10A79000897B07006666A63F2DE9F843416099462C
:10A7A0004B680B9F90469A790A9B80F82C20038572
:10A7B0008D7D044605F0300605F0060572B34B6842
:10A7C000D8684EF080F9E0842DB10023C4E90289F5
:10A7D000C4E90433A361002384F82D3084F82A30BF
:10A7E000A384089BE361099B23621AB3EFB11B4961
:10A7F000224638460AF0D4FD5DB115F0040118BFB9
:10A80000012160681ABF84F82B10002201220FF08A
:10A8100073FDDEB1B20616D4012315E04FF6FF73C7
:10A82000C3842B4635461E46CEE70C4821460AF027
:10A830009BFDE1E767B10A49224638460AF0B0FDC0
:10A8400026B17307E8D4022384F82B30BDE8F883DF
:10A85000034821460AF088FDF2E700BF7D87080023
:10A86000E78708002DE9F04F89B081469DF84860E0
:10A8700015465FFA81F81C46002B36D043681A79DA
:10A880001B680621C3F800151D4B342101FB023360
:10A8900086F00106022283F82D207201194E4FF036
:10A8A000000AB4F5806F274603A928BF4FF48067DC
:10A8B0004846CDE9047ACDE9065A8DF80CA08DF80A
:10A8C0000D80019200F0C2FDB042834603D1E41B2B
:10A8D000019A3D44E5D1D9F8040035F003FC58460F
:10A8E00009B0BDE8F04F45F0FDBA41460FF04AFF10
:10A8F000A0420CBF6FF01200204609B0BDE8F08FF7
:10A90000985C01200000AD0B074A002311688142CA
:10A9100001D1184670470133082B02F10402F5D12A
:10A920004FF0FF30704700BF0C4701200C4B1878E8
:10A9300001280DD10B4B1B78FF2B0BD10A4B18684C
:10A94000C20708D4C30308D4800C00F00400704789
:10A950000228F3D17047052070470120FAE700BFB5
:10A96000BC690120C46901207C6101202DE9F0410E
:10A97000094D0746884600244FF6FF7635F8140047
:10A98000B04203D0424639465FF0D2FA4434B4F5BF
:10A99000AA7FF3D1BDE8F081A0090120034B53F851
:10A9A000203013B19A6801329A607047E420012088
:10A9B00038B5144B53F82040ECB1207935F04EF8FF
:10A9C0000546607935F04AF8A2790F49E37940EA03
:10A9D000450000F0030040EA8202A0718A5C134443
:10A9E00094F908205BB29342E37105DBE36801331D
:10A9F000E3600023E37138BD52429342FBDCE3681D
:10AA0000013BF5E72C470120291D0A002DE9F04FF5
:10AA10000546A7B08A460146002058F0F7F909AC70
:10AA2000002841D1CDE913000CAA7E21284629F047
:10AA3000E1FCA94B0F9301224023CDE9102316AB73
:10AA400012930FAB0E93A54B09940A93002608208E
:10AA5000CDE9050656F00BFA07902046CDE90366CE
:10AA60008DF8206055F0AAFEDFF880B237463546F3
:10AA70009DF85490B9F1000F13D0204655F09EFE7A
:10AA8000B9F15D0F00F092804AD8B9F13A0F3BD886
:10AA9000B9F11F0F14D8B9F10A0F31D8B9F1080F65
:10AAA000E6D88F4845F03CFE0121284628F096FE66
:10AAB00043680A93002309950B938DF85430C5E73A
:10AAC000A9F12002D2B20123934013EA0B0F40F008
:10AAD0000F81844A1340CBD1B9F1220FE1D1069303
:10AAE0009DF854100029DCD0222940F0A480204693
:10AAF00055F064FEDDE906102CF080F881462CE06C
:10AB0000B9F10D0FB4D0CCE7B9F15B0FC9D100207A
:10AB100022F032FA8146002D3AD04FF0010821E0B0
:10AB2000B9F1740F70D039D8B9F1660F4FD0B9F1BF
:10AB30006E0FB6D19DF85430752BB2D1204655F02A
:10AB40003DFE6C28ADD1204655F038FE6C28A8D1CA
:10AB5000204655F033FE4FF00E09002D00F00E8117
:10AB60004FF00008604B9F4240F0F5804946284670
:10AB700057F09AFEB8F1000F3FF47AAF049B002B18
:10AB800040F0F780012101A82BF00CFE049B1D6012
:10AB900048462AF01FFF4D46074669E7B9F17B0F8B
:10ABA00000F0D580B9F17D0F7FF47BAF002D3FF42D
:10ABB00078AF039B002B00F00081013B049A0393C4
:10ABC00052F8235028462AF005FF074650E79DF823
:10ABD0005430612B7FF465AF204655F0EFFD6C28B3
:10ABE0007FF45FAF204655F0E9FD73287FF459AF3D
:10ABF000204655F0E3FD65287FF453AF204655F01D
:10AC0000DDFD4FF01E09A8E79DF85430722B7FF44C
:10AC100048AF204655F0D2FD75287FF442AF20465C
:10AC200055F0CCFD65287FF43CAF204655F0C6FDBD
:10AC30004FF03E0991E75C290CD1204655F0BEFD4E
:10AC40007528014606D86D2808D8622840D06628A5
:10AC500008BF0C2105A862F0E6FB35E0A0F16E0309
:10AC6000072BF7D801A252F823F000BF8DAC0200E9
:10AC700055AC020055AC020055AC0200D5AC020048
:10AC800055AC020091AC020095AC02000A21E1E74C
:10AC90000921DFE74FF000084FF00409204655F086
:10ACA0008DFD40F02000A0F130025738D2B2C0B282
:10ACB000092A88BF0246B9F1010942EA0818EDD114
:10ACC000414605A862F0C1FB204655F077FD07E735
:10ACD0000821BFE70D21BDE77C5A09006F07080076
:10ACE000A631090001100004E85909000020FF0303
:10ACF000002306939846494605A862F094FB9DF808
:10AD00005490B9F12E0F17D009F0DF03452B13D063
:10AD1000B9F12B0F12D0B9F12D0F0FD0484645F0E5
:10AD200037FC024650B9DDE90610B8F1000F09D032
:10AD3000134657F0D9FFE1E64FF00108204655F0E1
:10AD40003DFDD8E743460A222DF00EFED6E6002050
:10AD50002BF0FAFDDEE62EB9B8F1000F7FF4A1AEBC
:10AD60004E4685E631464A46284657F0E2F9002627
:10AD700000E7294601A857F097FD09E7BAF1000F4F
:10AD800011D0B9F1000F3FF48CAE039B002B7FF480
:10AD900088AE05A862F0BEFB484627B0BDE8F08F3C
:10ADA000204655F00BFD9DF85450284645F004FC14
:10ADB0000028F5D1002DE4D073E6A946BAF1000FC2
:10ADC000F1D0E2E7C20713B5044603D5C0F347004C
:10ADD00002B010BD830707D102680E4B9A4203D11F
:10ADE0002AF0E6FDC0B2F3E7204657F02AFD48B14D
:10ADF00020462AF065FDFCEEC07ACDED017A9DF883
:10AE00000400E5E720462AF0E5FD5E22C1880248FD
:10AE100045F07AFC202F0900273D09002DE9F04F6D
:10AE20000546E3B058484EF044FE061E09DB574C79
:10AE30006388B3F57F7F08D340F2512323803DF030
:10AE400077FA002063B0BDE8F08F1A1DAA4200F225
:10AE50009880591E251D4E486A5C2F2A4FF000022B
:10AE60000CBF6A54EA5405A954F0D2FA494B07467C
:10AE7000186010B11BF09CF820B940F251332380C8
:10AE80003046DCE707F18000059A06A953F057FC2D
:10AE900040F2511345F8043C0023C4E9013307464E
:10AEA000E36010B103236370EAE71AAD294606A8F0
:10AEB00053F031FD08B9AB7E93B9002106A853F0D9
:10AEC0002AFD4FF00009A7604F450FD106A853F0A7
:10AED00037F90023A26863806260E360A361CFE773
:10AEE000294606A853F017FD0137E3E7294606A8CF
:10AEF00053F011FD6B892989C4F8049003F01F02F7
:10AF00005200480A0192C3F344120092DB0A01F096
:10AF10001F0200F2BC70C1F3431161F03DF91E4BFA
:10AF2000A0FB0303C4E904032B7B13F0100318BF39
:10AF300001230DF1820B15BFE360E36000232B6852
:10AF4000A361584660F09AFA6080824630463DF030
:10AF5000EFF94FF00008C24502D809F10109B3E743
:10AF6000AAEB0802042A4FF0000328BF04220BEBCF
:10AF700008010548009303920FF09CFA039A90444D
:10AF8000E9E701205EE700BF18500120D4510120FD
:10AF9000D8510120DC50012000CA9A3BF8B5284B5B
:10AFA0001D68284B1B681A68012151641B68264ADA
:10AFB000D3F844650023146814B12179814230D05C
:10AFC0000133082B02F10402F5D1F8BD6369A069D1
:10AFD000E289218AEB1A89B211FA82F2301AA18928
:10AFE000B2FBF1F7C3EB034303444FF6FF7001FBE1
:10AFF00017228342A16828BF034621F81230238A12
:10B00000A2899BB2934203D2238A0133238214E0A4
:10B01000E3899BB20133B3FBF2F102FB1133E3810D
:10B020000BE0E379002BD1D034F018FD637900F008
:10B030000100834201D00023E3716561A661C4E78A
:10B040006C6101201C6301200C4701202DE9FF41A8
:10B0500004460F464EF023FA6368DB6853F8275026
:10B0600040F2FE40294657F0D1FE064600285CD04B
:10B07000436828469847B36801A95B6880469847AB
:10B08000B36800219B68054640469847B368002195
:10B090009B694046984763682849DB6853F8270056
:10B0A00056F0EEFFC0B190F85030B0F9382023F0E0
:10B0B000100380F85030B0F93C309A421FBFADF811
:10B0C0000830C38F826BADF80A304FF000031ABF0F
:10B0D000019201250025836263681949DB6853F8F2
:10B0E000270056F0CDFF064668B190F82A3023F0CD
:10B0F000020301A980F82A3017F01AFD0021054645
:10B10000304652F044FB6DB194F82A30DB070ED480
:10B11000019BA361029BE36194F82A3043F0010391
:10B1200084F82A3004B0BDE8F0810546B3E704F1A5
:10B13000180201A9104651F0F6FCEDE7FCC1090028
:10B1400060C209002DE9F74F404B019000201870B4
:10B150003F4BDFF820A1DFF820C1FF2002EB81097F
:10B1600018703C493C48144615464FF001084FF012
:10B17000FF32A94520D1013204D0019B002B51D1CF
:10B1800014F08CFB354E364800220023C6E900231C
:10B1900000231A46A5424BD15AB193ED017ADFED57
:10B1A000317A67EE277A17EE900AFDF7F1FFC6E9CC
:10B1B000000103B0BDE8F08F55F8047BBB07D8D180
:10B1C0003B685345D5D17B681A79A2F12003C2F1BF
:10B1D000200628FA06F608FA03F333433E7A08FA03
:10B1E00002FEAEB1DCF804600096DCF8006046EACE
:10B1F0000E0B009E1E43CCE900B67E7A002EB8D01E
:10B20000D1E9007647EA0E071E43C1E90076B0E7B0
:10B2100046680096066846EA0E0B009E1E43C0E98B
:10B2200000B6EAE7104A00231360104A1370A9E73A
:10B2300021688F0708D10F68874205D112B10C48E9
:10B2400045F06EFA0B4601220434A3E7BC690120E5
:10B25000C4690120200D0120100D0120280D0120BE
:10B26000E08A090000007A447C61012070690120B5
:10B270009A440900FC8A0900000D0120242B2DE9C5
:10B28000F047884601D8012B06D1FDF77BFF162336
:10B2900003600020BDE8F087344E0D46294615F8BE
:10B2A000014B375D17F00807F8D12D2C10D12C7801
:10B2B00001278D1C33F0100115D1302C0DD12978C8
:10B2C00001F0DF01582908D16C78023510230AE01B
:10B2D0002B2C04BF2C788D1CECE7002BF6D1302CE6
:10B2E00014BF0A23082307F1004E0EF1FF3E002190
:10B2F000BEFBF3F90E4603FB19EAA4F1300CBCF1D6
:10B30000090F10D86446A3421EDDB1F1FF3F07D0FC
:10B31000B14516D301D1A24513DB06FB034601213B
:10B3200015F8014BE9E7A4F1410CBCF1190F01D864
:10B33000373CE8E7A4F1610CBCF1190F04D8573C85
:10B34000E1E74FF0FF31EBE74B1C05D1222303600F
:10B35000764632B930469DE707B17642002AF9D0E9
:10B3600009B105F1FF38C2F80080F3E7297A0A0035
:10B370002DE9F043344E86460D46284615F8014B1C
:10B38000375D17F00807F8D12D2C10D12C78012744
:10B39000851C33F0100015D1302C0DD1287800F029
:10B3A000DF00582808D16C78023510230AE02B2CD6
:10B3B00004BF2C78851CECE7002BF6D1302C14BF91
:10B3C0000A2308234FF0FF380026B8FBF3F803FBED
:10B3D00008F96FEA09093046A4F1300CBCF1090FF5
:10B3E00010D86446A3421EDDB6F1FF3F07D080456A
:10B3F00016D301D1A14513DB00FB0340012615F84C
:10B40000014BE9E7A4F1410CBCF1190F01D8373C1D
:10B41000E8E7A4F1610CBCF1190F04D8573CE1E74F
:10B420004FF0FF36EBE7731C06D12223CEF8003035
:10B43000304632B9BDE8F08307B14042002AF9D066
:10B4400006B1691E1160F5E7297A0A002DE9F74F68
:10B4500080460D46019260F006F9D8F80430AC4FF2
:10B4600001225A72D8F804301E791C68342303FB79
:10B470000677002387F82E30EB6803F06043B3F1C2
:10B48000005F81468B4607D0A248D8F804300022DE
:10B490005A7203B0BDE8F08F9F4BC4F8083397F899
:10B4A0002F3003F0FF0A23B1BB689C48C4F8043373
:10B4B000EBE787F82F20AE46BEE80F0007F10C0C33
:10B4C000ACE80F00DEF80030CCF8003087F830A090
:10B4D0006B78C4F888354FF4827120465CF088FFA1
:10B4E0004FF4927120465CF083FFC4F850A5C4F875
:10B4F00040A52B78032B00F2B380DFE803F0729AAB
:10B5000052022B6903F06043B3F1005FBCD14FF4EA
:10B510008073C4F800326B68EA68C4F844254FF4BD
:10B52000A871C4F8483520465CF062FF4FF4B07152
:10B5300020465CF05DFF4FF4A47120465CF058FF9C
:10B5400001232362A360D4F85031002BFBD04FF4C9
:10B55000A87120465CF04CFFAB682A69C4F844250A
:10B56000C4F848356A4B342202FB06336C4A9A60B1
:10B570004FF4827308226B4F2978654D03291CBF55
:10B580000121A15034227243A918AA58002A79D067
:10B590008B68C4F80433634B9F4200F0A880624874
:10B5A00073E76B68EA68C4F84425C4F848352B692A
:10B5B00003F06042B2F1005F7FF466AFAA68C4F89E
:10B5C00034354FF48453C4F83825C4F80032504B56
:10B5D000342202FB063340F202229A6001232362E6
:10B5E000C6E701996B68EA68C4F84425C4F8483591
:10B5F0003422474B89B102FB06334FF48071C4F803
:10B600000012474A9A604FF4A47120465CF0F0FEA5
:10B610004FF4A47301222262ACE702FB06334FF41D
:10B62000007140F20222C4F800129A604FF4827353
:10B63000F0E76B68EA68C4F83425C4F838354FF48D
:10B640008053C4F80032324B342202FB063340F2FE
:10B6500002229A600123236200224FF482738AE758
:10B66000314F4FF48273082286E7D4F8242152B177
:10B670004FF4927120465CF0BBFE012323626361AC
:10B680004FF4827323441A68002AEED03422D4F88F
:10B69000C434C4F8C43402FB0651002281F82F20C0
:10B6A0008BB1224A224813F0010F08BF104613F055
:10B6B000020F02F5803218BF104613F0040F1D4B25
:10B6C00018BF1846E1E6204648F012FD00287FF436
:10B6D00062AF1648D9E65FF0C6FF814574EB010101
:10B6E00009D2D8F80430144800225A72D1E619F56C
:10B6F0007A794BF10004D8F804305A7A002AEAD15A
:10B700009B7A042B96BF0D4A084852F82300C0E6E6
:10B71000985C01200A00AD0B02029C010B00AD0BEE
:10B72000000204000000AD0B0400AD0B0100AD0BE6
:10B730000000AE0B0200AE0B0700AD0B701E0A003E
:10B74000F8B590F82A309B0704462DD4F8BDDB6885
:10B7500053F8256040F2FE40314657F057FB07464C
:10B7600068B1436830469847BB6804F108019B689C
:10B770009847013563689A689542E8D3E6E70B4934
:10B78000304656F07DFC20B104F1080152F05CFA1D
:10B79000EFE70749304656F073FC0028E9D004F182
:10B7A000080151F0F4FFE4E70025E3E7FCC10900DC
:10B7B00060C2090090F950301F4A10B5002B836A0F
:10B7C000B4BF418A018AB0F90C40002B08BF134670
:10B7D0000C44997B8289B9B193F9051011FB02F1F0
:10B7E0005A88114409B2A0F8461093F905205B88E5
:10B7F00012FB04331BB29942D2BFA0F84A30A0F822
:10B800004A10A0F8463010BD93F9041011FB02F164
:10B810001A88114409B2A0F8441093F904201B8837
:10B8200012FB04331BB29942D2BFA0F84830A0F8F3
:10B830004810A0F84430E6E7A005012090F9503008
:10B840001F4A10B5002B836AB4BF018A418AB0F940
:10B850000E40002B08BF13460C44997BC289B9B136
:10B8600093F9041011FB02F11A88114409B2A0F8EF
:10B87000441093F904201B8812FB04331BB2994235
:10B88000D2BFA0F84830A0F84810A0F8443010BD4E
:10B8900093F9051011FB02F15A88114409B2A0F87E
:10B8A000461093F905205B8812FB04331BB29942C2
:10B8B000D2BFA0F84A30A0F84A10A0F84630E6E718
:10B8C000A005012008B510EE103A23F00042B2F1B5
:10B8D0007E5FF0EE405A10D308D19FED2F0ADFEDC6
:10B8E0002F7A002BB8BFB0EE670A08BD70EE405A41
:10B8F000DFED297A87EEA50AF7E7B2F17C5F11D276
:10B90000B2F14A5F9FED266A42D920EE000AFCF7A9
:10B910007FFEDFED247AE0EE657A75EEE75A36EECB
:10B92000650AE2E7002BB7EE000AF6EE007A14DAB9
:10B9300075EE805A25EEA70AB1EEC06AFCF768FEE4
:10B94000DFED197AE0EE067A9FED150A77EE867A3A
:10B9500030EE670A30EE000AC7E730EE650A20EEE7
:10B96000270AB1EEC05AB0EE407A15EE103A6FF3E6
:10B970000B0305EE903AA5EEE57A75EE257A87EE93
:10B98000276AFCF745FEA0EE056A36EE250AE1E7D8
:10B99000B0EE460AA9E700BF00000000DA0F4940F8
:10B9A000DA0FC93F6821A2336821A2B308B510EEAF
:10B9B000103A5A00F0EE407A0FD4B7EE007A70EEEB
:10B9C000477ABDE8084037EEA77AA7EEA77AB1EE2E
:10B9D000C70A37EE800A21F0CFBC23F00043B3F151
:10B9E0008B4F13D2FFEE006AE0EE006ABDE808401C
:10B9F000B1EEE67AF7EE006A37EE007A86EE870A55
:10BA0000B0EE007A97EE870A21F062BD21F060FD6A
:10BA1000DFED027A30EE270A08BD00BF1872313F11
:10BA200030B589B0084611461A4602AB0193194B4E
:10BA30000093032355F060FC1749029D0C2056F03B
:10BA4000C0FF9DF80C30037245609DF8103004462D
:10BA5000EBB128460DF0A2FE606805AA40F2F7415E
:10BA600028F0C8FC237A5B0043F0010305AA0021FB
:10BA70000120079355F089FD56F0EFFE05466068FA
:10BA80004DF0A6FE1DB9217A044844F051FE20462F
:10BA900009B030BD84200A0038C90900C445090036
:10BAA00010B58EB003AB51F8044B0193194B0093C2
:10BAB0000138032324F0BCF840F21B51606806AA49
:10BAC00028F098FC237A5B0043F001030893039B62
:10BAD000099340F626130A93049B5B0043F001038D
:10BAE0000B93059B6FF0004293421FBF40F2E6426A
:10BAF0005B000C9243F0010314BF0221012106AA4E
:10BB00004FF0020018BF0D9355F03FFD0E200EB010
:10BB100010BD00BF6C200A0010B58EB003AB51F809
:10BB2000044B0193194B00930138032324F080F850
:10BB30004FF4CF61606806AA28F05CFC237A5B00B2
:10BB400043F001030893039B099340F626130A93DD
:10BB5000049B5B0043F001030B93059B6FF00042D5
:10BB600093421FBF40F2E6425B000C9243F0010398
:10BB700014BF0221012106AA4FF0020018BF0D9345
:10BB800055F003FD0E200EB010BD00BF54200A007A
:10BB900010B596B003AB51F8044B01932D4B0093B5
:10BBA0000138062324F044F809AA606840F279615C
:10BBB00028F020FC237A5B0043F001030B93039BE6
:10BBC0000C93049B0D9344F636430E93059B5B0048
:10BBD00043F001030F93069B6FF00042934235D070
:10BBE0005B0043F0010344F60642119310920923CF
:10BBF000032116AA02EB830244F2F60042F8340C49
:10BC000016AA02EB8300079A520042F0010240F8A4
:10BC1000302C089A6FF00040824210D016A800EB3A
:10BC2000830044F2C60440F82C4C16A800EB8303B2
:10BC3000520042F00102013143F8282CC9B209AA8E
:10BC4000032055F0A2FC0E2016B010BD07230221E0
:10BC5000CFE700BF24200A00F0B58BB0084611469C
:10BC60001A4603AB01931B4B0093072355F044FB8B
:10BC7000DDE903600E2816D010F0030203D101683D
:10BC8000154B99420CD029F0A5FEC38800931348A8
:10BC900040F28F134FF4917240F2FF2144F034FDD3
:10BCA00001214EF01BF80E49182056F08AFE9DF82F
:10BCB00020409DF824109DF81C50069F049A9DF882
:10BCC00014300573C0E90167447381730261037521
:10BCD0000BB0F0BD24210A0038C30900B64D09009D
:10BCE0001CC9090030B58BB004466A464068244D33
:10BCF00040F2226128F07EFB00216A46084655F09A
:10BD000044FC56F0AAFD002831D060686A4640F233
:10BD10001F3128F06FFB42F6D6330293A3685B0015
:10BD200043F00103039344F6B6630493237B5B0063
:10BD300043F00103059344F6B6530693637B5B001F
:10BD400043F00103079342F6C6421123CDE90823CD
:10BD500004216A46002055F018FC23690E2B03D0FD
:10BD6000217D58684DF0A6FF60680BB030BD04F02F
:10BD700079FDAB6A002BBFD0012027F055FEBBE751
:10BD8000745D01202DE9F341054601F134000E46B2
:10BD900004F02CFD2B88102B05D0112B41D0002056
:10BDA00002B0BDE8F081314C002388224FF6FF71CC
:10BDB00002FB03F7E05B884205D00133052BF7D186
:10BDC0004FF40877042388225343A988E152E218EC
:10BDD0004FF000080E2307F16000D365204424498A
:10BDE00082F85A80A2F87680E21909F0D9FAC6F8EA
:10BDF0001880286969696C373C4403C468465EF062
:10BE000067F8BDF800302A8A9A4202D86A8A9A42B4
:10BE100003D2A88869465EF043F80023F36001204E
:10BE2000BEE7AB88114F0024882202FB04F1785A48
:10BE3000984205D00134052CF7D14FF40871042441
:10BE400039440B4809F0C2FA88235C433A194FF68B
:10BE5000FF733B53002382F85A30D26D0E2A1EBF67
:10BE60005360297A1172B361D9E700BFA00901209C
:10BE7000C5F903002DE9F0418AB0084611461A467B
:10BE800005AB0193234B0093052355F035FA0522AA
:10BE9000059802A927F050FC039EA6F11002102A73
:10BEA00003D81D4BD340DB0702D41C4844F038FCB8
:10BEB000069C022C04DC002C04DC194844F0D4FB62
:10BEC000062CFAD10798DDF80880A0B90746154975
:10BED0004FF48A7056F075FD089B80F80C41C0F84D
:10BEE000103132463B46414605464DF029FD284675
:10BEF0000AB0BDE8F081012202A927F01DFC00284C
:10BF0000E4D0039840F26512102123F035FF029F20
:10BF1000DDE700BFCC200A0001010100C74609008F
:10BF200081430900D8C8090070B588B003AB51F847
:10BF3000045B0193184B00930138022323F078FE31
:10BF40000522039805A927F0F7FB069CA4F110022F
:10BF5000102A03D8114BD340DB0702D4104844F019
:10BF6000DFFBDDE9040640B9034628462246314698
:10BF70004DF0E6FC0E2008B070BD012205A927F0A7
:10BF8000DBFB0028F0D0069840F26512102123F068
:10BF9000F3FE059BE9E700BFBC200A000101010098
:10BFA000C746090010B50446084656F037F902287E
:10BFB00004DC002804DC044844F056FB0628FAD1CF
:10BFC00084F80C010E2010BD814309001FB503AB9E
:10BFD00001930F4B0093054601230E46002023F0EA
:10BFE00027FE3146284646F04DFD03982AF0ACFB6B
:10BFF000441004D0074840F2F34144F03DFB294689
:10C0000001203246FFF79EF80348214660F032FED9
:10C01000B8210A00914E090094210A0070B5054626
:10C020000E46002844D046F02DFD32462946002019
:10C03000FFF788F800F0A4F900231A4641F08AFEC1
:10C040001C4B9C6A94BB4DF09AFC78B3FEF76EFCD7
:10C05000012818D002280BD1174A234656F823404E
:10C06000A10702D12168914203D001339D42F5D14D
:10C070000E2420463CF05EFD00F060F820463CF0C7
:10C0800059FD204670BD0D4B0D491A78234656F8D0
:10C090002340A00706D12068884203D16068007958
:10C0A0009042E6D001339D42F1D1E1E70E24E3E76F
:10C0B0000E24E6E7745D0120E08A0900C4690120CE
:10C0C000FC8A090010B586B0084611461A4602AB34
:10C0D0000193114B0093042355F00EF940F2DF4118
:10C0E000029846F097FC0D4904460C2056F069FC76
:10C0F0009DF8102012B10A4844F012FB22792F2A31
:10C1000001D95DF0F4F89DF814209DF80C1001722F
:10C110004460427206B010BD74210A00FC8A090016
:10C12000234A090010B5044C23781BB913F0B6FB61
:10C130000123237010BD00BF70690120F8B5344C95
:10C14000344A23686FF3172393421CD04FF4807254
:10C150000021314854F084FF304A00231370304AE4
:10C160004FF4403113701A0102F180420133082B61
:10C17000C2F80419F7D14FF080434FF47C12C3F892
:10C180008429244B2360274E274D0024D5E9000144
:10C19000D6E90032C4F1200703430A430120A4F189
:10C1A000200100FA01F120FA07F73943A0400340CB
:10C1B0000A40134308D0E0B23AF050F8204633F07A
:10C1C00063FD204633F048FE0134402CDED1174990
:10C1D000174800220023C6E90023C5E90023C1E96E
:10C1E00000234FF40033C0F84833D0F804239203FF
:10C1F00008D5C0F80833D0F844311BB14FF4A27110
:10C200005CF0F6F80B4B00200021C3E90001F8BDFB
:10C21000C0690120AF0000ADC5690120BC690120E3
:10C22000C4690120000D0120100D0120200D012006
:10C2300000400240280D0120F0B50E4687B00025D1
:10C240001446002A5ED08A075FD10A68414B9A42A1
:10C250005BD16A464FF4807056F015FF10B93E4826
:10C2600044F002FADDE90035042CA5EB030536D0D5
:10C27000A30732D12368394A934208D0384A9342FF
:10C2800005D0384A934202D0374A934225D105223D
:10C2900003A9204627F050FA049BAB4202D0334852
:10C2A00044F03EFA9DF81410039C0022402023F035
:10C2B00003FE012801D02E48F2E7009B5A19B2F57F
:10C2C000807F07D82B482A462146184454F087FE21
:10C2D0000E2417E0284844F0F1F92848C0E7284622
:10C2E00054F0C5FD009B5A19B2F5807F044604D86E
:10C2F00020492A46194454F072FE214628462AF065
:10C30000D3FA0446204607B0F0BD32460068002349
:10C310004FF4807127F02EFA042C064600F1010735
:10C3200008D1B7F5807F9CBF124B1D5C6D0045F0B6
:10C330000104E7E7204655F071FF4223FF22002168
:10C34000044655F00CF8B7F5807FC3D8094B9C55CF
:10C35000BEE700BFCC58090037340900406209002D
:10C360007C5A09009C590900485E09002D430900C8
:10C37000B84B0900C5690120FB4009006B3E09006C
:10C3800038B5084BD3E9004554EA050305D05FF002
:10C390006AF9201A65EB010138BD4FF0FF30014604
:10C3A000FAE700BF280D012010B52DED028B88B0F3
:10C3B000084611461A4603AB01932D4B0093022306
:10C3C00054F09AFFDDE90304B0F10E0218BF012218
:10C3D000B4F10E0318BF01239A4202D1254844F05C
:10C3E0009FF90E2836D029F06BFAB0EE408A5FF044
:10C3F0003AF9FBF7EFF8DFED207A07EE100A0E2C82
:10C40000C7EE278A1FD0049856F0A9F804463AF0E0
:10C41000A1FE05A93EF030FF9DF81A3001939DF86A
:10C42000193000939DF817209DF818309DF81610CC
:10C43000BDF8140042F040FC231A08EE103AB8EEA2
:10C44000C88A38EE288AB4EEE88AF1EE10FA04D5EC
:10C450000A48C4E79FED0A8AC9E70A49082056F04E
:10C46000B0FA80ED018A08B0BDEC028B10BD00BFB0
:10C4700064210A00DF42090000007A4400420900FA
:10C4800000000000E08A09001FB5084611461A4660
:10C4900003AB0193084B0093012354F02DFF40F2AE
:10C4A000DF41039846F0B6FA0449082056F089FAAD
:10C4B000002044F0D9F800BF5C210A00C48A0900BA
:10C4C00010B5094B094C1B6823B1A34202D00848A0
:10C4D00044F0F4F8C0220021064854F0C1FD054B99
:10C4E00043F8044C181F10BDF8550120A060090046
:10C4F000CF410900FC55012010B5084C20681EF002
:10C500009FFB014610B1064844F0D8F8B422201D24
:10C5100054F0A6FD034B2360204610BD480C0120BB
:10C52000C8410900A060090038B51C4608461146FC
:10C530004FF0021223F044FB206840F2DF4146F046
:10C5400069FA09490446082056F03BFA6379054622
:10C550000BB95CF0CCFE207933F01EFA20790CF098
:10C560000BFF6C60284638BD54C8090008B5406808
:10C570004CF066FFBDE808409FED010A2AF04EBA74
:10C580003333534037B5054640684CF059FF304AC5
:10C5900000230321ADF80630C2F8F0150121C2F8DE
:10C5A000F435C2F8001519461A0102F1804202F56D
:10C5B000E0420133082BC2F81415C2F81015F3D16C
:10C5C000234C4FF49053C4F818356B685B79C4F86A
:10C5D0001435C4F810350DF10603C4F82C360123C8
:10C5E000C4F830362360D4F80031002BFBD0184853
:10C5F0004FF480715BF0FCFE01236360144CD4F8AF
:10C600000431002BFBD012484FF482715BF0F0FE36
:10C610000123A360D4F81431002BFBD00C484FF455
:10C620008A715BF0E5FE0023C4F80035C4F81435C8
:10C63000C4F81035BDF9063023EAE373181340EA55
:10C64000830080B2400040F0010003B030BD00BF65
:10C65000007000401C4608B5084611464FF0021213
:10C6600023F0AEFA40F2DF41206846F0D3F90449E6
:10C67000042056F0A6F90348F02143F0FDFF00BF67
:10C6800038C80900914E09002DE9F04F2DED088BB7
:10C690008FB009AB01936D4B0093052323F0C8FACB
:10C6A0000021099830F0F8FD002180460A9830F00A
:10C6B000F3FD044600210B9830F0EEFDE379012BE9
:10C6C00005460AD1C379012B07D1A268012A04D9F2
:10C6D0008368012B01D99A4202D05D4844F020F8CA
:10C6E0006621D8F808005BF05DFDE66927790590C2
:10C6F000394630465BF0E5FCA368A069013B00FBCE
:10C7000003603946B0EE40AA5BF0DBFC0C98EE69A2
:10C710000E28F0EE40AA28D1297930465BF0D1FCF2
:10C720000D980E28F0EE408A22D1A868AB692979CD
:10C73000013803FB00605BF0C4FCEB690493D8F89C
:10C740001C300293059BD4F81CB0DB690393B0EE58
:10C75000409A4FF00009D8F808304B450BD805989F
:10C760000FB0BDEC088BBDE8F08F29F0A9F8D7E732
:10C7700029F0A6F8E1E7029898F804105BF0A1FC14
:10C78000029AD8F81830B4EEC0AA1A44F1EE10FAA2
:10C79000B0EE408A029252DCF4EEC0AAF1EE10FA3A
:10C7A00050D4A668D4F818A02179013E0027F31BC5
:10C7B000012B32D80AFB07B006915BF082FC069988
:10C7C00006FB0AB0F0EE40BA5BF07BFCAB69049A62
:10C7D0002979079103FB0720F0EE409A06935BF05E
:10C7E00070FC049A069B079906FB0320B0EE40BA42
:10C7F0005BF067FC38EE6B8A30EE4B0A79EEEB9A11
:10C8000028EE008A88EE290A30EE0B0A039BA3EC7F
:10C81000010A039309F101099DE707EB530303FBA9
:10C820000AB0079106935BF04CFC069B0799B4EEA7
:10C83000C80AF1EE10FAB4BF1F461E46B7E7B0EEC5
:10C84000680AE3E7B0EE490AE0E700BF88660A003D
:10C85000B03709002DE9F04F2DED048B87B003AB05
:10C860000193504B0093032323F0E2F90398002136
:10C8700030F012FD8368012B044640F28C80C679AB
:10C88000012E02D0484843F04BFF007930F088FD7C
:10C8900081460498E5690E2857D0002130F0FCFC51
:10C8A000C779012F834603D1A26883689A4201D0D9
:10C8B0003E48E8E700799FED3E8A30F071FD824600
:10C8C0002846DBF81C80C847A3694046EE18F0EE06
:10C8D000408AD047DBF81830B0EE409A9844A568FB
:10C8E000BD4211D86B1E00EE103AF6EE007A28EE2B
:10C8F000278AB8EE400A20EE080A07B0BDEC048B88
:10C90000BDE8F04F2AF08AB83046C847A3694046D0
:10C91000F0EE409A1E44D04778EEA98A30EE499A4C
:10C92000F0EE486AD9EE286ADBF8183007EE907A04
:10C93000B8EE677A9844C6EE877A0137B0EE409A2F
:10C9400038EE278AF0EE698AC9E705989FED188AC4
:10C9500028F0B6FF2846B0EE409AC847A568F0EE2A
:10C96000408AB54202D828EE098ABBE732462179CF
:10C97000E0695BF06DFB07EE906A78EE808AB8EEB6
:10C98000677A78EEC88A0136C8EE877AF0EE408A78
:10C9900038EE278AE5E7074807B0BDEC048BBDE811
:10C9A000F08F00BF70660A000B31090015310900D5
:10C9B00000000000020080801E280CD03E280AD013
:10C9C00010F0010307D1820707D10068044BC31A96
:10C9D000584258417047012070471846704700BFC1
:10C9E000202F0900F0B51B288DB006460C461546D1
:10C9F00072D03CD80E2800F09C8004D8042840F265
:10CA0000B580002430E01028FBD115F0010206D1DA
:10CA100015F00303F5D12968704A9142F1D12846F7
:10CA200055F0FCFB0122054609A9204600F024F937
:10CA3000102E0A9F3DD121790022402023F03CFA9C
:10CA4000A3686B4300FB03F1E06854F031FAA3687C
:10CA5000E0606B43A360636803F0FF0363601DB194
:10CA6000013DC319002F34D120460DB0F0BD1D2863
:10CA7000CBD02428C5D1012203A9284626F05CFE8C
:10CA8000002860D0A10712D12268554B9A420ED1DE
:10CA9000012209A9204600F0EFF801230093DDE907
:10CAA0000901DDE9032352F06AFE00285CD11E244F
:10CAB000DAE7A1689DF82C00694300F035F9C368F6
:10CAC0000446CFE7184609993A4654F088FA013DE2
:10CAD000C319002DF6D1C7E70A68424B9A4290D09D
:10CAE00009A90122204600F0C7F806A90522284618
:10CAF00026F022FE9DF82C100022402023F0DCF9C5
:10CB0000A168079DB5FBF0F5064629449DF82C0069
:10CB100000F00AF90446DDE90912C06854F05FFA32
:10CB2000E0680A9B069905FB06F2184454F057FA90
:10CB30009AE70A682B4B9A423FF463AF2946204696
:10CB40004BF0A0F990E7EA0702D5002043F08CFDF6
:10CB5000AB0703D12A68214B9A42F6D0284655F0FC
:10CB600070FE0028A3D0F0E73E247DE7012209A94A
:10CB7000204600F081F8012206A9284626F0DCFDB7
:10CB8000002894D00B9A012A21D05A2A21DC203285
:10CB90000146089B012B1ED05A2B01DC2033014695
:10CBA0009342D2D123F00203642BCED0022E01D0C7
:10CBB0000029CAD0079B0093DDE90912069B304685
:10CBC00056F0D3F9002814BF3E241E244CE742221D
:10CBD000DDE70021DDE74223E0E700BF202F090069
:10CBE0007C5A09009C590900F0B5012885B0074618
:10CBF0000E4608D08B0727D10B681C4A934202D0FF
:10CC00001B4A934220D1012201A9304626F094FD0F
:10CC1000D0B139460022402023F04EF9029BB3FBED
:10CC2000F0F100FB01F5AB4202D0124843F078FD71
:10CC3000384600F079F8019904462A46C06854F055
:10CC4000CEF9204605B0F0BD304629F08DFD58B133
:10CC500045102946384600F067F82B463A463146DB
:10CC600004464BF055F9ECE70546F2E7485E09004B
:10CC70007C5A0900763D090070B50D4601790446DD
:10CC800001F07F0116464020002223F015F9E368E9
:10CC90002B60A26842436A60227902F07F02AA6098
:10CCA0002168094A91420BD194F90420002A01DB42
:10CCB000B20707D46268C2F3172200FB02332B606D
:10CCC000002070BD0120FCE79C590900074BC1E919
:10CCD00000300023C1E90233054B02689A4202BFCB
:10CCE0004368C3F317238B6008467047B06209009E
:10CCF0009C59090038B50D461C4611462846094A7C
:10CD000022F05EFF20682AF065FF012D007804D133
:10CD1000BDE83840002100F007B86168BDE8384040
:10CD2000FFF762BF040002007828F8B505460E46FA
:10CD300002D10F4843F0F4FC00220146402023F0CA
:10CD4000BBF80C4B0C490746012D18BF19461020A3
:10CD500055F037FE0571436803F0FF030446C0E950
:10CD6000013606FB07F054F0A0F8E0602046F8BD5D
:10CD7000E33D0900406209007C5A090070B50A7958
:10CD8000012A05460C460DD1184956F023F8D4E97E
:10CD9000022128462CF0ECFC28461549BDE87040DD
:10CDA00056F018B8134956F024F8A368002BF3D0B6
:10CDB0001149284656F00EF80026A368B34204D85D
:10CDC0000E49284656F006F8E6E71EB10C492846FB
:10CDD00056F000F83246E168207923F045F9012247
:10CDE000014628462AF076F80136E6E718DE080004
:10CDF0008C1E090024DE08002FDE0800971C0900A5
:10CE0000CA1F09002DE9F04F044687B00D461646AB
:10CE10000AB90025D0E011F003078068DFF82CA2E2
:10CE200040F0DF800B68814A934240F0DA806A4626
:10CE300056F029F910B97E4843F016FC2179042EEA
:10CE400001F07F013A464FF0400000F0968023F059
:10CE500033F816F00302054655D131688B7B002B61
:10CE600042D001EB83031869724B98423CD131796F
:10CE7000402001F07F0123F01FF8A84202D06E4845
:10CE800043F04EFC33685345D6E9028B38D17368C2
:10CE9000C3F3172905FB09F9DDE900062368E768F4
:10CEA000361A5345A8EB06062FD194F90430002B0F
:10CEB000AFDA002EE3D16368C3F3172305FB0377D2
:10CEC00005FB08F20BEB090105FB007054F0B2F80A
:10CED0000199A268009B521A08EB03006A4305FB04
:10CEE000017105FB007039E0544B99420BD1012DC3
:10CEF000C5D1052203A9304626F01EFCDDE903B8A2
:10CF00004FF00009C8E74E4896E7002ED8DD636869
:10CF1000B6EB132F2FD9A16831446943384653F03B
:10CF2000C7FF6368E06066F31F2382466360BB450A
:10CF300008BF83460098A268019940443244121AFF
:10CF40006A4301FB05A105FB00A054F073F80098AB
:10CF500005FB08F20BEB090100FB05A054F06AF891
:10CF60006368C6EB132262F31F236360A368334434
:10CF7000A3600E2520E0BA46DCE722F09DFF216881
:10CF8000009B514506461BD1B3F1807F03DB2D4941
:10CF90002D485FF06FFE102055F013FD054694E814
:10CFA0000F0085E80F00009A02EB112363F31F21A5
:10CFB0006960019B9B1AAB60284607B0BDE8F08F03
:10CFC00001992079C91AFFF7AFFEDDE90032E16867
:10CFD000D21A0546724306FB0311C06853F0FFFFE7
:10CFE000EAE700232A460146206826F0C3FB2368AF
:10CFF0005345024620790ED16368042E02EB1322BA
:10D000000BD003067FF505AFE168334600F07F00E3
:10D0100023F022FBADE7042EF6D1E16800F07F009B
:10D0200007B0BDE8F04F23F01FB800BFCC5809008F
:10D030003734090005CE0200CB360900485E0900EE
:10D040006B3E090019360900A05409009C590900DB
:10D0500010EE102A08B522F00043B3F17E5FB0EE67
:10D06000406A12D319BF76EE467A9FED1F7ADFED44
:10D070001F7A9FED1F7A12BF87EE276AE0EE077ACC
:10D08000B0EE676AB0EE460A08BDB3F17C5F0BD222
:10D09000A3F50003B3F1645FF4D320EE000AFBF7BD
:10D0A000B7FAA0EE066AEDE7B0EEC06AB7EE000A86
:10D0B00030EE460AF6EE007A20EE270AB1EEC06A9C
:10D0C000FBF7A6FA002ADFED0B7AA0EE066AB0EEB7
:10D0D000007AE6EE077A9FED066A36EE676AB8BF19
:10D0E000B1EE466ACEE700BF0000000000008003FA
:10D0F000DA0FC93F6821A2B31FB58DED010A019B6C
:10D1000023F00042B2F18B4F00EE102A4FEAD370A9
:10D110000AD320F0DDF9DFED1E7A30EE270A08B1E0
:10D12000B1EE400A05B000BD5B0014D5B7EE007A41
:10D13000F0EE476AE0EE006AF1EEE67A77EE807A8A
:10D14000C7EE276AF0EE007AE0EE276AB0EE660AD4
:10D1500020F0BEF9E3E7B2F1665F10D320EE007A6B
:10D16000F7EE006A37EE266AF1EEC67A77EEA67A17
:10D17000C7EE276A36EE800A20F0FEF8CFE7DFED33
:10D18000057A70EE277ACDED037A039BC7E700BFDF
:10D190001872313F0000807B08B5044B1A68044BBD
:10D1A0009A4202D00D2039F043F808BD009C0320BC
:10D1B000EF2978011FB5044690B10E2810D00079F0
:10D1C0004DF01EF860B94FF4F773039301A92046A0
:10D1D00003AB02AA1BF038F90399024843F0A8FAFE
:10D1E00004B010BD554E0900F4EE400AF1EE10FAFD
:10D1F00010B5F0EE407A04D770EE207AB0EE670AF0
:10D2000010BD10EE902AB2F17E5F03D1BDE8104050
:10D2100000F082B810EE103A940F04F0020444EAD1
:10D22000D37433F0004308D1022C59D09FED317AEA
:10D23000032C08BFF0EE477AE0E732F0004209D154
:10D24000DFED2D7A9FED2D7A14F0010F08BFF0EE7F
:10D25000477AD3E7B2F1FF4F10D1B3F1FF4F04F19A
:10D26000FF3407D1022C3ED8254B03EB8403D3EDCA
:10D27000007AC3E7022C39D8224BF6E702F150615D
:10D280009942DDD3B3F1FF4FDAD0A10703D503F103
:10D29000506393420CD387EEA00AB0EEC00A00F0B0
:10D2A0003BF8012CF0EE407A04D1F1EE407AA5E78C
:10D2B000DFED157A022C0AD0002C9FD09FED137A57
:10D2C00077EE877A9FED127A77EEC77A96E79FED31
:10D2D0000F7A77EE877A9FED0E7A77EE677A8DE791
:10D2E000DFED0B7A8AE7DFED0B7A87E7DFED067A71
:10D2F00084E700BFDB0F49C0DB0FC9BFDB0FC93FAD
:10D30000E8610A00DC610A00000000002EBDBB33AA
:10D31000DB0F4940DB0F493F10EE102A22F000439B
:10D32000B3F1994F82B04FEAD2700ED3B4EE400AF7
:10D33000F1EE10FA07D69FED410ADFED417A0028A1
:10D3400018BFB0EE670A02B070473E498B420BD857
:10D35000B3F1665F5AD212F0FF4FF4D160EE007A5B
:10D36000CDED017A019BEEE7374A9342F0EEC07AA9
:10D3700037D8A2F5D002934229D8F0EE006ABFEE6A
:10D38000007AA7EEA67A002377EEA67A87EE270A20
:10D390005A1C60EE006A9FED2D6ADFED2D7ADFEDFD
:10D3A0002D5A26EEA67AE7EE067A9FED2B6AA7EEB7
:10D3B000876ADFED2A7AE7EE257A67EE877AE6EE6E
:10D3C000267A67EE807A24D130EE670ABBE7B7EEA3
:10D3D000007A77EEC76A77EE877A012386EEA70A8E
:10D3E000D6E71F4A93420BD8F7EE086AB7EE007AE9
:10D3F000A7EEA67A022337EEE66A86EE070AC7E7AB
:10D40000BFEE007A87EE270A0323C1E74FF0FF3310
:10D41000BEE7144A144902EB830201EB830393ED48
:10D42000007A77EEC77A37EEC00AD2ED007A37EE8F
:10D43000C00A002887D0B1EE400A84E7DA0FC93F5E
:10D44000DA0FC9BFFFFFDF3EFFFF973F25AC7C3DF2
:10D450000DF5113E4712DABDA9AAAA3E98CA4CBEE4
:10D46000FFFF1B4004620A00F4610A002DE9F84F37
:10D47000D1F800800128064640468CBF01F1040B1C
:10D480004FF0000B0F46914629F09EF830B9404608
:10D4900028F0A0FAC188274843F036F906F1FF3A90
:10D4A000B9F1000F2DD0D9F80050C5F3DC051AEB07
:10D4B000050404D02C44A00053F0D9FC04460022FB
:10D4C000924520D804EB86000022954221D11A4EC5
:10D4D000DFF868903168D9F800000131090153F094
:10D4E000E7FC3368C9F800005A1C32601A0100EBEF
:10D4F000031340F802A0C3E90158DC603868BDE8B6
:10D50000F88F4D46D3E75BF8223044F822300132E1
:10D51000D6E7D9F80830083053F8323040F80C3CE0
:10D52000D9F8083003EBC20301325B6840F8083CCD
:10D53000CBE700BF2D4D090000510120F85001201C
:10D54000F0B50023DFF838E00C4E19460E27DEF860
:10D550000020934201D30E20F0BD346804EB031287
:10D560004FEA031C9568854208BF44F80C1003F18C
:10D57000010304BFC2E90117D160E8E7F8500120B8
:10D580000051012070B590F82330FF2B04461CD0C9
:10D590000F4B012200265A60C3F80065FF2590F862
:10D5A000210038F05BFE94F8220084F8215038F016
:10D5B00055FE94F8230084F8225038F04FFE054BB6
:10D5C00084F823501E603EF043FC0E2070BD00BF67
:10D5D00000500240985901202DE9F04389B00846D7
:10D5E00011461A4603AB0193304B0093052353F0C9
:10D5F00083FE40F2C521039845F00CFA40F26C61BD
:10D600008046049845F006FA40F23A3107460598FC
:10D6100045F000FA40F25E410646069845F006FAEB
:10D6200023490546282055F0D3F9044625B1214861
:10D6300040F25E4143F020F81F4B1D6815B11F48B2
:10D6400043F03CF8186098F804009DF81C900BF02B
:10D6500093FE38790BF090FE30790BF08DFE184B6D
:10D6600098F8042084F82120C3F864253A7984F8D6
:10D670002220C3F86825327984F82320C3F8702566
:10D680000122C3F80455C3F80855C3F80C25C3F8A4
:10D690001025C3F81C25C3F82055C3F824953EF087
:10D6A000F1FB204609B0BDE8F08300BF70220A00FC
:10D6B00008C80900914E0900985901201B4909002A
:10D6C0000050024010B5044690F823004BF0B2FE23
:10D6D0000A4AD2F8083143B194F8263023F0020305
:10D6E00084F826300023C2F8083194F8263013F06D
:10D6F000020F0CBF1E203E2010BD00BF0050024094
:10D7000010B5044690F823004BF094FE0C4AD2F872
:10D71000083143B194F8263023F0020384F8263010
:10D720000023C2F8083194F826309A0701D400F09B
:10D7300009F843F0100384F826300E2010BD00BF16
:10D740000050024008B5014842F0B8FF11450900F9
:10D750002DE9F04F0D4685B055F8044B064694F878
:10D76000230017464BF066FE02AB0193674B009314
:10D77000294602233A46701E22F05AFA644A029958
:10D78000D2F808319DF80C5043B194F8263023F0BC
:10D79000020384F826300023C2F8083194F82630BA
:10D7A00098070BD55A4A0123536094F8263043F06A
:10D7B000040384F826302023C2F8083394F82600A6
:10D7C000616065F3451084F826000A7BD1F804B047
:10D7D0004F4EDFF84881D20884F825208B7BCD7B23
:10D7E000497B84F82410003B18BF01239B01013AB8
:10D7F00043EAC51300F03F0018BF0122034384F839
:10D800002630C6F81C2594F8243042495A1E53424B
:10D8100053410022C6F82835B7EE007A9446964662
:10D820001546D6F81C35012B01D18B793BB307EE99
:10D8300090BA394BD1F800A0B1F9047098FBF7F712
:10D84000F8EE676A03F15809586897FBF0F007EEA5
:10D85000900AF8EEE77A76EEE77AF0EEE77A87EE6E
:10D86000A66AB4EEC76AF1EE10FA05D5D3F800C087
:10D87000B0EE467A0246D64608339945E4D10135E2
:10D88000092D01F10801CCD1214DC5F818E5C5F8E5
:10D8900014C594F8250094F8243062830BFB00F043
:10D8A000584300014FF47A73B0FBF3F0033020F0DB
:10D8B000030080B2208353F0F8FAA060208B53F06D
:10D8C000F4FAE06060684AF0F5FD0023C4E904332F
:10D8D00084F8203094F8263023F01E0343F002032E
:10D8E000204684F826301BF0E9FF238B9B08C5F8FF
:10D8F00050352023C5F804330123C5F800352B60CB
:10D900001BF0BEFF0E2005B0BDE8F08F60220A00BC
:10D910000050024018220A00C0210A000048E80115
:10D9200010B5044690F823004BF084FD064A01230D
:10D93000536094F8263043F0040384F82630202303
:10D94000C2F808330E2010BD0050024038B5084B15
:10D950001B6800220446C3F80025FF25007938F033
:10D960007DFC6079257138F079FC65710E2038BD39
:10D97000440201202DE9F0432DED028B8BB00846C7
:10D9800011461A4603AB01933E4B0093072353F015
:10D99000B3FC40F20631039845F03CF840F23D31CB
:10D9A0000746049845F036F89DF818506A07064671
:10D9B00004D040F2C621344842F0BAFE9DF820302F
:10D9C0005B0702D04FF49961F5E70998DDF8148000
:10D9D0009DF81C9010B327F073FFB0EE408A40F220
:10D9E000D15201210020B0EE480A53F09AFC274999
:10D9F000082054F0EDFF044638790BF0BDFC307977
:10DA00000BF0BAFC84F806903A792271337963718D
:10DA1000B8F57A5F05D01E4842F082FE9FED1D8A60
:10DA2000DDE7102D01D01C48F6E71C4BDFED1C7A1A
:10DA30001B681C49C3F840256279C3F8442528EEC9
:10DA4000278A4FF00462C3F804250022C3F820257A
:10DA5000FCEEC87A2822C3F81825C3F81C25012239
:10DA6000C3F8002517EE900AC3F86015C3F86425C3
:10DA70001A6025F01DFF20460BB0BDEC028BBDE8FF
:10DA8000F08300BF98220A00C14D0900ECC70900CD
:10DA90004B340900AE47E13D6234090044020120E5
:10DAA00000007A44BC5601202DE9FF411446074688
:10DAB00000790D464BF0B8FC40F24741204622F079
:10DAC000CBF940F247420021044653F054FCAB0727
:10DAD00006D12A682D4B9A4202D12D4842F0C4FD4E
:10DAE000062201A9284625F027FE9DF80C10029D6C
:10DAF0000022402022F0E0F9B5FBF0F5A54202D269
:10DB0000244842F00DFE039B482B01D02248F8E741
:10DB1000DFF89080019DD8F800300122C3F8082575
:10DB2000C3F86055C3F864451C4B4FF4485043F0AC
:10DB300001039847D8F800300022C3F80821184A9A
:10DB4000C3F8602501222E46C3F86425D8F80030BA
:10DB5000D3F808316BB105EB4405B5420CD1BB7964
:10DB600083B124F00104640044F0010004B0BDE876
:10DB7000F08102F077FEE9E73388A3F5004326F849
:10DB8000023BEAE724F00304EDE700BF68140A0053
:10DB90005D4A090030490900F43A0900F0220A0000
:10DBA000BC5601204402012070B58AB008461146D7
:10DBB0001A4606AB0193264B0093042353F09CFBBB
:10DBC0000698052203A925F0B7FD059C622C0ED00E
:10DBD000682C0FD0482C1FD0422C01D1002507E023
:10DBE000012C1BD01B4840F2E52142F0A1FD01258C
:10DBF000012401E0012502249DF8243083B9079B0C
:10DC0000049A63435B00B2FBF3F103FB11223AB1C8
:10DC1000114840F2E521E8E70025ECE70025EBE7B5
:10DC20000E49182054F0CDFEE4009DF824309DF8F4
:10DC30001C10089A039E0473049CC373002306619E
:10DC4000857384604173426003750AB070BD00BF84
:10DC5000D0220A00DB4D090089460900CCC7090023
:10DC60002DE9F0411C460D4692B0114628467F4AE8
:10DC700021F0A6FF26687E4B3340062B05D0B20765
:10DC800010D132687B4B9A4208D131467A4845F22E
:10DC9000661253F070FC8307064603D13268774B57
:10DCA0009A4202D0764842F027FD012D26D906225D
:10DCB00008A9606825F040FD0998089F40F2E52317
:10DCC0004FF48062082122F077F805466D49402024
:10DCD00054F077FE044606630022002306F1080094
:10DCE00050F037FA206B10226B460DEB0201083022
:10DCF00050F060FD28B1052042F0CAFC00252F46F7
:10DD0000E4E7009B102B0BD15F49042204A853F0D9
:10DD100052F928B95D49082206A853F04CF918B108
:10DD200040F2AE3021F076FF206B04226B460DEB03
:10DD30000201083050F03EFD0028DCD1009B042B8E
:10DD400002D1019A282A02D9514842F0E9FC206BFD
:10DD50006B4608A9083050F02DFD0028CBD1019A60
:10DD6000282A03D0BDF82030012B0CD1BDF8221099
:10DD7000022908D8BDF82E30102B04D8122A04D15D
:10DD8000BDF830208AB14348DFE7282A0DD1BDF81D
:10DD900020004FF6FE729042F5D1BDF83820012ADE
:10DDA000F1D1BDF832209A42EDD1082B099A2373A4
:10DDB00094BF00230123A3734FF40073A3600023D7
:10DDC00062606173E373206B6B46042202A9083022
:10DDD00050F0F0FC00288ED1009E042E8BD12E49ED
:10DDE000324602A853F0E7F88046206B6B46324675
:10DDF00003A9083050F0DEFC00287FF47CAF009BC4
:10DE0000042B7FF478AF206B039AB8F1000F0AD08F
:10DE1000D0E91013521843F10003083050F099F97B
:10DE20000028D0D067E72262036CA38465B94FF461
:10DE30008070E06253F039F803462061E06A63B90C
:10DE4000A561657342F0D6FB6D0827612F44E5623A
:10DE5000A761204612B0BDE8F08153F026F8A0611A
:10DE60000028F6D1E06A25616573EBE70400020043
:10DE70000F0080FF942D09005057090068140A0014
:10DE8000173A0900ACC709008E1E0900931E09004D
:10DE9000E8460900CA4709009AFB08002DE9F04F3F
:10DEA0002DED028B8DB0044607920493426A00293F
:10DEB00043D0079B012B00D1826A189BA16919608E
:10DEC000216A237F914240F05C83D4E90421002B36
:10DED00018BF1146049B02911960237F83F0010350
:10DEE0002377A3699B08069304F130030993002369
:10DEF0000893019394F82C30089A93421FDC019BFD
:10DF00003BB9029A0699019B02EB8101914240F0D4
:10DF10001883A37B002B00F01783236A013323624D
:10DF2000079B002B40F03483636A01336362012056
:10DF30000DB0BDEC028BBDE8F08F0791BDE7099BEA
:10DF400053F8046F0993B3680593002B40F0EC82FB
:10DF5000089B01330893CDE7B360019B002B00F0D1
:10DF6000E98201230193F3E752008A4228BF0A465F
:10DF70000399914228BF11468B4647E20A4692E236
:10DF800057F8203031FB03FC32FB13F32CF3CF3C6A
:10DF900023F3CF33CCEA034345F8203001308345E7
:10DFA000EED1039B607BA3EB0B030393059B5B7B91
:10DFB0009842D6E9041205EB8B0500F0F1814FEA97
:10DFC0005B0301EB8301D21AEEE11204E7E763453C
:10DFD00045D001982BF0010E4FF08028090412045F
:10DFE00005F104097045DCD057F8103093FA48FA6F
:10DFF0001FFA8AF343EA0A4331FB03FC32FB13F3B3
:10E000002CF3CF3C23F3CF33CCEA034345F8203045
:10E010004FEA1A431B0443EA1A4331FB03FC32FB69
:10E0200013F32CF3CF3C23F3CF33CCEA034349F86B
:10E0300020300230D6E757F8203093FA4CF331FB0A
:10E0400003FE32FB13F32EF3CF3E23F3CF33CEEA9E
:10E05000034345F8203001308345ECD1A1E7019816
:10E060004FF0802C09041204F6E763454FEA4B0990
:10E0700020D1DDF804804FF0802A09041204C8453D
:10E080008FD237F818005EF016FEA37B0BB990FA1A
:10E090004AF031FB00F332FB10F023F3CF3320F3CF
:10E0A000CF30C3EA00405AF041FB25F8180008F1D0
:10E0B0000108E4E7AB1CDDF804A00A93090412048C
:10E0C0000AF101004845BFF46CAF37F80A005EF072
:10E0D000F2FD8046A07B18B94FF0802398FA43F8F0
:10E0E0001FFA88FC4CEA084C31FB0CF032FB1CFC9C
:10E0F00020F3CF302CF3CF3CC0EA0C405AF016FB93
:10E100004FEA184C4FEA0C4C25F81A004CEA184C10
:10E1100031FB0CF032FB1CFC20F3CF302CF3CF3C56
:10E12000C0EA0C405AF002FB0A9B23F81A000AF1DD
:10E13000020AC5E7BEF1100F40F0B480A07B0028B2
:10E1400054D0634536D0043F28464FF0010C0904F3
:10E150001204E3457FF625AF57F804EF1FFA8EF35C
:10E1600043EA0E4331FB03F832FB13F328F3CF38B5
:10E1700023F3CF33C8EA034350F8088B93FA18F31C
:10E1800040F8083C4FEA1E431B0443EA1E4E31FB95
:10E190000EF332FB1EFE23F3CF332EF3CF3EC3EA42
:10E1A0000E4E50F8043C9EFA13F340F8043C0CF178
:10E1B000020CCEE7A5F1040C0020090412048345EB
:10E1C0003FF4EFAE57F8203031FB03FE32FB13F380
:10E1D0002EF3CF3E23F3CF33CEEA03435CF804EFB4
:10E1E00093FA1EF3CCF800300130E8E763453AD0EB
:10E1F000043F28464FF0010C4FF0802E0904120412
:10E20000DC45BFF4CEAE57F8043F93FA4EF81FFA40
:10E2100088F343EA084331FB03F932FB13F329F394
:10E22000CF3923F3CF33C9EA034350F8089B93FA5D
:10E2300019F340F8083C4FEA18431B0443EA184816
:10E2400031FB08F332FB18F823F3CF3328F3CF3830
:10E25000C3EA084850F8043C98FA13F340F8043C29
:10E260000CF1020CCCE7A5F1040C4FF0802E090450
:10E27000120483453FF495AE57F8203093FA4EF3DD
:10E2800031FB03F832FB13F328F3CF3823F3CF33FA
:10E29000C8EA03435CF8048F93FA18F3CCF8003013
:10E2A0000130E6E74FEA4B0063450A9072D1A5F1D1
:10E2B000020A4FF00009090412040A9B9945BFF4B1
:10E2C00070AE37F819005EF0F6FCA37B1BB94FF077
:10E2D000802390FA43F031FB00F832FB10F028F372
:10E2E000CF3820F3CF30C8EA00483AF8020F5EF08A
:10E2F000E2FC98FA10F05AF019FA09F10109AAF8AB
:10E300000000DAE7F85A0B935EF0D5FC8046A07B5C
:10E310000B9B18B94FF0802098FA40F81FFA88FC40
:10E320004CEA084C31FB0CF932FB1CFC29F3CF39C9
:10E330002CF3CF3CC9EA0C4935F813000B935EF07F
:10E34000BAFC99FA10F05AF0F1F90B9B4FEA184C0D
:10E350004FEA0C4C25F813004CEA184C31FB0CF832
:10E3600032FB1CFC28F3CF382CF3CF3CC8EA0C4816
:10E3700035F81A005EF09FFC98FA10F05AF0D6F9C2
:10E380000B9B25F81A0002330AF1020A0A9882450B
:10E39000B8D306E64FF0010A002309041204F5E79A
:10E3A00001EB8B01A2EB0B02C6E90412039B002BCD
:10E3B0003FF4D7AD7369BBB9737B33B9337B002BA3
:10E3C0003FF4CAADB0684AF075F8B06860B106F1C4
:10E3D000140206F110014AF028F873699B08736172
:10E3E000431E5842584170730598637B407B3769E0
:10E3F000726998424FEA03217FF4B6AD914228BF7B
:10E400001146039A8A4228BF0A469346D4ED017A00
:10E41000BBFBF3F3F8EE677AF7EE000A80EEA77A1B
:10E42000634A06F1180007EE903AF8EEE77A614B7E
:10E430009FED610A67EE877A27EE287AC3ED007AAE
:10E440005E4B83ED007A1378013313705DF0DFF9D2
:10E45000DFED5B0AB0EE408A06F11C009FED590A21
:10E460005DF0F1F9DFED587A637B28EE278A022B05
:10E47000BCEEC88A18EE102A91B27FF47FAD10F47A
:10E48000004F47F6FF7C11BF00EB0C02ACEB000025
:10E4900080B24FF400421CBF92B24FF400404A4396
:10E4A0004843D213C113059894F80CE090F80DC0BE
:10E4B000019800287FF43EAEBEF1100F7FF4D5AD79
:10E4C000A07B00283FF483AD634501984FEA0141EA
:10E4D0003FF47BAD4FEA024E05F1040883457FF619
:10E4E00060AD57F8102093B243EA024331FB03FCBE
:10E4F0003EFB13F32CF3CF3C23F3CF33CCEA03439F
:10E5000045F82030130C1B0443EA124331FB03F29D
:10E510003EFB13F322F3CF3223F3CF33C2EA03429D
:10E5200048F820200230D9E7069B029DDFED278ABC
:10E5300003933BE7039B01999A00284652F090FD14
:10E540000FE542F8043BE1E4237B069A102B029B83
:10E5500003EB82020AD04FF080309A423FF4DDACE8
:10E56000196881FA40F143F8041BF6E74FF0802068
:10E570009A423FF4D2AC196891FA40F143F8041B77
:10E58000F6E71BB92369049A1360C9E46369FAE7E3
:10E59000079B012B7FF4CBACA36A227B0133A362E0
:10E5A000049B1B6803EBD203049A1360BFE400BF13
:10E5B000896901200063012000000000FC62012045
:10E5C00000FE7F3F00FE7FBF00000047DB0FC94019
:10E5D0002DE9F04788B0084611461A4602AB019370
:10E5E000364B0093062352F087FE40F25C63FF2215
:10E5F0000121029852F0B3FE40F2FB2306460222AC
:10E600000498012152F0ABFE079D002D804604DCEA
:10E610004FF4AE61012021F09DFBDDF814A0BAF1AA
:10E62000080F05D0BAF1100F02D0254842F078F853
:10E6300006F10D002349800054F0C3F9039F9DF8B3
:10E6400018900446F8088000A06152F02EFC0346A2
:10E650002061A0691BB96373636141F0CBFF52F085
:10E6600024FC606118B960732061A069F5E76560FA
:10E670000025A76084F80CA084F80E9084F80D8023
:10E68000E57384F82C6004F13007B5420ADB94F896
:10E690002C0004F1340128F04DFB2063204608B023
:10E6A000BDE8F087002308481A46194600F062F8D2
:10E6B000013547F8040F4460E7E700BF2C240A0047
:10E6C000C63D09008CC7090010240A00F0B50C46AD
:10E6D00087B054F8045B0646687B174649F0A0FEF5
:10E6E00003AB01930E4B00933A4603232146701E61
:10E6F00021F09EFA95F82C209DF810309A4203D80C
:10E7000040F25B6021F086FA05EB83039DF814204C
:10E71000586B03990BF062F9284607B0F0BD00BFB3
:10E72000F8230A00F0B50D4685B055F8044B0646AF
:10E73000607B174649F074FE03AB01930C4B0093CA
:10E740003A4601232946701E21F072FA94F82C20D3
:10E750009DF80C309A4203D840F25B6021F05AFADF
:10E7600004EB83040022636B0E209A6005B0F0BDB9
:10E77000F0230A0010B508461146002221F020FAC5
:10E780000B49202054F01DF900230446836000F15A
:10E7900018014FF4896207483EF0D8FA064840F263
:10E7A000D14204F11C013EF0D1FA204610BD00BF59
:10E7B00010240A00020000C0020080801FB502ABD6
:10E7C00051F8044B0193074B00930138022321F0C9
:10E7D0002FFA20469DF80C2002990BF0FFF80E202E
:10E7E00004B010BDE0230A001FB503AB0193064B34
:10E7F00051F8044B00930138012321F019FA00234A
:10E800000E20A36004B010BDD8230A002DE9F04FFC
:10E81000AFB0446A04901CB9389B1C60022021E010
:10E8200000290499896814913899149C0C60049902
:10E8300091F9541008BF00228A42049915D1049816
:10E8400091F9551000EB8101496B01EB42021A600E
:10E85000FF2380F85430389B1A68836D03EB520312
:10E86000836501202FB0BDE8F08F91F84410049C1F
:10E87000B1FA81F1490984F8441084F85510C2F1C5
:10E88000010204EB810184F854204A6B1A6006925D
:10E8900052F07BFC0498002152F052FC049B044689
:10E8A00070B99A680146069852F0DAFB389B1C60F2
:10E8B000049B93F8450080F001004000C0B2D1E70E
:10E8C000049ADB6A126BD21A0992049A12690392B3
:10E8D000002A01F01685049A0398576A1F443946A6
:10E8E00047F028F8421C064601F00F85039BD3F839
:10E8F0000090B9F1000F00F03D81D3F80480B8F129
:10E90000000F00F0378199F800B099F81C303C18DE
:10E91000BBF1000F3ED1032B4FF0090114BF4FF0A4
:10E92000200A4FF0110A2AA8CDE92A4BCDE92CBACA
:10E930005FF0FAF8C8F8000099F81C30032B14BFF8
:10E94000032105212AA85FF0EFF8454645F8040F9A
:10E95000039BD3F8BC379B450DDB4FF0000B039BAB
:10E96000D3F8C4379B4580F2C880902303FB0B8506
:10E970000023059392E005F1100301212AA80593D5
:10E980005FF0D2F8059B45F8040F9D42F5D10BF1DD
:10E99000010BDDE7032B4FF0080114BF4FF0110A04
:10E9A0004FF0090A00232AA8CDE92B332A94CDF889
:10E9B000B4A05FF0B9F8C8F8000099F81C30032B38
:10E9C00014BF022101212AA85FF0AEF8C8F80400A4
:10E9D000C3E70C212AA85FF0A7F80921A8622AA89A
:10E9E0005FF0A2F80821E8622AA85FF09DF828638A
:10E9F00099F80030002B14BF092104212AA85FF0E8
:10EA000093F8012168632AA85FF08EF8A8630028B4
:10EA100056D002212AA85FF087F80121E8632AA8CE
:10EA20005FF082F8052128642AA85FF07DF80521AF
:10EA300068642AA85FF078F80023EB64A8640321D7
:10EA40002AA85FF071F8032128652AA85FF06CF806
:10EA5000032168652AA85FF067F8EB6BA86533BBF4
:10EA6000C5E90A336B63E86DC0F11400286699F8B4
:10EA70000030002B3FD101212AA85FF055F86866CD
:10EA800001212AA85FF050F80121A8662AA85FF0AA
:10EA90004BF8059BE866013305934835039B059ABF
:10EAA000D3F8BC379A4294DB0BF1010B57E7022BEA
:10EAB00004D12B6C13B90823EB65D4E70723FBE7DC
:10EAC000C5E90F0005212AA85FF02EF8052168642A
:10EAD0002AA85FF029F80521A8642AA85FF024F885
:10EAE0000421E8642AA85FF01FF80321E8652AA83A
:10EAF0005FF01AF8BAE70020C1E7039A0999D8F83D
:10EB00000080C2F8D88706EB0A028A1A0399099294
:10EB1000D1F8B817039A04EB0A05D2F8B0270029F8
:10EB20005AD0002A40F0A480039BD3F8CC27099B3D
:10EB3000934280F2AE800699039847F05EFE4FF054
:10EB4000FF34149A0698002152F08AFA049B93F835
:10EB500045300BB903341BD8049B06989A680021F2
:10EB600052F07EFA389A00231360049A012382F847
:10EB7000453053E60699039847F03FFE6FF00604D0
:10EB8000049B099A1B6B9B1A049AD362002CD8D160
:10EB9000049B149A9B6D03EB5203049A93651046F1
:10EBA00052F0F3FA0498002152F0CAFA049B049A36
:10EBB0001B6BD26A9A1A049B9B6A9B1AB3F5007F5F
:10EBC000044607DD049AAE4B02F11400C2E9053297
:10EBD00001F00CFE204645E6002A49D10399DDF8F4
:10EBE00024B00122C1F8B027A946594648460593EA
:10EBF00047F017FE431C059B18D019F800C0397860
:10EC00008C4509EB00021DD192F801C079788C4542
:10EC100018D197F802C091788CEA0101032911D824
:10EC20001CF0020F18BF02F1FF32501B039A00289C
:10EC3000C2F8B4070CDA0699104647F0DEFD6FF013
:10EC400002049DE7033002F10309ABEB000BCCE7B4
:10EC5000039A0644D2F8C02756445643039AD2F882
:10EC6000C8275343039AF60096FBF3F3C2F8B8376C
:10EC7000039BD3F8B4271B6843B15B69003B18BF03
:10EC800001231344039AC2F8CC374DE74FF0FF330A
:10EC9000F7E7039B0399D3F8DC37434501F11C00E8
:10ECA0003DDBA3EB0801424641180A9052F0C2F93D
:10ECB000039BD3F8D807D3F8CC270A9B29461844DE
:10ECC00052F08DF9039B0399D3F8CC27D3F8D837AA
:10ECD0001344C1F8DC37DB001093039B099903F25E
:10ECE000DC738A1A1A93002309920C930593039BF1
:10ECF000059AD3F8C4379A4281F21E837C2353438A
:10ED00001193902353431993119B013B1F93119B24
:10ED100008931A9B189300230D939B46FEE3294604
:10ED2000184452F05CF9039B0399D3F8CC27D3F82D
:10ED3000DC3703981344C1F8DC37099B06999B1A0A
:10ED400009936FF0010447F058FD19E7039B1E6813
:10ED5000002E00F0D4805B680793002B00F0CF807A
:10ED6000039B9D68002D00F0CA800A9B229300231C
:10ED7000CDE923330C9A109B9A18D31D48BF02F19A
:10ED80000E03DB1025930C9B1BB1194622A85EF0E5
:10ED9000CBFE059B317890225A43482303FB0B227C
:10EDA000079B1A44536BD2F83CC0002940F04E81B7
:10EDB000344810F8136000EB4300BCF1020F4778B1
:10EDC00062D1D2F84090B9F1000F10D0089B88466C
:10EDD00005EB0309314622A85EF0A6FE08F1010802
:10EDE000B8F1080F09F8010BF4D14FF00309119B9A
:10EDF00005EB03080D9B984409EB49039844314601
:10EE000022A85EF091FE314688F8170022A85EF035
:10EE10008BFE314688F8180022A85EF085FE09F1C5
:10EE20000109B9F1060F88F8190008F10308E6D1C5
:10EE3000089BEE18394622A85EF076FE394686F821
:10EE4000290022A85EF070FE394686F82A0022A822
:10EE50005EF06AFE09F10109B9F10C0F86F82B008A
:10EE600006F10306E6D1059A7C2353433E2202FBBA
:10EE70000B332B44002283F83B209A8724E000BF09
:10EE80005DFB040074600A00059B002B3ED10D9BC6
:10EE9000DDF8148005EB0309314622A85EF044FE3C
:10EEA00008F10108B8F10B0F09F8010BF4D10D9B23
:10EEB0001D44394622A85EF037FE05F8080008F127
:10EEC0000108B8F1150FF4D1059B189A90265E43FE
:10EED0004820079B00FB0B6633449B6A5360229BD0
:10EEE0000A9A9B1A249AC2EBC302D71007D4189B24
:10EEF00053F804CF1893109B634580F2ED81069977
:10EF0000039847F07AFC6FF0070439E64FEA0B13D9
:10EF1000079A083302EB030952F80380B8F1000F97
:10EF20001FD00D9B8846EB181F9913F8012B5A54DC
:10EF300008F10108B8F1060FF6D1D9F80430FBB991
:10EF4000089B4FF0060805EB030A314622A85EF045
:10EF5000EBFD0AF8080008F10108B8F10B0FF4D135
:10EF600021E0089B05EB030A314622A85EF0DCFD98
:10EF700008F10108B8F1060F0AF8010BF4D1DCE73B
:10EF8000059C3E2303FB0BF37C20EA1800FB0433B3
:10EF90002B4491799971D179D971117A1972517A79
:10EFA0005972927A9A72D9F808306BB9089B0B267D
:10EFB00005EB0308394622A85EF0B6FD08F8060006
:10EFC0000136102EF6D112E0059C3E2303FB0BF315
:10EFD0007C20EA1800FB04332B44D17AD972117BD0
:10EFE0001973517B5973917B9973D27BDA73D9F87A
:10EFF0000C306BB9089B102605EB0308394622A894
:10F000005EF092FD08F806000136152EF6D112E0EA
:10F01000059C3E2303FB0BF37C20EA1800FB043322
:10F020002B44117C1974517C5974917C9974D17C56
:10F03000D974127D1A75059A7C2353433E2202FB34
:10F040000B332B4400225A759A753DE7366A16F049
:10F05000010603D0BBF1010F00F0B280B3F5C87F09
:10F060007BDA1911052291FBF2F2269202EB820261
:10F07000891AC3F38102289203F003030022279127
:10F08000299311461346BCF1020F40F0CE80059C37
:10F09000902060434827079C07FB0B002044006C2E
:10F0A000002808BF4FF0010C01EB41018948614481
:10F0B00010F821702A9700EB810148782B9088780E
:10F0C000C9782C902D910EB3BBF1010F1ED10DF11B
:10F0D000980C05F1FC070DF1A80E664603CE7645A7
:10F0E00038607960B44607F10807F6D10DF1A80C35
:10F0F00005F58677664603CE79602EA98E42386084
:10F10000B44607F10807F5D1C5F8F8200599902213
:10F110004A43482101FB0B2207990A445366D36BEB
:10F12000022B40F0C580176C002F00F0A880089BD0
:10F130000026EF18269922A85EF0F6FC0136062E6E
:10F1400007F8010BF6D14FF001080327119B05EBDF
:10F15000030A0D9B0AEB03048BE0B3F5FA7F12DA86
:10F16000A3F5C87399100522B1FBF2F2269202EBC7
:10F170008202891A03F0030300222791289329921F
:10F18000134601217FE7A3F5FA730321B3FBF1F1E5
:10F1900001EB4102059826919B1A0022CDE9282215
:10F1A00090224243482000FB0B22079827930244F9
:10F1B000126C0AB1CDE9271300220123022162E774
:10F1C000B3F5B47F03F001024FEA630110DA2420A3
:10F1D00091FBF0F3269300FB1313062093FBF0F151
:10F1E00000FB1133289300232791299303214AE739
:10F1F000F3290CDCB4390B112693C1F38103279357
:10F2000001F0030100232891299304213BE7F439FD
:10F210000323B1FBF3F3269303EB4303C91A002343
:10F220002791CDE9283305212DE74FF0000C3BE76E
:10F2300026AB22A853F828A051465EF075FC514633
:10F24000F07522A85EF070FC5146307622A85EF080
:10F250006BFC033609F10109B0752AAB53F828207D
:10F260009145E5DB08F10108B8F1040F3FF4FBAD6F
:10F270004F4407EB470626444FF00009EDE7B84638
:10F2800064E753F8261022A85EF04EFC09F8010B43
:10F29000013726AB5AF826209742F2DB0136042EBE
:10F2A0000DD0B84404EB080900270DF1A80AF1E7D6
:10F2B000089B4FF00008EC18464626ABF2E7059A8B
:10F2C0007C2353433E2202FB0B331D440023AB75CA
:10F2D0006B75F9E594600A00039B1D68002D00F032
:10F2E000C2815B680B93002B00F0BD81039B9B6880
:10F2F000002B00F0B881039BD968002900F0B3818E
:10F3000002F0070313930C9B139AC3EBC703134438
:10F310001C93BCEB0303079300F1A5810A9B6A6B66
:10F320003B441D930B9B1E44B36B002B00F02381C9
:10F33000F36B022B40F01F81336C002B40F00381F4
:10F34000059C9023634300FB0B330B98034403207D
:10F35000DB6D013393FBF0F302EB4303B3F92E00B3
:10F3600000EB40004FF41072059C90236343482546
:10F370000B9C05FB0B332344DB6A5B00B3F5107F6A
:10F38000A8BF4FF410739342D4BF2C932C920A93CE
:10F390002D938342D4BF2B932B9001EB8B032093AF
:10F3A00003F580530A9AC3F800224FF4106303FB5D
:10F3B0000B131593139B0F931D9B0C930023169314
:10F3C0000E93199B4033E31821930E9B169F013334
:10F3D0002AAA0E9352F823301693A3EB070EBEF120
:10F3E000000F23DD159B0E9A0C9903EB8707219BD9
:10F3F00053F82250B14B03EBC5031E790F9B5A42C1
:10F4000002F0070213462AB111F8010BC2F12002E3
:10F4100000FA02F2002E40F0C08033463A1D47F851
:10F42000263042F826300236B645F8DC00230F9A23
:10F430000C991A4401EBE20102F007020F92079ABD
:10F440000C91D31A07930E9B032BBED1109B1C9AD1
:10F450009B1A0E93079B002B00F09F82159B0A9A24
:10F460000C9803EB8205059A90235343482202FB34
:10F470000B330B9AD318924ADB6E52F823200B926F
:10F48000904A52F823100F9B5B4203F007031A4681
:10F490002BB110F8016BC3F1200306FA03F3079CAC
:10F4A000A61A0A9C4FF00009C4F50F7AC1F1200199
:10F4B0004F460AF1010A0A91BA4500F3F081209BF8
:10F4C00003F58052D2F800323B44C2F800320022E9
:10F4D000B3F5107FC0F26382079A0F9B13440C9A16
:10F4E00002EBE30203F007030C93089B0A923E33FE
:10F4F00008930D9B3E330D93199B48331993134684
:10F500001D9A9B1A00F1AF80139AC2EBC3030C9AA9
:10F5100013440E9AD31A10930BF1010B039BD3F8EB
:10F52000BC379B45FFF612AC0599039844F016FED4
:10F53000013040F057850699039847F05EF96FF067
:10F540000904FFF71DBB2B785BB9059C902363432F
:10F5500000FB0B330B980344DB6D013332F91300CE
:10F5600000E7B2F93600B2F93430C31AB2F90C0030
:10F5700000EB4300F6E6059B90255D43482303FB23
:10F580000B550B9B1D44EB6D2D6E013332F91300AF
:10F590002B44013332F91320E6E64B4850F825C0DE
:10F5A0004A4800EB4C0017900798012EA0EB03008F
:10F5B00040F08E80454C34F81C6006F00F064FF08A
:10F5C00000094FF0004AC6F120060F2853DD8C4693
:10F5D000C3F118081CF8025B497805FA08F5C3F175
:10F5E000100801FA08F10D432A4310331038614620
:10F5F0000A2BEADD22FA06F5179C013534F815507E
:10F600004FEA153C15F0F00F02FA0CF218BF02F0A9
:10F61000004CA3EB1533C5F303181EBF520003F1D2
:10F62000FF334CEA080815F4706FC5F3032C1FBFB5
:10F6300003F1FF3302F0004545EA0C0C52004B4544
:10F6400011DB47F8088BAEF1020EBEF1000F47F850
:10F6500004CCCDDCA3EB0903079A0344D31A079A21
:10F6600093427FF6E4AE0699039847F0C6F86FF030
:10F670000804FFF785BA1D18002DF4DD002812DDFF
:10F68000082891F800C0C8BF4878C3F118080CFAE0
:10F6900008FCC8BFC3F1100342EA0C02C9BF98407E
:10F6A0000131024302316B1E4AFA03F31A404FF054
:10F6B0000B0905F10B0300209AE700BF703D0A001B
:10F6C0006C600A0064600A00945F0A00703E0A00E1
:10F6D000A6F1020CBCF1010FC5D8DFF8F0C25CF84E
:10F6E0003580DDF85CC00024129408F101041B94FD
:10F6F000C8F120041E940F2827DD8946C3F1180A9B
:10F7000019F8025B497805FA0AF5C3F1100A01FA03
:10F710000AF10D432A431033103849460A2BEADD1B
:10F72000BCF8009009F00F09C9F1200522FA05F58F
:10F7300001353CF815505FEA153A2AD1A3EB0903CD
:10F7400002FA09F20CEB450CE8E7C518002D8ADD3A
:10F75000002812DD082891F80090C8BF4878C3F14E
:10F76000180A09FA0AF9C8BFC3F1100342EA0902EC
:10F77000C9BF98400131024302314FF000406B1E77
:10F7800040FA03F30B201A40129005F10B030020FE
:10F79000C4E7C5F30319B9F10F0FA3EB0A0302FA8B
:10F7A0000AF2C5F3032523D1032E24D11B9C03EBBE
:10F7B000000C002D0CBFA24604F1010AE2453FF700
:10F7C00052AF9C46E24552DC0344B3EB0C0006D535
:10F7D000581E9C464FF0004303411A4000201E9BD8
:10F7E00022FA03F909F10F09ACEB080302FA08F257
:10F7F000B9F1000F05D002F0004C49EA0C095200A3
:10F80000013B0F2D1DD1032E1CD11B9C1D18AC429A
:10F810003FF729AF9C461B9C644533DC0344B3EBA4
:10F820000C0006D5581E9C464FF0004303411A4079
:10F8300000201E9B22FA03F50F35ACEB080302FAF9
:10F8400008F22DB102F0004C45EA0C055200013BD4
:10F85000129CA342FFF607AFAEF1020EBEF1000FFD
:10F86000C7E9009518DDDDF85CC0083756E711F8E8
:10F87000019BCCF1180409FA04F942EA09020CF1DF
:10F88000080C9FE711F8015BCCF1180A05FA0AF59C
:10F890002A430CF1080CBEE7129A9B1ADCE60F2EE5
:10F8A00056DD8446C2F1180E1CF8021B407801FA9E
:10F8B0000EF1C2F1100E00FA0EF001430B431032AC
:10F8C000103E60465745BFF6F7AD092A7FF7F4AD05
:10F8D0000A990B9C23FA01F121443B4C615C4FEAED
:10F8E000111C03FA0CF311F00808A2EB11121FBF50
:10F8F00003F0004802F1FF325B0048F0010811F00C
:10F90000040E1FBF03F0004E02F1FF325B004EF009
:10F91000010E11F0020C1FBF03F0004C02F1FF3288
:10F920005B004CF0010C11F001011FBF03F000411E
:10F9300002F1FF3241F001015B004A45FFF6BFAD25
:10F9400045F8108B043745E903EC45F8041CB9E78A
:10F95000B11800297FF7B3AD002E12DD082E90F804
:10F9600000C0C8BF4678C2F1180E0CFA0EFCC8BF22
:10F97000C2F1100243EA0C03C9BF96400130334381
:10F9800002304A1E4FF0004444FA02F213404FF096
:10F990000A0901F10A02002694E7079F8FE51599ED
:10F9A00041F82320013393E5059903982A4645F051
:10F9B00095FB01300CD10699039846F01EFF6FF0BD
:10F9C0000A04FFF7DDB800BF14600A00703D0A00AA
:10F9D0000135039BD3F8BC379D42E5DB039AD2681F
:10F9E000002A00F08684039A52690B92002A00F0E4
:10F9F0008084039A92690792002A00F07A84039A1D
:10FA0000D2F8C867059A5643069A5E43022B02EB6A
:10FA1000460640F0E9820B9B1193331D08930023A7
:10FA20000E93079B03F500530D930E9B0D9A0799B8
:10FA3000119803F001030F930B9B03F580554FF0D2
:10FA40000077D5F8183B0093D2F800220F9B45F0C1
:10FA500025F8D5F81C3B0D9A079911980093D2F818
:10FA600000220F9B803100F5106045F017F80F9BC6
:10FA70000D9A5B42D2F8002203F488631344079A7C
:10FA800002EB830B4FF0000C52F82320DBF85C30C4
:10FA90006046C2FB007C6FF07301C3FB017C4FF03A
:10FAA0000076DBF88020DBF8DC300546C2FB006521
:10FAB000C3FB01654FF45579DBF80430DBF85820BF
:10FAC000C3FB097C834BC2FB037CDBF88410DBF8AF
:10FAD000D820C1FB0965C2FB036541F6D478DBF889
:10FAE0000830DBF85420C3FB087C7B4BC2FB037C53
:10FAF000DBF88810DBF8D420C1FB0865C2FB036586
:10FB000046F2B86EDBF80C30DBF85020C3FB0E7CFD
:10FB1000724BC2FB037CDBF88C10DBF8D020C1FBFE
:10FB20000E65C2FB03656E4ADBF81030DBF84C1043
:10FB3000C3FB027C6B4BC1FB037CDBF89000DBF862
:10FB4000CC10C0FB0265C1FB0365DBF81420DBF8B9
:10FB50004830C2FB0E7C45F28401C3FB017CDBF81C
:10FB60009420DBF8C830C2FB0E65C3FB0165DBF8EF
:10FB70001820DBF84430C2FB087C40F22C71C3FB38
:10FB8000017CDBF89820DBF8C430C2FB0865C3FBBE
:10FB90000165DBF81C20DBF84030C2FB097C7421D6
:10FBA000C3FB017CDBF89C20DBF8C030C2FB09659D
:10FBB000C3FB01650C2438464FF014080CFA04F31B
:10FBC0004CFA08FC20FA08F040EA030046F008FB73
:10FBD000089B23F8040C304605FA04F345FA08F5AF
:10FBE00020FA08F040EA030046F0FAFA089B0BF509
:10FBF000805723F8020C3B684FF4D0704FF000722E
:10FC00004FF0000CC3FB002C4FF00073D7F88010AE
:10FC10000026C1FB003641F67C007968C1FB002C50
:10FC2000D7F88410C1FB003649F2FC70B968C1FBFB
:10FC3000002CD7F88810C1FB00362B49F868C0FBB0
:10FC4000012CD7F88C00C0FB013628493D69C5FB63
:10FC5000012CD7F89050C5FB01366FF0B3057969D8
:10FC6000C1FB052CD7F89410C1FB05364FF4127573
:10FC7000B969C1FB052CD7F89810C1FB05366FF0A8
:10FC8000130EF969C1FB0E2CD7F89C101D46C1FB61
:10FC90000E5610460CFA04F34CFA08FC20FA08F051
:10FCA00040EA030046F09CFA089B9887284606FA2B
:10FCB00004F346FA08F620FA08F040EA030046F09A
:10FCC0008FFA089B0A49D88704331293089B043B98
:10FCD00013930FE0D4F8FFFF7CAFFFFF3CB6FDFFAE
:10FCE00078940400C44902004CE803002464FFFF38
:10FCF00050390A00D1F840E0DBF80051DBF85C0134
:10FD00004FF000730022C5FB0E324FF000764C6CB2
:10FD10004FF00009C5FB0469C4F1000CC0FB0C32B4
:10FD2000C0FB0E69DBF8DC01DBF8804115904FF079
:10FD300000774FF0000AC4FB0E7A4FF00075486C54
:10FD40004FF00008C4FB00581598C0FB0C7AC0FBAC
:10FD50000E58D1F848E0DBF804C1DBF85801CCFBC1
:10FD60000E32CC6CCCFB0469C4F1000CC0FB0C322D
:10FD7000C0FB0E69DBF8D801DBF884411590C4FBA9
:10FD80000E7AC86CC4FB00581598C0FB0C7AC0FBF7
:10FD90000E58D1F850E0DBF808C1DBF85401CCFB79
:10FDA0000E324C6DCCFB0469C4F1000CC0FB0C326C
:10FDB000C0FB0E69DBF8D401DBF888411590C4FB69
:10FDC0000E7A486DC4FB00581598C0FB0C7AC0FB36
:10FDD0000E58D1F858E0DBF80CC1DBF85001CCFB31
:10FDE0000E32CC6DCCFB0469C4F1000CC0FB0C32AC
:10FDF000C0FB0E69DBF8D001DBF88C411590C4FB29
:10FE00000E7AC86DC4FB00581598C0FB0C7AC0FB75
:10FE10000E58D1F860E0DBF810C1DBF84C01CCFBE8
:10FE20000E324C6ECCFB0469C4F1000CC0FB0C32EA
:10FE3000C0FB0E69DBF8CC01DBF890411590C4FBE8
:10FE40000E7A486EC4FB00581598C0FB0C7AC0FBB4
:10FE50000E58D1F868E0DBF814C1DBF84801CCFBA0
:10FE60000E32CC6ECCFB0469C4F1000CC0FB0C322A
:10FE7000C0FB0E69DBF8C801DBF894411590C4FBA8
:10FE80000E7AC86EC4FB00581598C0FB0C7AC0FBF4
:10FE90000E58D1F870E0DBF818C1DBF84401CCFB58
:10FEA0000E324C6FCCFB0469C4F1000CC0FB0C3269
:10FEB000C0FB0E69DBF8C401DBF898411590C4FB68
:10FEC0000E7A486FC4FB00581598C0FB0C7AC0FB33
:10FED0000E58D1F878E0DBF81CC1DBF84001CCFB10
:10FEE0000E32CC6FCCFB0469C4F1000CC0FB0C32A9
:10FEF000C0FB0E69DBF8C001DBF89C411590C4FB28
:10FF00000E7AC86F1691C4FB00581599C1FB0C7A84
:10FF1000C1FB0E580C241846142102FA04F342FACD
:10FF200001F220FA01F040EA030046F059F9129B71
:10FF300023F8040C384614270AFA04F34AFA07FA9D
:10FF400020FA07F040EA030046F04AF9129B23F832
:10FF5000020C304609FA04F349FA07F920FA07F0CF
:10FF600040EA030046F03CF9139BA3F87C002846C6
:10FF700008FA04F348FA07F820FA07F040EA030009
:10FF800046F02EF9139B1699A3F87E00129B0433BA
:10FF90001293139B043B1393DE4B40318B420BF5C2
:10FFA000807B7FF4A7AE0D9B0F9AD3F800329B1A8B
:10FFB0000D9A03F00703C2F800320E9B01330E9333
:10FFC000119B80331193089B803308930E9B122B57
:10FFD0007FF42BAD059B013305931A9B08331A93CD
:10FFE000FEF785BE0025F4E4079B4036002703F5A5
:10FFF000005807F001030E930B9B0B98079903F52C
:020000023000CC
:10000000805300EBC710D3F8183B0093D8F80022B8
:1000100007F0010344F042FD07F00103D8F8002285
:100020005B4203F488631344079A02EB83090020C0
:1000300052F82310D9F85C204FF000730446C1FB3E
:1000400004306FF07301C2FB01304FF4557ED9F8D4
:100050000420D9F85810C2FB0E30AF4AC1FB023061
:1000600041F6D47CD9F80820D9F85410C2FB0C30E2
:10007000AA4AC1FB023046F2B865D9F80C20D9F87B
:100080005010C2FB0530A64AC1FB0230A54AD9F880
:100090001010C1FB0230A44AD9F84C10C1FB023049
:1000A000D9F81410D9F84820C1FB053045F2840175
:1000B000C2FB0130D9F81810D9F84420C1FB0C302C
:1000C00040F22C71C2FB0130D9F81C10D9F8402045
:1000D000C1FB0E307421C2FB01300C2402464FF0EC
:1000E000140A184602FA04F342FA0AF220FA0AF055
:1000F00040EA030046F074F809F5805126F8400CF8
:100100000A684FF0007000234FF4D075C2FB05035E
:1001100041F67C054A68C2FB050349F2FC758A6812
:10012000C2FB0503814DCA68C2FB0503804A0D6905
:10013000C5FB02036FF0B3054A69C2FB05034FF428
:1001400012758A69C2FB0503CA696FF01301C2FB0D
:10015000010303FA04F243FA0AF320FA0AF040EA30
:10016000020046F03DF8DFF8CCA126F8200CA6F1FD
:1001700040030D930896DAE910ECD9F80021D9F87C
:100180005C114FF000700023C2FB0E034FF00075AE
:100190004FF0000BC2FB0C5BCCF10002C1FB020371
:1001A000C1FB0E5BDAE912ECD9F80411D9F8582139
:1001B000C1FB0E03C1FB0C5BCCF10001C2FB0103D0
:1001C000C2FB0E5BDAE914ECD9F80811D9F8542116
:1001D000C1FB0E03C1FB0C5BCCF10001C2FB0103B0
:1001E000C2FB0E5BDAE916ECD9F80C11D9F85021F4
:1001F000C1FB0E03C1FB0C5BCCF10001C2FB010390
:10020000C2FB0E5BDAE918ECD9F81011D9F84C21D1
:10021000C1FB0E03C1FB0C5BCCF10001C2FB01036F
:10022000C2FB0E5BDAE91AECD9F81411D9F84821AF
:10023000C1FB0E03C1FB0C5BCCF10001C2FB01034F
:10024000C2FB0E5BDAE91CECD9F81811D9F844218D
:10025000C1FB0E03C1FB0C5BCCF10001C2FB01032F
:10026000C2FB0E5BDAE91EECD9F81C11D9F840216B
:10027000C1FB0E03C1FB0C5BCCF10001C2FB01030F
:10028000C2FB0E5B0C24142103FA04F243FA01F3BF
:1002900020FA01F040EA020045F0A2FF0D9B23F88E
:1002A000020F14210D9328460BFA04F34BFA01FBBD
:1002B00020FA01F040EA030045F092FF089B23F882
:1002C000020D0893134B0AF1400A9A4509F580790B
:1002D0007FF451AFD8F800320E9A01379B1A03F021
:1002E0000703122FC8F8003206F140067FF481AEF2
:1002F00070E60699039846F080FA6FF00B04FEF75B
:100300003FBC6FF00404FEF73BBC6FF00504FEF742
:1003100037BC00BF103D0A00D4F8FFFF7CAFFFFFE1
:100320003CB6FDFF78940400C44902004CE8030089
:100330002464FFFF50390A000024FEF721BC00BFEF
:100340002DE9FF411C460D4628461146424A1FF042
:1003500037FC2768414B3B40062B05D0BA070AD132
:100360003A683F4B9A4206D139463E4845F26612FA
:1003700051F001F907460121384623F02FFA067C97
:1003800016F0010602D0384840F0B6F9012D2BD9FD
:100390006068062201A923F0CFF9DDE9015633494F
:1003A0005C2052F015FBEB0704461FD50135013EDA
:1003B000B6F5305F1CD905F590536563A6F5105668
:1003C00005F51055A3636562A6620023C4E90B33EB
:1003D0005DF038FB2061002835D1204649F0E9FA6C
:1003E000234924485CF046FC3546D8E7002DDFD190
:1003F0004FF40068C4F82880404650F056FD606213
:1004000028B9204649F0D5FA404640F0F3F8B6F551
:10041000105F04D3656305F59055A563D5E74FF4E8
:10042000905050F042FD606328B9204649F0C1FA6F
:100430004FF49050E9E74FF4905050F036FDA06330
:100440000028C2D1F1E72046394609F007FB2046D3
:1004500004B0BDE8F08100BF040002000F0080FF7F
:10046000942D090050570900173A09006CC709007C
:100470008B490900182D090010B50446407B47F050
:10048000CFFFA3689FED107A5A0800EE102A94F867
:10049000442004EB820423F00103626B13449A426C
:1004A00009D1F1EEC77ABDE81040B8EEC00A87EE78
:1004B000800A26F0B3BA32F9021B07EE901AF8EE62
:1004C000E77AA7EEA77AEAE70000000038B504460D
:1004D0000D46407B47F0A4FF45F2661229460448CA
:1004E00051F049F80146204609F0B8FA0E2038BD0F
:1004F0005057090038B50D460446407B47F090FF41
:100500000121284623F06AF9037CDB0702D5044861
:1005100040F0F2F82046294609F0A0FA0E2038BD36
:10052000173A0900F0B587B0084611461A4603ABE2
:100530000193274B0093032350F0DEFE40F2444129
:10054000039842F067FA40F24F510746049842F090
:100550006DFA20490646242052F03AFABDF81450AC
:100560001D49044600220B68D3F80005C0070AD5D0
:100570000132042A01F10401F5D10023A36033B94B
:10058000164840F09BF816498A5C2277F6E700226D
:10059000C3F80C25A3680122C3F81025A2683B7993
:1005A0002376C2F86035387908F0E6FE3EB1A268DD
:1005B00033796376C2F86835307908F0DDFEA368D8
:1005C0002D0A01222046A582C3F8002507B0F0BD00
:1005D00074250A0050C709004C1D0A00034C09008D
:1005E000461D0A00F0B50D4685B055F8044B064689
:1005F000A068174648F013FF02AB0193504B0093DD
:10060000701E294602233A461FF012FB2046029E26
:100610009DF80C5049F0DEF910B1204649F0E5F99B
:10062000666084F82050337B7568DB08E376F37BE3
:1006300084F82230B37B003B18BF012384F82130BB
:10064000B768737BA376384640F2E5224FF6FF7118
:10065000BF001FF09DFB384650F027FC94F8223075
:10066000E0601BB9384650F020FC206105F574436A
:100670002333B3FBF5F36B43590801F5740101F51E
:100680001051B1FBF3F14B08A26803F5740303F5B5
:100690001053B3FBF1F303EB5503B3FBF5F3013B4D
:1006A000C2F84835A268C2F828354B1EE382A36819
:1006B000C3F80815A3680122C3F81425606847F041
:1006C000F9FE204A00231146106890BB41F82340F0
:1006D0003BF0D8FBA36800250422A5772046C3F889
:1006E000002229464EF0F0FEA368D3F82025C3F877
:1006F0004025A368D3F82425C3F84425A368C3F88C
:100700000851A368C3F80C51A368C3F81051A3683B
:10071000C3F81451A368C3F80451A3680C22C3F8AA
:100720000423A26801230E2093606377E57705B068
:10073000F0BD0133042B02F10402C5D1CAE700BFAA
:1007400064250A00CC50012010B50C4C206890B1F3
:100750000B4B1B6883B95AF082FF236898422368C9
:10076000A0EB030038BF00F1FF3040F2EE239842C7
:1007700094BF0020012010BD0020FCE79C590120FF
:10078000EC500120024A136823EA0003136070470B
:10079000EC500120024A136803431360704700BF06
:1007A000EC50012038B50C4B1B78A3B10B4B1B68E8
:1007B0008BB90B4C25685AF052FF2060236813B99F
:1007C00023680133236035B9064B01221A70064BAA
:1007D00003F174029A6238BDA6680120EC50012032
:1007E0009C590120DC670120745D012010B504468E
:1007F0000BF054FAE3681BB90A4A1168A14203D10D
:10080000BDE810400BF05CBAA360074B1968E160CB
:10081000196809B119688C60116801B914601C600D
:10082000EEE700BFFC5001200451012008B50BF099
:1008300035FA044A1368013B1360BDE808400BF029
:100840003FBA00BFF050012008B50BF027FA044A68
:10085000136801331360BDE808400BF031BA00BFE4
:10086000F05001202DE9F041134E33680BB3134DC6
:100870000BF014FA2C681CB1BDE8F0410BF020BA63
:100880000F4A01232B603368346014601BB92B6856
:10089000013B2B60F0E7D3E900689F68C3E902449D
:1008A0000BF00EFA0EB14046B0470BF0F7F93B469D
:1008B000ECE7BDE8F08100BFFC500120F0500120C2
:1008C0000451012008B525F085F8C188034897290F
:1008D00014BF972242223FF017FF00BFFC3C0900E3
:1008E00010B5064A002352F83340844202EBC3019C
:1008F00001D90133F7E7486810BD00BF081E0A00A0
:10090000F0B595B0054601A80E4617461C4657F0AF
:100910003AFD10B1002015B0F0BD3A4631462846E8
:100920001FF02CFC2FF00AF8830703D10268034B59
:100930009A42EFD020600120EDE700BF6C2D090046
:10094000014A042333F09CBD68350A00F0B587B036
:10095000084611461A4602AB0193254B0093042327
:1009600050F0CAFC2349182052F032F8DDE9042384
:100970000361214B9A428CBF0123B3FBF2F3C360A6
:100980001E4BD3F8A431DDE9027604465BB317F0C1
:1009900095F980F00105EDB204F1150300930022F2
:1009A0002B4640F27951384610F01AFC04F1160338
:1009B00060600022009340F27C512B46304610F0DC
:1009C0000FFC01221146A060606810F08DFC01222E
:1009D000A068114610F088FC20465AF0E7F820B9CC
:1009E00005203FF055FE0125D6E7204607B0F0BDB3
:1009F00044250A0034C7090020A10700745D0120C6
:100A0000F0B50C4687B054F8045B064628461746F6
:100A100048F020FD284648F02AFD02AB0193094B1F
:100A200000933A462146701E04231FF001F9059BEE
:100A300000932846DDE90323029958F021FE0E2099
:100A400007B0F0BD24250A00F0B50C4687B054F875
:100A5000045B06462846174648F0FCFC284648F04A
:100A600006FD02AB01930A4B00933A462146701EE5
:100A700004231FF0DDF801230193059B0093284612
:100A8000DDE9032302995CF06EFF0E2007B0F0BD94
:100A900004250A00F0B50C468BB054F8045B0646FA
:100AA0002846174648F0D6FC284648F0E0FC03AB41
:100AB00001930E4B00933A462146701E07231FF008
:100AC000B7F800230193079B0093DDE90312069B0F
:100AD00028465CF048FF099B00932846089B059A2E
:100AE000039958F0CDFD0E200BB0F0BDCC240A00C8
:100AF000F0B50D4687B055F8044B0646204617461C
:100B000048F0A8FC204648F0B8FC02AB0193204B0B
:100B100000933A462946701E04231FF089F840F2DC
:100B2000EB4301220021039850F019FC40F2DB4313
:100B3000012200210646C5B2049850F010FC4FF483
:100B40003373092208210746059850F008FC0299E2
:100B5000104AB2FBF1F301FB132202B1013323610E
:100B6000237DC3F38002AA420AD066F38203237571
:100B70006B1E594260684FF00002594110F0B4FBFF
:100B8000237D0E2067F3C303237507B0F0BD00BFBC
:100B900094240A0020A107002DE9F04186B0084600
:100BA00011461A4603AB01932D4B0093032350F0DB
:100BB000A3FB2C49182051F004FF2B4B059ED3F8C2
:100BC000A431DDE903870446002B47D017F076F8FF
:100BD00080F00105EDB204F11503009300222B46CD
:100BE00040F20531404610F0FBFA217D60600022A2
:100BF000C1F3800110F078FB04F116030093012289
:100C00002B4640F29341384610F0EAFA227DA0606C
:100C1000B0F10E0318BF012363F34102930722755D
:100C200003D50022114610F05FFB04F11703009377
:100C300001222B4640F28441304610F0D1FA0523C0
:100C40002361237DE06023F00D030E2818BF43F0DD
:100C500001032046237506B0BDE8F0810125BAE7FF
:100C6000B4240A0018C70900745D01202DE9F04F73
:100C70000D468DB055F8044B06462046174648F001
:100C8000E9FB204648F0F9FB08AB01934A4B00937F
:100C900029460423701E3A461EF0CAFF062205A903
:100CA000089822F049FD9DF81C10002240201FF0FA
:100CB00003F9099B04930546069B0A99B3FBF0F3DD
:100CC00003AA04A8039357F076FB049E039B6E438C
:100CD0005D4304960395002D4BD0237DDF0704D49C
:100CE000364840F284413FF023FD9807DDF814A018
:100CF000DDF82C90276940D4554406EB0A083544AA
:100D00005FFA89F64FF0080B4FF0000A237D990730
:100D100003D5A068F1094BF025FD217D0A0735D4E4
:100D200038462EF0A7FF217D606881F00401C1F3F1
:100D300080014BF017FD0DF10B01E0684BF0F9FC61
:100D40009DF80B30217D43EA4A0A0B072BD4384625
:100D50002EF090FF217D6068C1F380014BF002FD11
:100D60007600BBF1010BF6B2D0D108F801AB4545D6
:100D7000C6D10E200DB0BDE8F08FA06800214BF069
:100D8000F1FC0028B8D105203FF082FCC1F38001BE
:100D900081F00101606801F001014BF0E3FC38468D
:100DA0002EF068FFC7E76068C1F380014BF0DAFC02
:100DB00038462EF05FFFD3E75C240A00E0450900C7
:100DC0002DE9F04F0D468BB055F8044B06462046F2
:100DD000174648F03FFB204648F04FFB07AB019316
:100DE000444B0093294603233A46701E1EF020FF11
:100DF000052204A9079822F09FFC9DF818100022F4
:100E000040201FF059F8089B03930546059B09995C
:100E1000B3FBF0F302AA03A8029357F0CCFA039BAA
:100E2000029A6B43554303930295002D5AD0227DBD
:100E3000920704D4304840F293413FF079FC049A81
:100E4000D4F8109002EB0308002798F800604FBB1D
:100E5000A068F1094BF086FC002847D0BA46217DF6
:100E60000B0708F1010B24D448462EF003FF217D27
:100E7000606881F00401C1F380014BF073FC4846C7
:100E80002EF0F8FE217D6068C1F380014BF06AFC12
:100E90000AF1010ABAF1080F21D07600F6B203E098
:100EA000D846D2E74FF0000AA068F1094BF05AFC8F
:100EB000D5E7C1F3800181F0010101F00101606813
:100EC0004BF050FC48462EF0D5FE217D6068C1F302
:100ED00080014BF047FC48462EF0CCFED8E70137A6
:100EE000BD42DDD10E200BB0BDE8F08F05203FF0F4
:100EF000CFFB00BF7C240A00E04509002DE9F04F3C
:100F00000D4697B055F8044B06462046174648F064
:100F1000A1FA204648F0B1FA10AB0193614B00935F
:100F200029460623701E3A461EF082FE05220DA9B0
:100F3000109822F001FC9DF83C10002240201EF089
:100F4000BBFF129B1399099305460E9BB3FBF0F36D
:100F500008AA09A8089357F02EFA06220AA91198A0
:100F600022F0EAFB9DF83010002240201EF0A4FF82
:100F7000149B1599079306460B9BB3FBF0F306AA47
:100F800007A8069357F017FA089A099B06996B432E
:100F90005543079A099372434E43B5420895079209
:100FA000069602D040483FF0BBFB002D76D00D994D
:100FB000C8180390207D860706D4CE1826B140F2CB
:100FC00093413A483FF0B4FB0A9EC00706EB020A81
:100FD00005D4BAF1000F02D040F28441F1E7CE5CB3
:100FE000A068D4F810B0F1094BF0BCFB00283BD14D
:100FF00005203FF04DFB7600F6B2A068F1094BF0FA
:10100000B1FB217D0A0733D458462EF033FE217DF3
:10101000606881F00401C1F380014BF0A3FB0DF186
:101020001701E0684BF085FB9DF81730217D43EAFE
:1010300049090B0729D458462EF01CFE217D606813
:10104000C1F380014BF08EFB08F10108B8F1080FE5
:10105000D1D10AF807900137BD421FD0039B4FF052
:101060000008DE5DC146C8E70027B846B946C8E7B4
:10107000C1F3800181F00101606801F001014BF0D2
:1010800071FB58462EF0F6FDC9E76068C1F3800198
:101090004BF068FB58462EF0EDFDD5E70E2017B05B
:1010A000BDE8F08FCC250A00903D0900E04509001D
:1010B0000E2AF7B506460D46174602D133483FF0D3
:1010C000AFFA806848F0ABF9AA0706D12A68304B1E
:1010D0009A4202D12F483FF0C7FAEB071FD5B288DA
:1010E000F3885343B3EB650F4FEA650405D8013B22
:1010F00000225C2128483FF0ABFA94FBF2F502FB9A
:101100001544042F24B22DB22AD12A462146304656
:1011100048F0FCFD400040F0010003B0F0BD01AA22
:101120000221284624F08EFB019B186851F076F8C6
:10113000041EB38801DB9C4204DB013B002240F229
:101140007A61D7E7019B586851F068F8051EF3886B
:1011500001DB9D42D5DB013B00224FF4D061C9E7A2
:10116000384651F05BF8B27B4FF0FF31C2F12002FC
:1011700021FA02F2A223002150F0F1F82A46034698
:101180002146304648F0F8FD0E20C6E7954A090092
:10119000CC580900264309000D4E09002DE9F04FF7
:1011A00093B00DAB0193684B009305231EF040FDF7
:1011B0000D9D664940F2553228461EF01FFEDDF8AF
:1011C0003880624940F2CB5240461EF017FEDDF8EF
:1011D0003C905E4940F2CC5248461EF00FFE109CF7
:1011E000204625F0F1F920B12146594850F0B7F9D1
:1011F0000446012120464EF08AFD824660B9204611
:1012000024F0E8FBC3880093524840F20E234322A7
:1012100040F259413FF078FA119F0E2F13D04B49FD
:1012200040F2644238461EF0E9FD4146284607F088
:10123000D7FE4946284607F0D3FEAB7B102B04D0DF
:1012400045483FF06DFA0027EFE7EB88049300264E
:10125000049BB34203DC0D9813B0BDE8F08FAB895B
:10126000AA68734302EB83030593AB880693B8F82F
:101270000C30D8F80820734302EB83030393B9F8CA
:101280000C30D9F80820734302EB8303089333B280
:101290004FF0000B0B93069B5B4501DC0136D7E753
:1012A000039B33F8024B03933FB10B9A0FFA8BF178
:1012B000384648F02BFD00283FD163BAADF8243002
:1012C000089B33F81B305ABAADF82820C3F3C40288
:1012D000C4F304210792C4F3002242EA4102C3F39B
:1012E000042EC3F3002141EA4E014FF0400012FBEF
:1012F000001207991AF80220C4F3C40CC3F3C00308
:10130000C4F3C00443EA410344EA4C04402114FB03
:101310000134099B1AF804406408E40244EA5204C8
:101320000A9AC3F34513C2F3451213FB01231AF8BB
:10133000033044EA431464BAA4B2059B23F81B406B
:101340000BF1010BA7E700BF0C260A00C0C2090081
:101350006CC50900B64D09006E30090070B586B045
:1013600003AB0193164B009303231EF061FC039E15
:10137000144940F2C92230461EF040FD049D124936
:1013800040F2CF4228461EF039FDA86840F2CF4215
:101390004FF480711EF0F0FC059C0E2C0DD0094915
:1013A00040F2644220461EF029FD30466A6821461C
:1013B00037F01EFC039806B070BD0024F5E700BFAF
:1013C00044260A00C0C209001CC209002DE9F04FE2
:1013D000A7B003AB01934B4B009303231EF028FCF3
:1013E000039D494940F2C92228461EF007FD049C8E
:1013F000204624F0EFFAC37B002B40D000EB8300A3
:10140000424B02699A423AD1606840F25942032144
:101410001EF0B2FCD4E90378A4680DF11809002687
:10142000324621461F2058F03BFC444509F8010B89
:1014300004D0324641461F2058F032FC0136202E9F
:1014400089F85F00ECD10DF13706002422463946B9
:101450003F2058F025FC0134402C06F8010FF5D14F
:10146000059F0E2F0ED0284940F2644238461EF0E8
:10147000C5FCAB7B102B07D025483FF051F9A046A7
:101480002746CAE70027F4E7B5F806900026B145DD
:1014900003DC039827B0BDE8F08FAB89AC68B5F8E2
:1014A00004A0734304EB83044FF000080FFA86FB9B
:1014B000C24501DC0136EAE737B15A460FFA88F136
:1014C000384648F023FCC8B9228853BAC3F3451301
:1014D00098336B4413F8601CC2F30423C2F3C402B4
:1014E000983398326B446A4413F8203C12F8802CED
:1014F00043EAC22343EA41135BBA238008F101089F
:101500000234D5E75C260A00C0C209008D7F0500C1
:101510006E3009002DE9F04FABB00FAB0193924B49
:10152000009303231EF084FB0F9C904940F2C922D4
:1015300020461EF063FC3022002112A84FF090FDDF
:10154000109E16F0030566D13368894A934224D170
:1015500012AF294630464EF020FA01353B46032DA6
:1015600007F1140783ED000AF3D1119F0E2F63D00A
:101570007E4940F2644238461EF040FC12AD0DF147
:1015800078080026731E0B2B71D8DFE803F06D700E
:10159000686A706A57706D706873764A934217D1A3
:1015A0000DF148084746294630464EF0F6F94346C5
:1015B000691C83ED000A30464EF0EFF90235062D26
:1015C00087ED030A08F1140807F11007EBD1CCE707
:1015D000694A934211D14FF00308294630464EF034
:1015E000DCF9B5FBF8F72AAB2F44013503EB87078D
:1015F000092D07ED180AF0D1B7E7604A93420AD1E6
:1016000012AF294630464EF0C8F901350C2DA7EC33
:10161000010AF6D1A9E7304624F0DCF9C38801932A
:101620004FF487730093564840F20D1340F227227F
:1016300040F226213FF07CF800279FE7514BB5ECA4
:10164000010A07EE903AF8EEE77A013627EE800AB3
:1016500035F03EFDBDEEC00AA8EC010A92E74A4B08
:10166000EDE74FF40033EAE74FF40043E7E74FF4C8
:101670008033E4E7A37B102B02D044483FF050F8BE
:101680001E9B02931F9B0393209B0493219B059316
:10169000229B0793239B0893249B0993259B0A93E2
:1016A000269B0B93279B0C93B4F80690289BDDF8A0
:1016B000A4A00D930026B14503DC0F982BB0BDE824
:1016C000F08FA389A568B4F804B0734305EB8305D4
:1016D0004FF0000832B2C34501DC0136EBE747B1F9
:1016E0000FFA88F13846069248F010FB069A002857
:1016F00035D1B5F800C0039B9CFA9CF1C1F34511AC
:1017000003FB01F0029BCCF3C40E03FB0E00049B11
:10171000CCF3042C03FB0C00059BC3180693089B19
:1017200007984B4300FB0E33099800FB0C330A98D3
:1017300003440C9841430B9800FB0E110D9800FBDD
:101740000C110698A3F306435144A0F305405B0136
:1017500043EAC023A1F305410B435BBA2B8008F198
:1017600001080235B7E700BF8C260A00C0C2090095
:1017700098C6090048C60900ECC5090084C50900DF
:10178000DB2F0900C1FF3E00E1FF1E006E300900A3
:101790002DE9F04F2DED028BA7B002AF07F17003DA
:1017A00001938F4B009308231EF042FAD7F870B0D4
:1017B0008C4940F2C92258461EF020FBD7F88C30E5
:1017C0003B660E2B1CD0874940F2644218461EF03F
:1017D00015FBF86F24F074F8D7F874804046F0EEEB
:1017E000408A24F0B1FFC4070DD4404624F0F2F83B
:1017F0004FF40B72C3887C484FF4CD613EF098FFE4
:1018000000233B66E5E7441007EE904AB8EE677A9E
:10181000F1EEC77AFDEEE77A17EE905AE90703D5A5
:1018200005FB05F39C4202D070483EF079FFA3000F
:10183000073323F00703ADEB030D02AB4FF00009B4
:101840007B654E46A1451AD1B86F0E2828D024F0EA
:1018500037F8B0EE408A6B08FB6697F880307B6300
:1018600097F884303B6397F88830FB62FB6E013356
:10187000BB669BF80E30102B1FD05D48D5E74FEAB2
:101880004901042241F00101404626F0C7FA50F018
:10189000C5FC7B6D064443F8290009F10109D1E735
:1018A000B7EE007A36B107EE906AF8EEE77A87EE87
:1018B000278AD0E7B0EE478ACDE7BBF804304D4D1C
:1018C0004D4CD5F800A001335B10BB65BA6DBB6E03
:1018D00002FB03F6B60040D1BAF1000F02D0504629
:1018E00032F08EF9002323602B609A469FED430A65
:1018F00028EE000A35F0ECFBFDEEC07A9FED400AC1
:10190000C7ED127A28EE800A35F0E2FBFDEEC07AD0
:10191000BBF806303B6217EE903A5B007B61FB6ED2
:10192000C7ED117A5B42FB65FB6E5B003B614FF0DC
:1019300000093B6A4B4500F3D181BBF80650FB6EB2
:10194000EC1A24EAE474A54200F33383386F943729
:10195000BD46BDEC028BBDE8F08FBAF1000F00F080
:10196000B38123689E42C1D9264B1C6820465AF099
:10197000FBFC864280F09F8155460C2E55F8043DB5
:10198000B04623F0030938BF4FF00C08C14580F082
:101990009B8005EB09004168CA0706D521F00301C9
:1019A00009F104030B4443452ED2314620465AF038
:1019B000E2FC0546002800F07E81B1454A465146CA
:1019C00028BF32464FF00BFB514620463DF074FADB
:1019D000AA46084BC3F800A0074B1E6086E700BF6D
:1019E0008C250A00C0C209009E4D0900EF2F090096
:1019F0006E300900A8610120AC6101200000804721
:101A000000007C4ACC560120638AC3F3C713994275
:101A1000AAF1080980F007812269C2F38532B3FB7D
:101A2000F2F30022B1FBF3F37B66D0E902C1CCF8FC
:101A30000C10C1F808C021697B6ED4F820E0C1F316
:101A4000853102FB01315EF8213098421AD1A4455C
:101A50004EF821C016D1D4F81CE07B6E5EF822103F
:101A60004FF0010C0CFA03F321EA03014EF82210A7
:101A7000E36953F822302BB9A3690CFA02FC23EA7C
:101A80000C03A3615AF8043C4268043322F00302B9
:101A900013444AF8043C23F0030343F80590BA4B7F
:101AA0001BB101221021AFF300805AF8043C23F04F
:101AB00003032B445A6822F002025A605AF8043C8D
:101AC00023F001034AF8043C23F0030308F1100259
:101AD0009342FFF47EAF4544A3EB08036A68043BDE
:101AE00002F0030213436B605AF8043C03F0030353
:101AF00043EA08034AF8043C6B6805F1080E23F03A
:101B00000303734443F8045C53F8042942F00202CF
:101B10005A60686820F0020320F0030043F00103DC
:101B200070446B6050F80419CB074DD5638A21F0DF
:101B30000301C3F3C7138B4240F28E8022694FF03A
:101B4000000CC2F38532B3FBF2F3B1FBF3F37B6617
:101B5000D0E90212CA60916022697B6ED4F82090AD
:101B6000C2F385320CFB023259F82230984219D167
:101B7000A14249F8221015D1D4F81C807B6E58F888
:101B80002C20012101FA03F322EA030248F82C2059
:101B9000E36953F82C302BB9A36901FA0CF123EA5D
:101BA0000103A3616B684268043322F0030213440B
:101BB0006B6023F003039E44734B4EF8045C1BB12F
:101BC00001221021AFF300806968638A206921F047
:101BD0000301C3F3C7139942C0F3853053D2B3FB5B
:101BE000F0F3B1FBF3F30022216A02FB003051F85D
:101BF0002010C5E90214CD602169206AC1F3853146
:101C000002FB013140F821500125A16905FA02F0DB
:101C10000143E069A16150F8221005FA03F319436A
:101C200040F82210D5E6A9B1B1FA81F2C2F1200242
:101C300094F812C0531ECCF3021CA3EB0C0321FA40
:101C400003F3012101FA0CF14B40217C7B66A2EBEE
:101C50005112EAE60A46EBE799B1B1FA81FCCCF100
:101C6000200CA27C0CF1FF33C2F302129B1A21FA62
:101C700003F301219140227C4B407B66ACEB521C6C
:101C800066E78C46EDE7A1B1B1FA81F2C2F120021C
:101C900094F812C0531ECCF3021CA3EB0C0321FAE0
:101CA00003F3012101FA0CF14B40217CA2EB51120C
:101CB0009AE70A46ECE7504631F0A2FF334B002288
:101CC0001A6030463EF096FC304632F049F8266005
:101CD0008246286000287FF409AEF2E7BBF80C309A
:101CE000DBF8082009FB03F302EB8303BA6EFB6306
:101CF000BB6EB9FBF3F302FB1393BA6D53430AEBCC
:101D00008303FB61BBF80430BB613B690133BB63F8
:101D1000FB6EA9EB0303BB600FFA89F34FF00008D9
:101D20007B60BB6943451DDCFB6E4B4517DCBBF894
:101D30000C00BD6EBC6EBBF80420A9EB0301484348
:101D4000B1FBF4F405FB1411BC6DDBF80830614302
:101D500052000AEB810103EB80004FF040F909F1DA
:101D60000109E6E53B6E9BB17A680FFA88F11846E7
:101D700047F0CCFF60B1FB6B33F81830FA6922F8FA
:101D8000183008F10108CCE700000000A86101202C
:101D9000DBF808103964BBF80C103965F96EBBF834
:101DA0000430BBF80620414500F3BC80591A884531
:101DB00080F2B880F96E494500F3B480511A894524
:101DC00080F2B080BB683A6DD7F85CC002FB03F4C8
:101DD000A300FB643B6C002003EB4803BB6202469C
:101DE000786601467B6DFC6CFE6D03EB80033B6403
:101DF000BB6A23447B627B6A33F816503B6C53F812
:101E000004EB3B646CBAC5F3C4030EFB0311C4F3CB
:101E100045137C6E0EFB03437B66FB6E0136C5F3F8
:101E20000425B3420EFB0522E5DABB6B1844D7E963
:101E3000134304EB8303FB64FB6E0CF1010C63455D
:101E4000D0DAD7E911307C6E01FB00317B6904FBED
:101E50000033D7E91104A3F3064302FB0402A1F304
:101E600005415B01A2F3054243EAC12313437A6BA8
:101E7000002A54D01D1205F0F8027A66DA1002F03A
:101E8000FC01DB003965D9B2F964F96B31F818004F
:101E900041BAC1F3CC0606F0FC043C64FC6CC3F30D
:101EA000421323437C6EC5F3421525433C6DC2F3B8
:101EB0008112224302EB8202C2EB0212262415FB9E
:101EC00004254FF00F0413FB04533C6C3A6BC6F32C
:101ED0008116344300F0F80CC900C0F3421004EB43
:101EE000840401F0F80E4CEA0000C1F34211C4EB87
:101EF00004144FF02605C2EBE3134EEA01010F2252
:101F000010FB054011FB0201B3EBE11FF96AB4BFFE
:101F1000012200224FF6FF738A4208BF00235BBAFA
:101F20009BB22BE70024013A013BFE6DBA627B6253
:101F300022467C662146BB6AD7F85CC009EB0600E6
:101F400020EAE0709842A8BF18463B6D4343FB600F
:101F50007B6D03EB8403FB647B6A08EB0C0525EACD
:101F6000E5759D42A8BF1D463B6C03EB4505FB682C
:101F700035F82350FB6C53F804EBFB6468BAC5F3E7
:101F8000C4030EFB0311C0F34513786E0EFB03036D
:101F90007B66FB6E0CF1010CC5F3042563450EFB5B
:101FA0000522D9DABB6B1C44FB6E0136B342C2DAA0
:101FB00047E7BE6EBBF80C00B96EB4FBF1F106FB4F
:101FC0001141BE6DDBF80830BBF80420604371435B
:101FD00052000AEB810103EB80004FF000F801345E
:101FE000B1E400BF2DE9F04F2DED028B89B005ABB8
:101FF00001935E4B009303231DF01AFE0698C8B1AF
:1020000023F05EFCB0EE408A059C594940F2C9229B
:1020100020461DF0F3FE079F0E2F0ED0544940F2CC
:10202000644238461DF0EAFEA37B102B07D05148CE
:102030003EF076FBB6EE008AE6E70027F4E79FED78
:102040004E0A28EE000A35F043F8B4F806A0BDEEBB
:10205000C08A00264FF0260B4FF04009B24505DC40
:10206000059809B0BDEC028BBDE8F08FA3880393FF
:10207000A389A568734305EB83054FF00008039B14
:10208000434501DC0136E9E73FB132B20FFA88F18E
:10209000384647F03BFE002864D129884BBA01F04E
:1020A000F802C1F342111143C3F3CC0202F0FC0C5D
:1020B000C2F3811242EA0C00DB0000EB800203F065
:1020C000F80EC2EB0212C3F3421343EA0E034FF0C1
:1020D0000F0C18EE10EA11FB0B2213FB0C22BEEBC7
:1020E000E21F4FEAE21C3DDACCEB4E024FF6D57C04
:1020F00010FB0CFC4FF6EB7E11FB0ECC4FF6CA7EAC
:1021000010FB0EF011FB09014FF6F67013FB09CC22
:1021100013FB0013DB114BF2D2614FEAEC1C594365
:1021200045F61A0000FB0C11144882F30802A2EBDA
:102130002141434302EB2343114881F30801C900C5
:1021400083F3080301F4FC6100EA03230B430D4908
:1021500001FB0CFC02EB2C4282F3080243EAD2039F
:102160005BBA2B8008F10108023588E774260A0063
:10217000C0C209006E30090000008043E96601001A
:1021800000F8FFFFA2C501002DE9F04F2DED028BF5
:102190009FB014AB0193A94B00930A231DF048FD97
:1021A000A749149840F256321DF028FEA44940F287
:1021B000BD52074615981DF021FEA149834640F205
:1021C000BE5216981DF01AFE049018980E2836D0AC
:1021D00023F076FBF0EE408A19980E2832D1B7EE44
:1021E000008A38EE688A179E964940F212323046CD
:1021F0001DF004FE1A9D944940F2D72228461DF096
:10220000FDFDBB88BBF80410994215D1FA88BBF8D4
:102210000630934210D1B87B9BF80E2082420BD13E
:1022200004988088884207D10499C988994203D1CB
:10223000049B9B7B93420AD084483EF071FAF6EEF1
:10224000008AC9E723F03CFBB0EE408ACBE7347943
:10225000092C0EDC0121A14011F0AA0F05D1092C97
:1022600007D1082B07D07A48E7E7102B03D079482D
:10227000E3E77948E1E71B98B5F904500E281FD031
:102280004FF0CCFF0023089009931C980E281CD017
:102290004FF0C4FF00230A9005931D980E281ED00E
:1022A00040F2644266491DF0A9FDBB8882889A42CB
:1022B000804603D1C288FB889A420BD06748BCE7AE
:1022C00000230121CDE90831DFE701230593002335
:1022D0000A93E2E7837B082B03D06148ADE74FF018
:1022E0000008EBB20B93BB88ADF848300025FB88A3
:1022F000119511A93846ADF84A3013950FF026FF15
:10230000F0EE687AFEEECC7A092CCDED027AF0EE92
:10231000487AFEEECC7ACDED067A40F0BD809DF88D
:10232000203007939DF828300699089378E0BA8901
:10233000BB68DBF808406A4303EB820ABBF80C3049
:102340006B4304EB83030393049B9A899B686A4362
:1023500003EB8202B8F1000F00F09C80B8F80C008B
:10236000D8F80830684303EB8000D64652E0099B5A
:10237000002B5ED1039B079E1B789B1B18BF01237C
:10238000059E002E57D11678089C361B18BF0126D3
:1023900070B190F800C00699BCF1000F0CBF002688
:1023A00006F0010601FB0CF17F31FF2491FBF4F1F3
:1023B000002B63D0039C14F8013B0394029C6343FD
:1023C000002E57D00B9C12F8016B012C01FB06F676
:1023D00048D106FB03FC0CF57F4909F1FF093CEAF3
:1023E0002C0C28BFCC461E44A6EB2C46029B4B432C
:1023F0009C4648BF03F1FF0C029B0B44A3EB2C232C
:10240000002B45DD96FBF3F383F308030EF8013B45
:1024100000B10130BE88AEEB0A039E42A7DC013555
:10242000FB889D4283DB0E201FB0BDEC028BBDE814
:10243000F08F0123A4E7059EAAE700BF24270A0026
:10244000C0C2090088C20900C0C40900624B09006B
:10245000ED470900D14709005B40090063460900C8
:1024600076460900C1F58074634348BFFF3306EB2D
:102470002326BBE7002B06DAFF3304E02EB112F867
:10248000013B4B43F8D41B12BEE79EF80030BBE77C
:102490000023B9E7404668E704F0FB03069E0D936E
:1024A000FB889D42BFDABA89BB686A4303EB8203AB
:1024B000BBF80C200C93DBF808306A4303EB820373
:1024C0000E93049B9A899B686A4303EB82030F93E4
:1024D000B8F1000F00F00481B8F80C20D8F80830EB
:1024E0006A4303EB820307930023A7E00E9B039A42
:1024F000039933F812200F9B33F811100D9B032B17
:10250000099B01BF52BA49BA92B289B2002B40F07E
:102510009D80089BB3EB020C18BF4FF0010C059B8C
:10252000002B40F096800A9B5B1A18BF0123079886
:1025300080B10446069814F801EB079400FB0EF6F0
:10254000BEF1000F0CBF002303F001037F36FF2014
:1025500096FBF0F6BCF1000F00F0A880002B00F015
:102560008E80029B0298734348BFFF3300EB06093D
:10257000A9EB2329B9F1000F5EDD1312D410D200AC
:1025800003F0F80304F0FC04D2B243434443424353
:102590000B984FEA212E4FEAE10CC9000EF0F80E1D
:1025A0000CF0FC0CC9B2012806FB0EFE06FB0CFC6D
:1025B00006FB01F14FD10EFB03FA0AF57F40FF3015
:1025C0003AEA2A0A28BF824673440CFB04FEA3EBB6
:1025D0002A430EF57F4A0AF1FF0A3EEA2E0E28BF73
:1025E000D646644401FB02FCA4EB2E440CF57F4E5E
:1025F0000EF1FF0E3CEA2C0C28BFF44602EB010A58
:10260000AAEB2C4A0D9A93FBF9F394FBF9F41B0205
:10261000E40003F4784304F4FC6423439AFBF9FADE
:10262000032ACAF3C40A43EA0A0301D15BBA9BB284
:102630000C9A039922F81130039B01330393039AF8
:10264000BB889A42FFF652AF013529E74FF0010CE3
:1026500065E7059B6BE7C6F5807A5046434348BF64
:10266000FF33444348BFFF345043024648BFFF3264
:102670000EEB23230CEB242401EB222AC2E7029B5E
:10268000029802F47841594302F4FC6343434FEA51
:10269000212148BFFF3341EA2323029902F01F02A0
:1026A0004A4348BFFF3243EA2223C0E79BB101F40B
:1026B000784201F4FC63734306FB02F201F01F0150
:1026C00048BFFF331212714342EA232348BFFF3150
:1026D00043EA2123ABE70C9B039A33F81230A7E7B8
:1026E000CDF81C8000E700BF2DE9F04F99B011AB89
:1026F00001933F4B009307231DF09AFA3D4911982F
:1027000040F2C9221DF07AFB054605220BA912985A
:1027100021F012F8EB88AA8813A909A801F0DEFAC3
:10272000BDF92830BDF92690BDF924A0BDF92AB025
:102730000493A3EB0A049DF83410ABEB09030022C9
:1027400040205C431DF0B8FB0C9BB3FBF0F6179BDD
:1027500005900E2B4F46039308D018464FF05EFDB0
:102760000690B44205D924483DF06AFF0023069341
:10277000F7E7AB7B0B9C01269E40013EBB4534DC5A
:10278000049BADF83C30284600230EA9ADF838A0D4
:10279000ADF83A90ADF83EB010930FF0D7FC0E2094
:1027A00019B0BDE8F08F059B022B18D0042B19D06F
:1027B00014F8013B03990E2902D00699994207D0DB
:1027C00033400FFA88F1284607920FF0E3FC079A8E
:1027D00008F10108049B4345E5DC0137CEE734F8F6
:1027E000023BE7E754F8043BE4E7D0463AB2F1E7AE
:1027F00034280A00C0C209007B3809002DE9F04FD7
:1028000097B002AF07F140030193B54B0093042347
:102810001DF00EFAB349786C40F2BC521DF0EEFA8E
:10282000B049064640F25632386C1DF0E7FAFC6CAF
:10283000AD49814640F2912220461DF0DFFABD6C81
:10284000AA4940F2C15228461DF0D8FAB9F804A0AE
:10285000B388534509D1D9F80430BB60B9F80630C4
:10286000BB61BA69F388934202D0A1483DF044FFAE
:1028700099F80E30102B03D0012B01D09D48F5E7BD
:102880002A79092A06DC0121914011F0AA0F03D10F
:10289000092A06D09848E9E7B37B102B06D0974861
:1028A000E4E7B37B082B01D09548DFE7032AB4F9AE
:1028B000043053D0072A4FD0052A52D1002242F0CB
:1028C000020B904ADBB252F8235069780AEB4103BD
:1028D00003EB43035B0007336A46DB08A2EBC30349
:1028E0009D460A2301EB41084B4302AC03EB8A03EC
:1028F000D04404EB410204EB48081C440AF11F03D6
:1029000068465B09A0EB43139D46BA62C7F82C806A
:102910003C6343F8081B30467B62594600234CF069
:1029200074FE6B78009342460123594630464CF0C2
:102930006CFE6B78009322460223594630464CF0D9
:1029400064FE4FF000084446BB69434540F3DC8019
:10295000BB6A3B62002227E00122B0E74FF0010B87
:10296000AFE74FF0000BACE73B6A786A33F91230FF
:1029700023447F2BD4BF00210121802B8154B4BF7D
:102980000021FF215B1AFB61E81C4FF0000C297845
:102990008C4544DBAC78FB6914FB03F4002CB8BF16
:1029A000FF3444F30F2401329245DDDC7A6A41465C
:1029B00048465AF049FFFB6AFB61BB623B6B7B6197
:1029C000FB623B6A3B6308F101037B60BB6908F172
:1029D0000102934200F098806B7800933A6A08F104
:1029E0000303594630464CF010FE5246002A35D1BA
:1029F0007A6A796848465AF027FF7B69BB623B6A6E
:102A0000FB62FB693B636B780093FA6908F104038E
:102A1000594630464CF0F9FD08F1020894E790F968
:102A2000011090F9004007F1500303EB8101FB69AD
:102A300051F8281C796190F90210144411FB03F13C
:102A40007B69002933F814E0B8BFFF310EEB212E6B
:102A5000033023F814E00CF1010C98E7013AFB690C
:102A600033F81230234419B27F29D4BF002001204B
:102A700080297C6AB4BF0021FF215B1AA0543B610E
:102A8000E81C4FF0000C29788C4509DBAC783B69D9
:102A900014FB03F4002CB8BFFF3444F30F24A5E764
:102AA00090F9011090F9004007F1500303EB810108
:102AB0003B6951F8281CF96090F90210141B11FBB6
:102AC00003F1FB68002933F814E0B8BFFF310EEBC7
:102AD000212E033023F814E00CF1010CD3E700BFE2
:102AE00014290A00C0C20900A4C4090088C2090050
:102AF000CE3D09001D3209005E3009000F32090089
:102B0000063209000C290A00BA68002307F13401D3
:102B10004846C7E90E237B630FF018FB0E2054379D
:102B2000BD46BDE8F08F00BF2DE9F04395B00AAB7C
:102B30000193304B00930A231DF07AF82E490A982E
:102B400040F256321DF05AF940F27A638288044608
:102B500000210C984EF003FCE2884FF4D063002172
:102B600007460D984EF0FBFB234940F2BC528046CD
:102B70000B981DF043F90546C38882880EA908A862
:102B800001F0ACF8A27BAB7B9A4202D21B483DF02D
:102B9000C7FD12980E2825D04FF040FB4FF00009DA
:102BA000064613980E2821D04FF038FB0023CDE9BC
:102BB0000603BDF926300393BDF924300293BDF915
:102BC00022300193BDF9203000932046CDE90469FD
:102BD0000FFA88F33AB2294606F0DCFF0E2015B052
:102BE000BDE8F0834FF001090026DAE70123002059
:102BF000DDE700BF94280A00C0C209002D32090099
:102C00002DE9F04F91B00BAB0193974B0093052347
:102C10001DF00EF840F2563294490B981DF0EEF874
:102C20000E9B827B029301239340029A9A420646AE
:102C300002D38F483DF074FD0F9F6FF00042974222
:102C400003D0BB4201D88B48F4E7BDF93090B9F10D
:102C5000000F02DBB388994501DB8748EAE7BDF93D
:102C60003480B8F1000FF8DBF3889845F5DA029B61
:102C7000BB4200F0F58000201AF07EF90546484678
:102C80004FF0E7FE069040464FF0E3FE06A907909E
:102C9000022024F057F8014628464FF005FE6FF059
:102CA00000439F420CD106984FF0B8FA04460798AB
:102CB0004FF0B4FA21B202B2304647F027F8074687
:102CC000002304AA05A928460593CA464FF022FE10
:102CD000CDF80C80059A8AB9039BADF820900AF1D3
:102CE000010A013308A93046ADF82280ADF824A0CE
:102CF000ADF826300A920FF029FAB1E004AA05A92E
:102D000028464FF007FE0021284623F067FD0446C1
:102D100080684FF083FA8346E0684FF07FFA0FFA3D
:102D20008BF102B2304646F0F1FFB84205D004AA5A
:102D300005A928464FF0EEFDCCE7A0684FF00FFC48
:102D40008346E0684FF00BFCCB45039BB8BF0FFAFE
:102D50008BF9D345C8BF0FFA8BFA4045B8BF0FFABD
:102D600080F89842C8BF03B2A068C8BF03934FF071
:102D700055FA8346E0684FF051FA029B02B20FFA0F
:102D80008BF130460FF006FAE0684FF0E8FB0028C0
:102D900011DDA3680893E0684FF0E1FB01384000C3
:102DA00040F00100099008A9022023F0CBFF014662
:102DB00028464FF079FDA0684FF0D1FB002811DDC7
:102DC000A0684FF0CCFB0138400040F001000890B3
:102DD000E368099308A9022023F0B4FF01462846BE
:102DE0004FF062FDA0684FF0BAFBB3880130984203
:102DF00011DAA0684FF0B3FB0130400040F0010051
:102E00000890E368099308A9022023F09BFF01467C
:102E100028464FF049FDE0684FF0A1FBF3880130F0
:102E2000984211DAA3680893E0684FF098FB0130EC
:102E3000400040F00100099008A9022023F082FF21
:102E4000014628464FF030FD04AA05A928464FF058
:102E500061FDFDF707FD094B9B6A002B3FF43AAF7C
:102E60000E2011B0BDE8F08FA4270A00C0C20900EF
:102E70000F300900FD3D090082330900745D012017
:102E80002DE9F04F93B00DAB0193714B00930523E7
:102E90001CF0CEFE40F256326E490D981CF0AEFF8B
:102EA000827BDDF84480012393409845044602D399
:102EB00069483DF035FCBDF938A08288BDF9406015
:102EC00040F27A63002150464EF049FABDF93C9039
:102ED000E2884FF4D063002148464EF040FA40F2B9
:102EE0000D52002130464EF032FA0EAA8CCA00254F
:102EF000D11BCDE909553A44ADF81C10D91B3B4410
:102F0000ADF82020ADF82230A388ADF81E1007AA36
:102F10001046ADF82C300AA9E388ADF82E300C9598
:102F200049F0C3FD07A920460FF010F94B4940F2C4
:102F30007A6347F6FF7250464EF011FA4FF4D063B1
:102F400047F6FF72454948464EF009FAA088E288E4
:102F500050454FEA4703A8BF5046C3F103034A4513
:102F60001BB200B2A8BF4A4612B2039320EAE07334
:102F7000049322EAE277B54203DD0E2013B0BDE8E8
:102F8000F08F049B06EB070B05EB03090FFA8BF29E
:102F90000FFA89F1434620460FF0FCF8049BA7EB9B
:102FA000060A591B09B20FFA8AF2434620460591D8
:102FB0000FF0F0F80FFA8BF20599434620460FF018
:102FC000E9F80FFA8AF20FFA89F1434620460FF02A
:102FD000E1F8049B05EB070B03EB06090FFA8BF2F4
:102FE00043460FFA89F120460FF0D4F8049BA3EB77
:102FF000060A0FFA8BF24346A7EB050B0FFA8AF18C
:1030000020460FF0C7F843460FFA8BF20FFA8AF109
:1030100020460FF0BFF80FFA8BF243460FFA89F102
:1030200020460FF0B7F8039B002BC5BF039BAA1BDC
:1030300006330A33D2BF03EB850303EB820306F1A9
:10304000FF361BB2C8BF36B20393013593E700BF0A
:10305000E4280A00C0C20900823309000080FFFF93
:103060002DE9F0438FB008AB01932A4B0093062360
:103070001CF0DEFD40F25632274908981CF0BEFED7
:10308000827BDDF83490012393409945044602D3B6
:1030900022483DF045FB0B98099A0C990A9B15B202
:1030A00007B21EB20FFA81F8BD42B5BF421C3846C6
:1030B000284601324645B4BF4B1C0133ADF80E30F3
:1030C0004FF00003CDE90433ADF80C20A288ADF831
:1030D0001820E288ADF81A20B4BF3146414602AA52
:1030E000ADF80800ADF80A10104605A9079349F09D
:1030F000DCFC02A920460FF029F82046CDE9008922
:103100003B46324629464AF0B7FD0E200FB0BDE8D7
:10311000F08300BF74270A00C0C20900823309008F
:103120002DE9F04F9FB019AB01935B4B0093052342
:103130001CF07EFD5949199840F256321CF05EFE93
:10314000052210A906461A9820F0F6FA05220DA9C4
:103150001B9820F0F1FA9DF84810002240201CF046
:10316000ABFE9DF83C100546002240201CF0A4FE5A
:10317000854202D04A483DF0D3FA119BB3FBF5F3E8
:103180000993099A0E9BB3FBF5F39A4201D0454887
:10319000F1E71C9B0293B37B029A012404FA03F328
:1031A0009A4201D34048E6E79DF874300A93109B99
:1031B00007932A460D9B0798089300214DF0CBFA00
:1031C0002A4607B2002108984DF0C5FA0FFA80F898
:1031D000CDE90378C246CDF81880BB460597099B18
:1031E000A3422BD80A9B43B1029BDDE90312CDE930
:1031F000008330463B464AF03FFD059BADF84C301E
:10320000069BADF84E300023CDE91533ADF852A042
:10321000ADF850B0B288ADF85C20F288ADF85E2011
:1032200013AA16A91046189349F03FFC304613A97B
:103230000EF08CFF0E201FB0BDE8F08F21460798DE
:103240002A464DF088FA214603B22A4608980B9385
:103250004DF081FA029B0FFA80F9CDE90093DDE988
:1032600003120B9B30464AF007FD0B9B059A9A42CE
:10327000D4BF059205939B45069AB8BF9B464A4525
:10328000D4BF0692CDF81890CA45CDE90339B8BF2E
:10329000CA460134A3E700BF6C280A00C0C2090077
:1032A0009F490900B449090082330900F0B591B083
:1032B0000AAB0193274B009306231CF0B9FC40F2A4
:1032C000563225490A981CF099FD827B0F9F0123F5
:1032D00093409F42044602D320483DF021FA828861
:1032E000C3880BA902A800F0F9FC029B04930025F7
:1032F000039B059304A8069549F0C6FBA388ADF887
:10330000203004AAE388079507A91046ADF82230BB
:10331000099549F0CAFB04A920460EF017FFBDF934
:103320001050BDF91430AB4202DC0E2011B0F0BDDC
:10333000BDF91260BDF91630B34202DC01352DB281
:10334000EFE732463B462946204601360EF022FF83
:1033500036B2EFE7CC270A00C0C209008233090069
:103360002DE9F04786B003AB01931F4B0093032375
:103370001CF05EFC40F2C9221C4903981CF03EFD83
:10338000827BDDF81090012393409945044603D2D7
:10339000DDF814A09A4524D3154840F20D313DF0D4
:1033A000C7F93A462946204646F0B0FC814505D18A
:1033B00053463A46294620460EF0ECFE08F1010835
:1033C000E3880FFA88F79F42EBDB0136A38835B21A
:1033D0009D4203DB0E2006B0BDE8F0874FF00008E9
:1033E000EEE70026F2E700BF0C270A00C0C2090082
:1033F000834D09002DE9F04F2DED0C8B99B00BABEF
:1034000001930D4B00930D231CF012FC0B490B98FC
:1034100040F256321CF0F2FC40F2BC5280460749A2
:103420000C981CF0EBFC98F80E20837B9A42074620
:1034300008D203483DF074F9A4260A00C0C209006E
:103440002D320900B8F804100D98490859F00FFE04
:10345000B8F806100DEE100A49080E9859F007FE4C
:10346000B9880CEE100A4908119859F000FEF98845
:103470000BEE900A4908129859F0F9FD0023109CB0
:10348000009307AA0DF11E010BEE100A0F9811F020
:10349000F3F9B8F90620B8F904300092204606AADC
:1034A0000DF11A0111F0E8F9BDF91E20BDF91A005D
:1034B000824206DD1346ADF81E00ADF81A20024622
:1034C0001846BDF91C30BDF918108B4206DD1C46AC
:1034D000ADF81C10ADF818300B462146002ABCBFD1
:1034E0000022ADF81E20B8F80440002BBCBF00231A
:1034F000ADF81C30A242B8F80620C8BFADF81E4097
:103500009342C8BFADF81C2000284FF0000380F2A2
:103510001B829942ADF81A3002DAADF8183019461C
:103520008A424FF00003B8BFADF81820149C1398DE
:10353000009305AA0DF1160111F09EF9B7F90620C6
:10354000B7F904300092204604AA0DF1120111F0DF
:1035500093F9BDF91620BDF91200824206DD13462B
:10356000ADF81600ADF8122002461846BDF9143029
:10357000BDF910108B4206DD1C46ADF81410ADF8F5
:1035800010300B462146002ABCBF0022ADF81620A1
:10359000BC88002BBCBF0023ADF81430A242FA88CF
:1035A000C8BFADF816409342C8BFADF8142000283C
:1035B0004FF0000380F2D2819942ADF8123002DA66
:1035C000ADF81030194615988A42B8BFADF81020F2
:1035D0000E2800F0CD8122F073F9F0EE40CA169863
:1035E0000E2840F0C881B7EE00AA17980E2800F008
:1035F000CD814EF013FE002383460293BDF91630B1
:10360000BDF91C20039208EE103ABDF91430BDF943
:103610001A60BDF91E90BDF918A008EE903ABDF9E8
:10362000123009EE103ABDF91030B0EE6C0A09EE16
:10363000903A35F00BFEF0EE40AAB0EE6C0A0CF0BA
:1036400011FBF8EEEB4AB8EECB4A20EE647A2AEE94
:10365000843A27EE0A7A23EE0A3AF8EECD3A77EE6C
:10366000035A6AEEE47A60EE046A02EE906A75EE3E
:10367000A35A67EE8A7A66EE8A6AF8EEE22AB8EE14
:10368000CC5A37EEE66AF4EEE25AF1EE10FA36EE74
:10369000056A039A40F17F81FDEEE52A12EE903A29
:1036A0000FFA83FC02EE909AF8EEE22AF4EEE25A68
:1036B000F1EE10FA40F37181FDEEE55A15EE903A05
:1036C0001DB205EE90AAF8EEE55AB4EEE56AF1EE09
:1036D00010FA40F16481FDEEC65A15EE903A19B227
:1036E00005EE902AF8EEE55AB4EEE56AF1EE10FA2E
:1036F00040F35781BDEEC66A16EE103A1CB2BB8885
:103700001BEE900A1B1A06EE103AB8EEC66A02EEDD
:1037100090CA60EE065A2AEE866A65EE8A5A26EE4E
:103720000A6A33EE253AF8EEE22A33EE233A76EED1
:10373000666AB4EEE23AF1EE10FA76EE856A05D5E5
:10374000FDEEC32A12EE903A0FFA83FC02EE905A75
:10375000F8EEE22AB4EEE23AF1EE10FA04DDBDEE44
:10376000C33A13EE103A1DB203EE101AB8EEC33A84
:10377000F4EEC36AF1EE10FA04D5BDEEE63A13EEAC
:10378000103A19B203EE104AB8EEC33AF4EEC36A27
:10379000F1EE10FA04DDFDEEE66A16EE903A1CB288
:1037A000FB881BEE100A1B1A06EE903AF8EEE66A4A
:1037B00002EE90CA2AEEA63A60EE266A23EE0A3A94
:1037C00066EE8A6A75EEC35AF8EEE22A75EEA35ADF
:1037D00036EE266AF4EEE25AF1EE10FA36EE056A9B
:1037E00005D5FDEEE52A12EE903A0FFA83FC02EEC3
:1037F000905AF8EEE22AF4EEE25AF1EE10FA04DD05
:10380000FDEEE55A15EE903A1DB205EE901AF8EE6F
:10381000E55AB4EEE56AF1EE10FA04D5FDEEC65AAB
:1038200015EE903A19B205EE904AF8EEE55AB4EE6C
:10383000E56AF1EE10FA04DDBDEEC66A16EE103A46
:103840001CB277EEA67A37EE437A06EE90CA37EED0
:10385000237AF8EEE66A77EE857AB4EEE67AF1EE50
:1038600010FA05D5FDEEC76A16EE903A0FFA83FC02
:1038700006EE905AF8EEE66AB4EEE67AF1EE10FA49
:1038800004DDBDEEC77A17EE103A1DB207EE101A2E
:10389000B8EEC77AF4EEC77AF1EE10FA04D5BDEEB1
:1038A000E77A17EE103A19B207EE104AB8EEC77A67
:1038B000F4EEC77AF1EE10FA04DDFDEEE77A17EECA
:1038C000903A1CB2CAEE8ABA731EE1451BB2B8BF69
:1038D000E146AE42D8BF1D468A42B8BF0A460AF149
:1038E000FF331BB2A245D8BF1C466B1CADF8243079
:1038F000631C80EE0ABAADF8263008A900234046C2
:103900001646ADF82090ADF822200A9365EE2B7A8A
:1039100025EE0B5AE3EE8B7AABEEE35A74EEE7AA90
:1039200007EE902A34EE45AAF8EEE77AEBEEA7AA66
:10393000ABEE27AA0EF00AFCB44234DA0E2019B01E
:10394000BDEC0C8BBDE8F08F0029BCBFADF8183082
:1039500019468442B8BFADF81A40E1E50029BCBF62
:10396000ADF8103019468442B8BFADF812402AE6CF
:10397000DFED37CA33E621F0A3FFB5EEC00AF1EE62
:1039800010FAB0EE40AA7FF530AE2CE60123029388
:103990004FF0000B32E6B44684E64D4691E65146C0
:1039A0009EE61446ABE607EE909AF8EEE77AB0EEA4
:1039B0006ACAF0EE4ACAABEE27CACA46EBEEE7CABD
:1039C000554506DA01367AEEABAA3AEE0BAA36B2C4
:1039D000B2E7F8EEC87AF4EECC7AF1EE10FA2DD810
:1039E000F8EEC97AB4EEE7CAF1EE10FA26D5F8EE91
:1039F000E87AF4EEEC7AF1EE10FA1FD8F8EEE97AF4
:103A0000F4EEE7CAF1EE10FA18D5FDEEEC7A38467E
:103A1000CDED037AFDEECC7ABDF90C20CDED037A25
:103A2000BDF90C1046F072F9029A03460AB98345B3
:103A300004D03246514640460EF0ACFB0AF1010A72
:103A40003CEE0BCA7CEEEBCA0FFA8AFAB8E700BF6D
:103A5000000000002DE9F04F9DB002AF07F14C03CC
:103A60000193974B009307231CF0E2F89549F86CFB
:103A700040F2C9221CF0C2F9BE6D731E012B8246B2
:103A800005D9042E03D0904831463CF051FED7F8BA
:103A90005480B8F1020F05DCB8F1000F14DC8B483C
:103AA0004146F2E7A8F104031C2BF8D8884A01210B
:103AB00099400A4042B9142BF1D1012E04D0854817
:103AC000182231463CF034FE3B6DBB6297F85C3007
:103AD000FB6297F860303B6297F86430FB619AF8BC
:103AE0000E30B86A012101FA03F3013B7B611FF03C
:103AF00075FEBAF8043078600024A7F8443007F166
:103B00004001BAF80630A7F8463050463C64BC6421
:103B10000EF01CFBBAF804307C6308FB03F303EBE4
:103B2000C603F200013BB3FBF2F373433B63033381
:103B300023F003037B623B6B013323F00103BB6182
:103B40007B6A073323F00703BB60BAF806907B6BF0
:103B5000994504DC0E206C37BD46BDE8F08FBB688C
:103B6000C7F810D0ADEB030DFB6902AD9BB17B6BC9
:103B700009F1FF39A9EB03090023FB637B683A6B6A
:103B80005C68B86A294607F13C03A047F96B29B184
:103B900008463CF07DFDD7F83490EDE73B6B83425F
:103BA00002D04D4859F066F83B6A93B1022E0BD013
:103BB000042E0ED17A6A2B46A918994209D01A68A8
:103BC00012BA43F8042BF8E7BA692B465119994207
:103BD00010D108F1FF33AB460024FB600FFA89F9DE
:103BE000BAF804309C420ADB7B6BD7F810D0013363
:103BF0007B63AAE71A8852BA23F8022BE7E7B8F1E9
:103C0000080F08DCFA68072A0ED8DFE802F00F2751
:103C10000D360D0D0D45B8F1180F42D0B8F1200F3B
:103C20004AD0B8F1100F39D0002309E0FA6AE31046
:103C30008AB1E24302F00702EB5C134103F0010397
:103C40007A6921B2134050464A460EF0A3FA013475
:103C50000BF1030BC4E704F00702EDE7FA6AA310C7
:103C600042B1E24302F00302EB5C5200134103F065
:103C70000303E5E704F00302F6E7FA6A631042B1D2
:103C8000E24302F00102EB5C9200134103F00F03E8
:103C9000D6E704F00102F6E72B5DD1E735F81430E2
:103CA000CEE79BF801309BF800201B0243EA024359
:103CB0009BF802201343C3E755F82430C0E700BF48
:103CC000FC270A00C0C209006937090089370900CA
:103CD000111000107B3709007456090073B50446B3
:103CE0000D461E466846084B44F095FD291D0DF112
:103CF0000200064B324644F08EFD6B4603CB20603B
:103D00002046616002B070BD04260A00FC250A004E
:103D10002DE9F04F0D4687B00021924629F0BCFAFC
:103D200004460021284629F0B7FA2379662B02D0F1
:103D30000379662B02D1C8483CF0F2FC00230390C3
:103D400008208DF817304DF092F8074608204DF006
:103D50008EF8064608204DF08AF80399CDE90060F8
:103D600005463B460DF11702204654F066F80399CC
:103D700050B9384613F0E6FD304613F0E3FD28460F
:103D800013F0E0FDB548D7E70AF1FF3A9DF81700B8
:103D9000D4F81C90D1F81C802279BAF1030F05D811
:103DA000DFE81AF0E901BD0398053B08AA46B346CF
:103DB0002379D4F81C90D1F81C80422B40F0C180AC
:103DC0000A79422A3DD1394654F0E4F9C2690446E1
:103DD0000020134698F800C099F8001001EA0C0181
:103DE00003F8011BDAF80410D4F810C0DBF804E083
:103DF00003918844991A8C45F144EBD8DBF8001004
:103E0000DAF800200CFB1E11894403990CFB1122E7
:103E10009044E2680130904211D3384613F092FD8D
:103E2000304613F08FFD284613F08CFD204607B076
:103E3000BDE8F08F5A461C46D3469246B8E71A466C
:103E4000C7E7622A28D13946682254F0A3F9C1692C
:103E500004460023002298F900C099F8000000EA07
:103E60000C0021F8020B2069DBF804E0DAF804C04A
:103E700001328242F144E044EDD3DBF8002000FB44
:103E80001E229144DAF8002000FB1C229044E268D4
:103E900001339342DED3C0E7482A27D1394654F094
:103EA00079F9C169044600230022B8F800C099F8E6
:103EB000000000EA0C0021F8020B2069DBF804E0A6
:103EC000DAF804C001328242F144E044EDD3DBF879
:103ED000002000FB1E229144DAF8002000FB1C2287
:103EE0009044E26801339342DED396E7682A41F0BA
:103EF0003782394654F04EF9C16904460023002246
:103F0000B8F800C099F8000000EA0C0021F8020B94
:103F10002069DBF804E0DAF804C001328242F1449F
:103F2000E044EDD3DBF8002000FB1E229144DAF8D8
:103F3000002000FB1C229044E26801339342DED350
:103F40006BE7622B40F08C800A79622A2CD13946CB
:103F500054F020F9C26904460020134698F800C0C6
:103F600099F8001001EA0C0103F8011BDAF80410BB
:103F7000D4F810C0DBF804E003918844991A614535
:103F8000F144EBD3DBF80010DAF800200CFB1E1133
:103F9000894403990CFB11229044E268013090425D
:103FA000BFF43BAF1A46D8E7482A27D1394654F028
:103FB000F1F8C169044600230022B8F800C099F95D
:103FC000000000EA0C0021F8020B2069DBF804E095
:103FD000DAF804C001328242F144E044EDD3DBF868
:103FE000002000FB1E229144DAF8002000FB1C2276
:103FF0009044E26801339342DED30EE7682A0B4611
:1040000021467FF417AF394654F0C4F8C16904461D
:1040100000230022B8F800C099F9000000EA0C0063
:1040200021F8020B2069DBF804E0DAF804C0013261
:104030008242F144E044EDD3DBF8002000FB1E2275
:104040009144DAF8002000FB1C229044E26801331E
:104050009342DED3E1E600BFD93409001D340900E4
:10406000482B57D10A79482A27D1394654F092F87B
:10407000C169044600230022B8F800C0B9F8000066
:1040800000EA0C0021F8020B2069DBF804E0DAF802
:1040900004C001328242F144E044EDD3DBF8002059
:1040A00000FB1E229144DAF8002000FB1C22904401
:1040B000E26801339342DED3AFE6682A0B4621461D
:1040C0007FF4B8AE394654F065F8C1690446002360
:1040D0000022B8F800C0B9F8000000EA0C0021F88E
:1040E000020B2069DBF804E0DAF804C001328242F6
:1040F000F144E044EDD3DBF8002000FB1E229144A4
:10410000DAF8002000FB1C229044E268013393425D
:10411000DED382E6682B41F023810A79682A0B46B8
:1041200021467FF487AE394654F034F8C16904461D
:1041300000230022B8F800C0B9F8000000EA0C0023
:1041400021F8020B2069DBF804E0DAF804C0013240
:104150008242F144E044EDD3DBF8002000FB1E2254
:104160009144DAF8002000FB1C229044E2680133FD
:104170009342DED351E6AA46B3462379D4F81C9085
:10418000D1F81C80422B40F0B5800A79422A31D107
:10419000394653F0FFFFC26904460020134698F8E1
:1041A00000C099F8001041EA0C0103F8011BDAF88D
:1041B0000410D4F810C0DBF804E003918844991A85
:1041C0006145F144EBD3DBF80010DAF800200CFB7A
:1041D0001E11894403990CFB11229044E2680130BE
:1041E0009042BFF41AAE1A46D8E75A461C46D34648
:1041F0009246C2E7622A28D13946682253F0CAFFA4
:10420000C16904460023002298F900C099F8000013
:1042100040EA0C0021F8020B2069DBF804E0DAF830
:1042200004C001328242F144E044EDD3DBF80020C7
:1042300000FB1E229144DAF8002000FB1C2290446F
:10424000E26801339342DED3E7E5482A27D13946B5
:1042500053F0A0FFC169044600230022B8F800C053
:1042600099F8000040EA0C0021F8020B2069DBF805
:1042700004E0DAF804C001328242F144E044EDD3B4
:10428000DBF8002000FB1E229144DAF8002000FB3E
:104290001C229044E26801339342DED3BDE5682AD4
:1042A00041F05E80394653F075FFC1690446002332
:1042B0000022B8F800C099F8000040EA0C0021F88C
:1042C000020B2069DBF804E0DAF804C00132824214
:1042D000F144E044EDD3DBF8002000FB1E229144C2
:1042E000DAF8002000FB1C229044E268013393427C
:1042F000DED392E5622B40F087800A79622A2CD1C6
:10430000394653F047FFC26904460020134698F827
:1043100000C099F8001041EA0C0103F8011BDAF81B
:104320000410D4F810C0DBF804E003918844991A13
:104330006145F144EBD3DBF80010DAF800200CFB08
:104340001E11894403990CFB11229044E26801304C
:104350009042BFF462AD1A46D8E7482A27D13946C1
:1043600053F018FFC169044600230022B8F800C0CA
:1043700099F9000040EA0C0021F8020B2069DBF8F3
:1043800004E0DAF804C001328242F144E044EDD3A3
:10439000DBF8002000FB1E229144DAF8002000FB2D
:1043A0001C229044E26801339342DED335E5682A4B
:1043B0000B4621467FF419AF394653F0EBFEC16935
:1043C000044600230022B8F800C099F9000040EA32
:1043D0000C0021F8020B2069DBF804E0DAF804C0D5
:1043E00001328242F144E044EDD3DBF8002000FBCF
:1043F0001E229144DAF8002000FB1C229044E2685F
:1044000001339342DED308E5482B57D10A79482A75
:1044100027D1394653F0BEFEC1690446002300226D
:10442000B8F800C0B9F8000040EA0C0021F8020B0F
:104430002069DBF804E0DAF804C001328242F1447A
:10444000E044EDD3DBF8002000FB1E229144DAF8B3
:10445000002000FB1C229044E26801339342DED32B
:10446000DBE4682A0B4621467FF4BFAE394653F0A1
:1044700091FEC169044600230022B8F800C0B9F8D3
:10448000000040EA0C0021F8020B2069DBF804E090
:10449000DAF804C001328242F144E044EDD3DBF8A3
:1044A000002000FB1E229144DAF8002000FB1C22B1
:1044B0009044E26801339342DED3AEE4682B40F0CF
:1044C0004F870A79682A0B4621467FF48EAE39461B
:1044D00053F060FEC169044600230022B8F800C012
:1044E000B9F8000040EA0C0021F8020B2069DBF863
:1044F00004E0DAF804C001328242F144E044EDD332
:10450000DBF8002000FB1E229144DAF8002000FBBB
:104510001C229044E26801339342DED37DE4AA4634
:10452000B3462379D4F81C90D1F81C80422B40F07C
:10453000B7800A79422A31D1394653F02BFEC2693D
:1045400004460020134698F800C099F8001081EA4C
:104550000C0103F8011BDAF80410D4F810C0DBF8E2
:1045600004E003918844991A6145F144EBD3DBF8E8
:104570000010DAF800200CFB1E11894403990CFB93
:1045800011229044E26801309042BFF446AC1A46D2
:10459000D8E75A461C46D3469246C2E7622A28D13B
:1045A0003946682253F0F6FDC16904460023002213
:1045B00098F900C099F8000080EA0C0021F8020B7D
:1045C0002069DBF804E0DAF804C001328242F144E9
:1045D000E044EDD3DBF8002000FB1E229144DAF822
:1045E000002000FB1C229044E26801339342DED39A
:1045F00013E4482A28D1394653F0CCFDC16904465A
:1046000000230022B8F800C099F8000080EA0C00EE
:1046100021F8020B2069DBF804E0DAF804C001326B
:104620008242F144E044EDD3DBF8002000FB1E227F
:104630009144DAF8002000FB1C229044E268013328
:104640009342DED3FFF7E9BB682A40F089863946FA
:1046500053F0A0FDC169044600230022B8F800C051
:1046600099F8000080EA0C0021F8020B2069DBF8C1
:1046700004E0DAF804C001328242F144E044EDD3B0
:10468000DBF8002000FB1E229144DAF8002000FB3A
:104690001C229044E26801339342DED3FFF7BDBB96
:1046A000622B40F089800A79622A2CD1394653F076
:1046B00071FDC26904460020134698F800C099F8BD
:1046C000001081EA0C0103F8011BDAF80410D4F899
:1046D00010C0DBF804E003918844991A6145F14465
:1046E000EBD3DBF80010DAF800200CFB1E11894434
:1046F00003990CFB11229044E26801309042BFF410
:104700008CAB1A46D8E7482A28D1394653F042FDE7
:10471000C169044600230022B8F800C099F90000DE
:1047200080EA0C0021F8020B2069DBF804E0DAF8DB
:1047300004C001328242F144E044EDD3DBF80020B2
:1047400000FB1E229144DAF8002000FB1C2290445A
:10475000E26801339342DED3FFF75FBB682A0B4662
:1047600021467FF416AF394653F014FDC169044663
:1047700000230022B8F800C099F9000080EA0C007C
:1047800021F8020B2069DBF804E0DAF804C00132FA
:104790008242F144E044EDD3DBF8002000FB1E220E
:1047A0009144DAF8002000FB1C229044E2680133B7
:1047B0009342DED3FFF731BB482B59D10A79482AFF
:1047C00028D1394653F0E6FCC16904460023002293
:1047D000B8F800C0B9F8000080EA0C0021F8020B1C
:1047E0002069DBF804E0DAF804C001328242F144C7
:1047F000E044EDD3DBF8002000FB1E229144DAF800
:10480000002000FB1C229044E26801339342DED377
:10481000FFF703BB682A0B4621467FF4BAAE394640
:1048200053F0B8FCC169044600230022B8F800C068
:10483000B9F8000080EA0C0021F8020B2069DBF8CF
:1048400004E0DAF804C001328242F144E044EDD3DE
:10485000DBF8002000FB1E229144DAF8002000FB68
:104860001C229044E26801339342DED3FFF7D5BAAD
:10487000682B40F075850A79682A0B4621467FF43B
:1048800088AE394653F086FCC169044600230022F5
:10489000B8F800C0B9F8000080EA0C0021F8020B5B
:1048A0002069DBF804E0DAF804C001328242F14406
:1048B000E044EDD3DBF8002000FB1E229144DAF83F
:1048C000002000FB1C229044E26801339342DED3B7
:1048D000FFF7A3BA422A40F0A8800B79422B28D1D7
:1048E000394653F057FCC26904460020134698F835
:1048F00000C099F8001001FA0CF103F8011BD4F87C
:1049000010C0D6F804A0D5F804E0991A6145D14446
:10491000F044ECD32A6831680CFB1E229044E26814
:1049200001300CFB1A1190428944BFF476AA1A4652
:10493000DCE7622B27D16822394653F02BFC044672
:10494000C0690023002298F900C099F8001001FA0C
:104950000CF120F8021B2169D6F804E0D5F804C058
:1049600001328A42F144E044EDD3326801FB1E2259
:1049700091442A6801FB1C229044E268013393426F
:10498000E0D3FFF74ABA482B27D11A46394653F0ED
:1049900001FC0446C06900230022B8F800C099F861
:1049A000001001FA0CF120F8021B2169D6F804E08E
:1049B000D5F804C001328A42F144E044EDD33268B4
:1049C00001FB1E2291442A6801FB1C229044E268EC
:1049D00001339342E0D3FFF720BA6822394653F0FF
:1049E000D9FB0446C06900230022B8F900C099F839
:1049F000001001FA0CF120F8021B2169D6F804E03E
:104A0000D5F804C001328A42F144E044EDD3326863
:104A100001FB1E2291442A6801FB1C229044E2689B
:104A200001339342E0D3FFF7F8B9622A40F0A8803F
:104A30000B79422B27D16822394653F0ABFB044651
:104A4000C0690023002298F800C099F9001001FA0B
:104A50000CF120F8021B2169D6F804E0D5F804C057
:104A600001328A42F144E044EDD3326801FB1E2258
:104A700091442A6801FB1C229044E268013393426E
:104A8000E0D3FFF7CAB9622B28D1394653F082FB35
:104A9000C26904460020134698F900C099F9001035
:104AA00001FA0CF103F8011BD4F810C0D6F804A0E9
:104AB000D5F804E0991A6145D144F044ECD32A6852
:104AC00031680CFB1E229044E26801300CFB1A1185
:104AD00090428944BFF4A1A91A46DCE7482B27D1AC
:104AE0001A46394653F056FB0446C069002300229B
:104AF000B8F800C099F9001001FA0CF120F8021B77
:104B00002169D6F804E0D5F804C001328A42F144A4
:104B1000E044EDD3326801FB1E2291442A6801FB78
:104B20001C229044E26801339342E0D3FFF775B949
:104B30006822394653F02EFB0446C0690023002248
:104B4000B8F900C099F9001001FA0CF120F8021B25
:104B50002169D6F804E0D5F804C001328A42F14454
:104B6000E044EDD3326801FB1E2291442A6801FB28
:104B70001C229044E26801339342E0D3FFF74DB921
:104B8000482A40F0A7800B79422B26D1394653F0B2
:104B900001FB0446C0690023002298F800C0B9F860
:104BA000001001FA0CF120F8021B2169D6F804E08C
:104BB000D5F804C001328A42F144E044EDD33268B2
:104BC00001FB1E2291442A6801FB1C229044E268EA
:104BD00001339342E0D3FFF720B9622B29D11A4663
:104BE000394653F0D7FAC26904460020134698F9B3
:104BF00000C099F9001001FA0CF103F8011BD4F878
:104C000010C0D6F804A0D5F804E0991A6145D14443
:104C1000F044ECD32A6831680CFB1E229044E26811
:104C200001300CFB1A1190428944BFF4F6A81A46D1
:104C3000DCE7482B26D1394653F0ACFA0446C0696C
:104C400000230022B8F800C0B9F8001001FA0CF1F6
:104C500020F8021B2169D6F804E0D5F804C001321F
:104C60008A42F144E044EDD3326801FB1E229144B4
:104C70002A6801FB1C229044E26801339342E0D38E
:104C8000FFF7CBB86822394653F084FA0446C0696E
:104C900000230022B8F900C0B9F8001001FA0CF1A5
:104CA00020F8021B2169D6F804E0D5F804C00132CF
:104CB0008A42F144E044EDD3326801FB1E22914464
:104CC0002A6801FB1C229044E26801339342E0D33E
:104CD000FFF7A3B8682A40F043830B79422B39468B
:104CE00025D153F057FA0446C0690023002298F8F2
:104CF00000C0B9F9001001FA0CF120F8021B21697B
:104D0000D6F804E0D5F804C001328A42F144E04408
:104D1000EDD3326801FB1E2291442A6801FB1C225C
:104D20009044E26801339342E0D3FFF776B8622BF8
:104D300025D153F02FFA0446C0690023002298F9C8
:104D400000C0B9F9001001FA0CF120F8021B21692A
:104D5000D6F804E0D5F804C001328A42F144E044B8
:104D6000EDD3326801FB1E2291442A6801FB1C220C
:104D70009044E26801339342E0D3FFF74EB8482BEA
:104D800025D153F007FA0446C06900230022B8F980
:104D900000C0B9F8001001FA0CF120F8021B2169DB
:104DA000D6F804E0D5F804C001328A42F144E04468
:104DB000EDD3326801FB1E2291442A6801FB1C22BC
:104DC0009044E26801339342E0D3FFF726B853F0F2
:104DD000E1F90446C06900230022B8F900C0B9F91E
:104DE000001001FA0CF120F8021B2169D6F804E04A
:104DF000D5F804C001328A42F144E044EDD3326870
:104E000001FB1E2291442A6801FB1C229044E268A7
:104E100001339342E0D3FFF700B8422A40F0A88064
:104E20000B79422B28D1394653F0B4F9C2690446B4
:104E30000020134698F800C099F8001041FA0CF1D0
:104E400003F8011BD4F810C0D6F804A0D5F804E08C
:104E5000991A8C45D144F044ECD82A6831680CFB8F
:104E60001E229044E26801300CFB1A1190428944E2
:104E7000BEF4D3AF1A46DCE7622B27D1682239464D
:104E800053F088F90446C0690023002298F900C055
:104E900099F8001041FA0CF120F8021B2169D6F8AC
:104EA00004E0D5F804C001328A42F144E044EDD375
:104EB000326801FB1E2291442A6801FB1C229044A7
:104EC000E26801339342E0D3FEF7A7BF482B27D116
:104ED0001A46394653F05EF90446C06900230022A1
:104EE000B8F800C099F8001041FA0CF120F8021B44
:104EF0002169D6F804E0D5F804C001328A42F144B1
:104F0000E044EDD3326801FB1E2291442A6801FB84
:104F10001C229044E26801339342E0D3FEF77DBF48
:104F20006822394653F036F90446C069002300224E
:104F3000B8F900C099F8001041FA0CF120F8021BF2
:104F40002169D6F804E0D5F804C001328A42F14460
:104F5000E044EDD3326801FB1E2291442A6801FB34
:104F60001C229044E26801339342E0D3FEF755BF20
:104F7000622A40F0A8800B79422B27D1682239465B
:104F800053F008F90446C0690023002298F800C0D5
:104F900099F9001041FA0CF120F8021B2169D6F8AA
:104FA00004E0D5F804C001328A42F144E044EDD374
:104FB000326801FB1E2291442A6801FB1C229044A6
:104FC000E26801339342E0D3FEF727BF622B28D17A
:104FD000394653F0DFF8C26904460020134698F9B9
:104FE00000C099F9001041FA0CF103F8011BD4F844
:104FF00010C0D6F804A0D5F804E0991A8C45D14425
:10500000F044ECD82A6831680CFB1E229044E26818
:1050100001300CFB1A1190428944BEF4FEAE1A46D0
:10502000DCE7482B27D11A46394653F0B3F804463B
:10503000C06900230022B8F800C099F9001041FAB5
:105040000CF120F8021B2169D6F804E0D5F804C061
:1050500001328A42F144E044EDD3326801FB1E2262
:1050600091442A6801FB1C229044E2680133934278
:10507000E0D3FEF7D2BE6822394653F08BF80446DF
:10508000C06900230022B8F900C099F9001041FA64
:105090000CF120F8021B2169D6F804E0D5F804C011
:1050A00001328A42F144E044EDD3326801FB1E2212
:1050B00091442A6801FB1C229044E2680133934228
:1050C000E0D3FEF7AABE482A40F0A7800B79422B16
:1050D00026D1394653F05EF80446C0690023002209
:1050E00098F800C0B9F8001041FA0CF120F8021B42
:1050F0002169D6F804E0D5F804C001328A42F144AF
:10510000E044EDD3326801FB1E2291442A6801FB82
:105110001C229044E26801339342E0D3FEF77DBE47
:10512000622B29D11A46394653F034F8C269044635
:105130000020134698F900C099F9001041FA0CF1CB
:1051400003F8011BD4F810C0D6F804A0D5F804E089
:10515000991A8C45D144F044ECD82A6831680CFB8C
:105160001E229044E26801300CFB1A1190428944DF
:10517000BEF453AE1A46DCE7482B26D1394653F02D
:1051800009F80446C06900230022B8F800C0B9F845
:10519000001041FA0CF120F8021B2169D6F804E056
:1051A000D5F804C001328A42F144E044EDD33268BC
:1051B00001FB1E2291442A6801FB1C229044E268F4
:1051C00001339342E0D3FEF728BE6822394652F0FD
:1051D000E1FF0446C06900230022B8F900C0B9F815
:1051E000001041FA0CF120F8021B2169D6F804E006
:1051F000D5F804C001328A42F144E044EDD332686C
:1052000001FB1E2291442A6801FB1C229044E268A3
:1052100001339342E0D3FEF700BE682A40F0A0803D
:105220000B79422B394625D152F0B4FF0446C069B0
:105230000023002298F800C0B9F9001041FA0CF1DF
:1052400020F8021B2169D6F804E0D5F804C0013229
:105250008A42F144E044EDD3326801FB1E229144BE
:105260002A6801FB1C229044E26801339342E0D398
:10527000FEF7D3BD622B25D152F08CFF0446C069E6
:105280000023002298F900C0B9F9001041FA0CF18E
:1052900020F8021B2169D6F804E0D5F804C00132D9
:1052A0008A42F144E044EDD3326801FB1E2291446E
:1052B0002A6801FB1C229044E26801339342E0D348
:1052C000FEF7ABBD482B25D152F064FF0446C06900
:1052D00000230022B8F900C0B9F8001041FA0CF11F
:1052E00020F8021B2169D6F804E0D5F804C0013289
:1052F0008A42F144E044EDD3326801FB1E2291441E
:105300002A6801FB1C229044E26801339342E0D3F7
:10531000FEF783BD52F03EFF0446C0690023002221
:10532000B8F900C0B9F9001041FA0CF120F8021BDD
:105330002169D6F804E0D5F804C001328A42F1446C
:10534000E044EDD3326801FB1E2291442A6801FB40
:105350001C229044E26801339342E0D3FEF75DBD26
:105360000024FEF75ABD00BF38B50C4BD3F8B0305F
:1053700004460D4643B90C204BF079FD2A462146E0
:10538000BDE8384000F00CB89A68A24202D15A68D1
:10539000AA4201D01B68EDE738BD00BF745D012053
:1053A00070B5094CD4F8B0502B462BB9C0E9005267
:1053B0008160C4F8B00070BD9E688E4202D15E6804
:1053C0009642F8D01B68F0E7745D012030B5094AB9
:1053D00052F8B03F4BB19C6884421C6806D15D68AE
:1053E0008D4203D1146000221A6030BD1A46234654
:1053F000F0E700BF745D0120044B1B7823B1044823
:1054000043680BB144F034BB18467047D5670120A0
:10541000F04F012008B50348012104F075FC0E206F
:1054200008BD00BF8851012070B52DED028B8EB0F4
:1054300006AB0193574B00930431022301381AF055
:10544000F7FB4FF42272544906981AF0D7FC40F249
:10545000096104469FED510A07981AF0BDFC2046E9
:1054600004A9B0EE408A41F0D9FF0E2200210AA81B
:105470004BF0F6FDDFED4A7A9FED4A7A4A4B4B4AF4
:105480000A9328EE278AA023C8EE077AADF82C30BD
:1054900010685168B6EE007A77EE877AFCEEE77A0C
:1054A00017EE903AADF82E3008AB03C3404803A97D
:1054B000FFF75AFF00238DF80E3008AA01230AA92E
:1054C00004A854F0F1FC044630B1394803A9FFF7B1
:1054D0007DFF204643F0DEFF9DF80E3063B1344877
:1054E00003A9FFF773FFBDF80C604FF6FF739E42F0
:1054F00005D1304823F0D4FCFBF7B4F9ECE70020E9
:105500002AF0D2F90446B8B16378012B36D123785A
:10551000DB0733D506220DF1110104F151004BF0E8
:105520004AFD58BB04F1240204F13601304654F020
:10553000C9FCB0FA80F46409002502A93046ADF830
:10554000085054F0C3FC4FF40071304654F0D4FCC2
:1055500043F0A0FF29462A46304654F0A9FC43F008
:1055600099FF154B882101FB05F2D0189A5AB242D7
:1055700006D00135052DF6D11048BBE72046BFE720
:105580000123837080F85A4000F0B4FD0EB0BDECEA
:10559000028B70BD841F0A00F8B0090000000000F3
:1055A0000024744900401C460001A000CCDC080027
:1055B000A7BF070036480900A0090120414809009B
:1055C00037B5012104F0A0FB684654F05BFC43F0C2
:1055D00061FF09490C204DF0F4F9062104460DF154
:1055E00001009DF8005021F06DF9C5F34605A0605B
:1055F0002046257103B030BDF8B009002DE9F04117
:105600000746806986B0F0B9104D044606464FF64D
:10561000FF782B8843450CD0E86D0E2803D128462F
:1056200000F068FDE86506AB03EB8403013443F842
:10563000140C0136052E05F18805EAD101A9204692
:1056400021F078FBB86106B0BDE8F081A009012027
:1056500008B501483BF008F89C4A090010B50C4613
:1056600086B0A068012203A91EF066F888B19DF8F3
:105670000430227962F347038DF80430039B1A68E3
:10568000CDF805209B88ADF8093001A854F0FCFB4B
:1056900010B1034823F004FC0E2006B010BD00BF7B
:1056A000974909002DE9F04F2DED028B95B00CAB19
:1056B00051F8044B01935F4B0093013808231AF013
:1056C000B7FA0C98052209A91EF036F80D980023A8
:1056D0000E28CDE90633089303D0052206A91EF053
:1056E0002BF8119808B95448119040F222411AF051
:1056F0009BFBDFED527AB4EEE70AF1EE10FAB0EE62
:10570000408A06D4DFED4E7AB4EEE70AF1EE10FAE5
:1057100004DD4C4A4C494D483BF00AF8DDF840A006
:10572000BAF1000F04DA40F2096100201AF012FB0E
:105730000A9B9DF838601F2B05D926B1079B13B132
:10574000434823F0ADFB13980E280DD00EB9414805
:10575000F7E7414940F265321AF050FB074694F8EA
:1057600044301BB13D48ECE70027F8E7E3689DF8BB
:105770003C80DDF8489013B1204604F023FC0A9DDC
:105780003146284603F082FBDDF81CB0314658460E
:1057900003F07CFB1F2D04D9BBF1000F02D0304871
:1057A000CFE715B10FB12F48CBE7B8F1000F09D102
:1057B0002D4B2E4A03FB0AF3934205D92C48B42102
:1057C00023F06EFB4FF0B40A616819B9FF2011F0A5
:1057D000EFFC6060A16819B9FF2011F0E9FCA0603E
:1057E000DDE9091260684BF0FAFBDDE90612A068FA
:1057F0004BF0F5FBCDE90497BDF81C300393A3688B
:105800000293BDF82830019363680093B0EE480A14
:105810005346424631462046F4F7DEFE43F03AFE58
:1058200001230E2084F8443015B0BDEC028BBDE896
:10583000F08F00BF841E0A00CECC4CBE0AD7A33C1A
:105840000AD723415E1D0900641D0900A437090021
:10585000664A0900AA440900F8B00900FA4B090099
:105860007B4809005C49090040420F000FBCBA0A9E
:10587000E64109002DE9F04F2DED068B93B00AAB00
:1058800051F8044B0193834B0093013808231AF01D
:10589000CFF90D980E2828D09FED7F0A40F20961BC
:1058A0001AF09AFAF0EE408A0E9808B97B480E90EA
:1058B0000F9B0BB9794B0F9340F222411AF0B4FAC7
:1058C000DFED777AB4EEE70AF1EE10FAB0EE408A37
:1058D00006D4DFED747AB4EEE70AF1EE10FA07DDD4
:1058E000714A724972483AF023FFDFED6B8ADBE7B9
:1058F000F5EE408AF1EE10FA07D0F4EEC08AF1EE30
:1059000010FA02D56B483AF00BFF0F9840F26B612A
:105910001AF08AFAB4EEC08AF1EE10FAB0EE409AAC
:1059200001D56548EFE70A980023049358B1052292
:1059300003A91DF001FF049B2BB1039812F0BEF9DF
:1059400008B95E48DFE70B9F002F04DC40F2E62138
:1059500001201AF0FFF923699DF83050DDF84090DE
:105960009DF84480DDE903BA3BB193F8293013B9BF
:10597000534823F095FA00232361E36843B162683A
:10598000934202D1112003F055FB204604F01AFB8C
:105990004C499FED4DAA2C204DF013F83946064690
:1059A000083054F0E0F8002DC6E907BAC6F8249094
:1059B00026610CBF1F26FF2606F108004BF075FA82
:1059C0002369586000F108030360868007460120C0
:1059D00042F068F843F05EFD21693C48FFF7C4FCE3
:1059E00068EE8A6A9FED3A7AC6EE877AF6EE009AFA
:1059F00077EEA97AFCEEE77A17EE906AB6F5803F6B
:105A000001D334487FE736B9F5EEC08AF1EE10FADB
:105A100001DD314877E70E22002106A84BF020FB7C
:105A200028EE0A8A9FED2D7AADF81E60C8EE077A3F
:105A300045F4807545EA880525F0FA05394606A83B
:105A4000ADF8185029EE0A9A77EEA97AFCEEE77ABB
:105A500017EE903AC9EE077AADF81A3077EEA97AC8
:105A6000FCEEE77A17EE903AADF81C3054F036FAB7
:105A7000054640B115482169FFF7A8FC00232361C2
:105A8000284643F007FD206913B0BDEC068BBDE846
:105A9000F08F00BFC41E0A0000000000CECC4CBE38
:105AA0000AD7233B66D62342691D0900731D0900EE
:105AB000A4370900F8340900D12F09001744090060
:105AC0003D43090020B0090000247449C57A06004E
:105AD00000401C46853109000835090000401C447F
:105AE000022838B50D46144610D193070CD1126820
:105AF000084B9A4208D1A168A8684CF02BFB18B15A
:105B00002A7923799A4203D01E2038BD0020FCE771
:105B10003E20FAE7F8B0090030B589B008461146D2
:105B20001A4603AB0193134B009302234BF0E4FBA3
:105B300005A9039805221DF0FFFD06984FF4227277
:105B400006211AF019F940F28B2303220498002150
:105B50004BF005FC084905460C204CF032FF0621AD
:105B60000446059820F0AEFEA0602046257109B0DD
:105B700030BD00BF741F0A00F8B0090010B50B4615
:105B800088B0044605A9986805221DF0D5FD059941
:105B900008780B794A7903904878029088780190C8
:105BA000C9780091204602494DF023F908B010BD94
:105BB0007A1D0900062837B50D4618D18C680D4BA3
:105BC0002340062B11D1200953F029FB30B901A93C
:105BD000204621F0D7FF019953F0F8FA2B7958406D
:105BE000400040F0010003B030BD6068EEE70020E7
:105BF000F9E700BF0F0080FF2DE9F04F97B00DAB24
:105C00000193344B00930431092301381AF010F842
:105C100031490D9840F28C521AF0F0F82F49089053
:105C200040F24D620E981AF0E9F89DF83C603F2E64
:105C3000834603D940F2FA4019F0ECFF9DF840701A
:105C4000384643F003FF9DF84480404643F0FEFE93
:105C5000129C002C04DA40F26D4100201AF07AF810
:105C600014989DF84C500E2804D15DB354B32046CF
:105C70004CF0D2FE0DF12809052249461DF05CFDCD
:105C80000B9840F216422146F5B11AF075F81598B6
:105C90000E281CD021F09EFF8246114928204CF08E
:105CA00090FECDE9059ACDE90345CDE90178089943
:105CB00000965B460022099004F0ECF9099817B0B1
:105CC000BDE8F08F0748D5E71AF062F8DFE74FF03C
:105CD000000AE2E72C1F0A0000B00900D8AF090053
:105CE000ACB00900E85E090010B54368044653B142
:105CF00001460648FFF76AFB0023C4E90333C4E901
:105D00000633636063610E2010BD00BF439307003C
:105D100070B52DED028B86B0084611461A4603ABCE
:105D200001931F4B009303234BF0E6FA1D490398A0
:105D30004FF43F721AF062F840F209610646B7EE7E
:105D4000000A04981AF048F8059D002DB0EE408A2C
:105D500004DC40F2E621012019F0FCFF1249242066
:105D60004CF02FFE044628464BF09FF8DFED0F7AEB
:105D7000666028EE278A0023BCEEC88AC4E90305C2
:105D8000C4E905330A4884ED028A84F82030E361CF
:105D90002146FFF7E9FA204606B0BDEC028B70BD44
:105DA000041F0A00ACB0090088B0090000007A4462
:105DB0004393070008B501483AF056FC154A09001C
:105DC00010B50446808A43F040FBE3692BB1BDE87F
:105DD0001040D3E9020120F0ADBF014810BD00BF63
:105DE000DC2D090070B58B6804460D4616466BB174
:105DF00007494CF0FEFFA9682046324600F03EFEFF
:105E000004492046BDE870404CF0F3BF0249F9E771
:105E1000A21D09008C1E0900B21D0900F0B50C4638
:105E200085B054F8045B0646A88A174643F00DFB7C
:105E300002AB0193084B00933A4602232146701EA1
:105E400019F0F6FE28469DF80C209DF8081004F085
:105E500053FA0E2005B0F0BD1C1F0A0008B501481A
:105E60003AF0E6FB17450900084930B500228825BD
:105E700005FB02F463180C5B844204D00132052A4E
:105E8000F6D1002030BD1846FCE700BFA009012074
:105E90002DE9F04F8BB004AB51F8048B0193784B94
:105EA00000930138012319F0C3FED8F804402046BE
:105EB00000F0F6F87348049D2146FFF755FA0020DC
:105EC00017F05AF80E2D606030D101210AE06268A7
:105ED0009368D26803F18043013B52F82330D98A9A
:105EE000013189B2002220460BF0CCFE0028EED111
:105EF000654F002663689A68964236D3214661480A
:105F0000FFF764FAD8F80440204600F0C9F8636847
:105F1000D3E9020120F00EFFD8F804300446586897
:105F20004CF0E5FC20460BB0BDE8F08F284606A9F2
:105F30001DF06EFC554E054628461DF02BFE002830
:105F4000D6D0830702D10368B34202D050483AF05A
:105F5000D3FB8388ADF8143005AA83798DF8163009
:105F6000012120460BF08EFEE6E7DB6853F8265051
:105F7000AB680BB90136BDE7AB8ADFF81C91EA8A42
:105F80009A4212D3ADF81830DFF810A1C9F80050CA
:105F90000023ADF81A203B702088012306A98AF857
:105FA000003053F0A5FF00283DD02B699B68029379
:105FB0000023029A9A42DDD02A69D1685A1C0392C2
:105FC000029A51F823B0501E834216BF01EB8301A1
:105FD00000234B68DBF8081009B3BBF8141001313B
:105FE00089B2002B32D09B8A013B1FFA83F9E88AE1
:105FF000884214D3494512D8264BADF81810DFF863
:106000009CA0C3F800B000213970ADF81A900121AE
:106010008AF80010208806A953F06CFFD8B1039BC2
:10602000C7E7FAF71FFC9AF80030002BF9D13B784C
:10603000002BBAD02A699368D26803F18043013BF0
:1060400052F823309B8A01339BB298E7B5F816903B
:10605000CDE7FAF707FC9AF800100029F9D1397852
:106060000029DCD0DBF81C008168C06801F18041A8
:10607000013950F82110898A013189B2B7E700BF90
:10608000CC1F0A00C51C04005F690120D8AF0900BD
:1060900032350900545D0120505D01205E69012008
:1060A00008B543F0F5FC10B901483AF0C1FA08BD53
:1060B000C649090038B544680D4D2046FFF7F0FF8A
:1060C00094F874306BB9B4F86C3000EE103AB8EE56
:1060D000C00AF7EE047ABDE8384020EE270A20F027
:1060E0009DBCAB6A002BEED1FAF7BCFBE8E700BF22
:1060F000745D012010B50446C06D0E2805D103491A
:106100000C204CF05EFC4460E06510BDC8B0090096
:1061100030B585B003AB51F8044B0193224B00938B
:106120000138012319F084FD9DF80C3033B91F4864
:106130004FF4A67240F2DD213AF09EFA64681C4DDD
:106140002046FFF7ADFF94F85A30012B01D1AB6A1E
:10615000EBB194F85A30022B22D00123154984F870
:106160005A302088124D53F099FE43F093F994F879
:106170005A30012B01D1AB6A63B1AB6A83B994F891
:106180005B1069B1882908D10B4822F097FEFAF715
:1061900069FBD8E7FAF766FBE9E7084822F08EFECC
:1061A0000E2005B030BD00BFD41F0A00554D0900B8
:1061B000745D0120241D0A0077400900CF400900CA
:1061C0002DE9F04796B00FAB0193544B0093043187
:1061D0000723013819F02CFD51490F984FF43F72F5
:1061E00019F00CFE4F4940F24D620746109819F025
:1061F00005FE9DF844908246484643F027FC9DF8F2
:106200004880404643F022FC139E002E04DA40F200
:106210006D41002019F09EFD15989DF850500E28F4
:1062200004D14DB346B330464CF0F6FB052204A929
:106230001DF082FA059840F216423146F5B119F088
:106240009BFD394918204CF0BCFBC0E9017A0023C2
:106250000446838280F8169080F81780DDE90401F7
:1062600020F030FBE060002D4FD1B6F5007F08DD57
:106270002E4A4FF400714EE02D48D7E719F088FD03
:10628000DFE72682A574FB69002B3AD0A368A17DC5
:106290009A889B798DF80E3085F001050DF108087C
:1062A00045F002050026404605F00705ADF80C2034
:1062B000ADF808608DF80A5042F032FBE17D0DF137
:1062C000090042F02DFB052207A9E0681DF034FA11
:1062D00003ABCDE90A38089BADF83030238AADF81E
:1062E00034300AA9079BB88A0E9304F11402ADF862
:1062F000326053F011FE43F0CDF8F86921464CF0BE
:10630000D3FA204616B0BDE8F087B6F5FF7FB8DDBA
:10631000084A4FF4FF7108483AF00AFA941F0A003D
:10632000ACB00900D8AF09006CB0090071DD0800FD
:10633000E85E09007CDD08008236090070B58B68D4
:1063400004460D4616466BB107494CF052FDA9684C
:106350002046324600F092FB04492046BDE87040DA
:106360004CF047BD0249F9E7DA1D09008C1E09000F
:10637000E61D09007FB504460522084601A91DF067
:10638000DBF9A58A65B163685E68F06842F09BFB43
:10639000B37901463BB1002301AA284642F017FC1D
:1063A0000E2004B070BDA07C029B228A20B19A42CC
:1063B00006D006483AF0B4F99A4201D20448F9E707
:1063C00001AA284642F02AFCEAE700BF354009004E
:1063D0002A400900022A70B504460E4615460BD124
:1063E00040F2722052F02FFF014620464CF0F2FCA2
:1063F000054920464CF0EEFC2A4631462046BDE8D1
:1064000070401EF079BF00BF66DD080070B506461B
:1064100086B008460D46144642F045FB00234FF473
:1064200000722048019401A9CDE90223ADF8105073
:106430008DF81430FEF798FF00223146284653F0BD
:1064400061FD11280446F7D030B1164801A9FEF7C6
:10645000BDFF204643F01EF89DF81430B3B1BDF8DF
:10646000100042F020FB01A90E48FEF7AFFFBDF877
:10647000121089B291B140F20513994209D040F24D
:106480000F13994208D0084822F00AFDFAF7EAF9FA
:10649000E2E7064822F012FD0548FBE7039806B044
:1064A00070BD00BF69740700E44009006A47090035
:1064B0006147090008B501483AF032F9B3450900CF
:1064C0002DE9F04788B0084611461A4605AB0193FE
:1064D0002D4B009303234AF00FFF2C4905984FF4EE
:1064E0003F7219F08BFC069D002D074604DC40F23C
:1064F000E621012019F02EFC07980E2836D17E8A5D
:10650000234930204CF05DFA40F2FD139E4228BF33
:106510001E467B68BA7D9B7902F03004804602F00B
:10652000060213B9134622461C4642B306F102097D
:1065300005FB09F948464AF0B8FC054614B3304655
:106540004AF0B3FC824630464AF0AFFC04460023D2
:10655000CDE902634046CDE900A44B462A463946C0
:10656000F4F71AF9404608B0BDE8F08740F26F41F1
:1065700019F072FC061EC3DC40F26F41B9E7154604
:106580009146DBE7A246E2E70C200A00ACB0090026
:1065900050B0090030B50D4685B00446406842F061
:1065A0004FFF062201A928461DF0C6F8DDE90112B9
:1065B000204643F0B9FA002803DA414203483AF092
:1065C000B7F8400040F0010005B030BD214B090094
:1065D00010B58AB002AB0C460193144B0093043102
:1065E0000223013819F024FB2468606842F028FF78
:1065F0000298052207A91DF09FF8039800230E2892
:10660000059303D0052204A91DF096F8059B00937D
:10661000DDE90712049B204603F04CFF20EAE070FE
:10662000400040F001000AB010BD00BFFC1F0A008E
:10663000F8B5354C354B236043F0E9F9002861D0BB
:10664000334B1A781AB9334A1278012A28D13248C2
:1066500000251D7003F004FF304B9A8A02B19D8221
:106660002F4B9A8A0AB100229A822E4D6B68BBB1D9
:106670002D4B1B78A3B1284603F004FF284603F0F6
:10668000EFFE2A4B9A8A0AB100229A82284B9A8AF4
:106690000AB100229A82274B9A8A0AB100229A8272
:1066A000194803F0ADFCE36813B1174803F08AFC06
:1066B0000023214DA3614FF6FF7705240E2628887D
:1066C000B84202D0132153F0FBFB013CEE6505F10B
:1066D0008805F4D154F0C7FF0B48214603F014FBA2
:1066E0004FF42A23154A1B68934205D14FF43122F7
:1066F000D2F8FC2F9A4201D000F072FBBDE8F840BE
:1067000035F06EBEF8BD00BF8851012020B10900F0
:10671000A768012090690120185001209C62012087
:10672000CC62012048500120D5670120CC610120B6
:106730001C6201204C620120A0090120313044423A
:1067400030B589B003AB51F8045B01930E4B009355
:106750000138022319F06CFA9DF81040039805A93E
:1067600005221CF0E9FF84F00104E8680094DDE9EB
:106770000523D0E9021042F095FA00280CBF1E2034
:106780003E2009B030BD00BFEC1F0A007FB50846AF
:1067900011461A4602AB0193104B009302234AF0B4
:1067A000ABFD40F24D6202980D4919F027FB0D49EF
:1067B0009DF80C60054618204CF00AF904460020AC
:1067C00016F0DAFB324603462946204640F0EAFB43
:1067D00042F060FE204604B070BD00BFDC1F0A001E
:1067E000D8AF090000B0090070B58B6804460D46AB
:1067F00016466BB107494CF0FCFAA96820463246B0
:1068000000F03CF904492046BDE870404CF0F1BA74
:106810000249F9E70A1E09008C1E0900131E09002F
:1068200008B5014839F020FFAC43090010B5022833
:1068300088B00B46144624D1A20720D12168124A01
:1068400091421CD19A79012A09D1A279012A06D153
:106850009A88A3889A4212D13E2008B010BD1846EB
:10686000694643F0A8F904A9204643F0A4F9102290
:106870000DEB020168464AF09EFB0028ECD01E207A
:10688000EBE70020E9E700BFD8AF090008B58B7837
:1068900013B9044822F004FB0B8883808B78837142
:1068A00008BD00BFEE4009001FB58379012B02D15E
:1068B000054839F0B5FE694643F07DF91021684678
:1068C00020F000F805B000BDEB340900F0B51C461F
:1068D00008468FB011464FF0021219F071F9206886
:1068E000C20706D410F0030317D10168414A914250
:1068F00013D14BF093FCA2234FF6FF7200214AF014
:106900002EFD3D49054608204CF05BF80123044666
:106910008580837120460FB0F0BD384A0240062AB8
:1069200005D0002B4DD10268354B9A4249D101A9BF
:1069300021F028F9019B242B02D0324839F0F0FED7
:10694000037A2D2BF9D1437B2D2BF6D1837C2D2B74
:10695000F3D1C37D2D2BF0D1461E00F12304002579
:1069600016F8017F384639F03BFE28B105F13803AF
:106970006B44013503F8207CB442F1D1202DDCD1E9
:1069800006AD0F2402AE287856F06CF907466878F9
:1069900056F068F940EA0710A055013C631C05F168
:1069A0000205F0D100231449BDF81450ADF814309D
:1069B00008204CF006F802A98580044643F0E5F86B
:1069C000A8E7012206A91CF0B7FE08B90E48B5E7F2
:1069D0000798A222102119F0CFF9069B02AC03F10F
:1069E000100518685968224603C20833AB421446A2
:1069F000F7D1D7E7202F0900D8AF09000F0080FF9B
:106A0000942D09005041090041410900F0B589B0B9
:106A100003AB51F8044B0193174B00930138022349
:106A200019F006F9062205A903981CF085FE069FB9
:106A30000498002140F2B3433A464AF090FCA6790C
:106A4000012E14BF802110210546C90840F2E5221D
:106A5000381A4AF090FC059B012E03EB050107D183
:106A6000A2885A55A3881B0A4B700E2009B0F0BDAE
:106A7000204643F0A0F8F8E7AC200A0010B58A7968
:106A8000012A92B0044606D18A881F4912B0BDE897
:106A900010404CF0AEB908460EA943F08CF89DF8B2
:106AA00038300D939DF839300C939DF83A300B93A4
:106AB0009DF83B300A939DF83C3009939DF83D309A
:106AC00008939DF83E3007939DF83F3006939DF85C
:106AD000403005939DF8413004939DF84230039374
:106AE0009DF8433002939DF8443001939DF8453062
:106AF00000939DF847209DF84630044920464CF00D
:106B000078F912B010BD00BF341E0900411E090003
:106B10002DE9F0472DED048B84B002AB0193344B8B
:106B20000093022319F084F8039C0E2C04D14FF437
:106B300080504BF063FF04460221204649F0E7F8FD
:106B4000074660B920461EF045FFC38800932948D8
:106B500040F257232E2240F2F65139F0D5FDDDF8F0
:106B600008809FED258ADFED258A002507EE905AE3
:106B7000B8EEE70A07EB851920EE080A1FF04EFF72
:106B800000268246B7EE009A07EE906AB8EEE70A52
:106B900020EE080A1FF042FF5146024640464AF0E6
:106BA000EAFC1EF08DFEB5EEC00AF1EE10FA1AD422
:106BB000B4EEC90AF1EE10FA17DC20EE280A30F024
:106BC00087FAFCEEC07A17EE903A09F806300136E3
:106BD000402ED9D10135402DC8D1204604B0BDEC9E
:106BE000048BBDE8F0870023EFE70123EDE700BF4A
:106BF00034260A00B64D09002108823C00007C4280
:106C00002DE9F04F754C85B0002600AFA4F10808BF
:106C10004FF0880909FB068393F87830002B65D084
:106C200054F021FDD4E91E23801A61EB0301B0F575
:106C30007A7F71F1000159D3002134F8080CF980F2
:106C40000323BA1D6D4653F075F9002847D1FB8820
:106C500034F8080C0733DB08A5EBC3039D46BA1DC7
:106C600003236946EA4653F065F9002837D1B4F8A2
:106C7000502014F8060C022148F06CFD834660B1E8
:106C8000FB88C2889A4205D100F1080168464AF0A3
:106C900092F920B3584649F0ACFC00233B7214F83B
:106CA000063C3A89F888F88143F4007302F0FE024A
:106CB00023F0FE0313433B81B4F850307B8134F85A
:106CC000083CBB810FF026FA0222834607F1080137
:106CD00031F062F8FA885146584656F026FD88236E
:106CE00003FB06830022AD4683F8782009FB068368
:106CF00093F87930002B41D014F8060C002847D0C7
:106D0000B4F82EA05246012148F024FD054650B1AA
:106D1000C288502A04D1214608304AF04CF940B3C9
:106D2000284649F066FC002028F0BEFD054690BBD1
:106D3000387214F8063C3A89A7F80AA043F4807325
:106D400002F0FE0223F0FE03134350253B81284648
:106D500034F8083CBB81FD810FF0DCF90222824649
:106D600007F1080131F018F82A462146504656F03E
:106D7000DCFC09FB0683002283F879200136052E0E
:106D800004F188047FF446AF1437BD46BDE8F08FA8
:106D9000B4F812A0B6E76B78012B1DD12B7814F84C
:106DA000062C03F001039A4216D1B5F806B0BBF1E8
:106DB000500F11D1062204F1490105F151004AF0AA
:106DC000FAF848B95A46214605F108004AF0F3F8A6
:106DD00010B1284649F00DFC2846A5E7A809012076
:106DE00073B5104D4FF42A244FF00106200B2E707E
:106DF00053F0BCF808B930F0BFFF04F58054B4F587
:106E0000322FF3D1084B019301A901224FF42A201C
:106E100030F0C2FF0548012201A930F0BDFF02B0E9
:106E200070BD00BF7569012031304442FC1F0B006A
:106E3000032A05D11E2914BF044905494BF0CABFD6
:106E40001E2914BF03490449F8E700BF15DD0800F7
:106E50001ADD08007CDD080071DD080030B587B060
:106E60000C460592D1E90123174904935528CDE931
:106E70000212236809D054F8042C02A9184620F005
:106E8000CDFFA4F1080007B030BD184600931EF0F6
:106E9000A1FD827B009B82B100EB820002A9056903
:106EA000019318460422A8470090F6F775F9DDE92A
:106EB000000310B120602046E5E718464BF0BAF910
:106EC0000146024839F020FCCC580900EB4C09007F
:106ED0002DE9F04F2DED028BB9B00AAF08461146EF
:106EE0001A4607F150030193BA4B00931A234AF054
:106EF00003FA3B6D786D3B60052207F144011CF0FD
:106F00001BFC40F2BA21D7F890003BF08FFDF863EC
:106F1000D7F898001EF0D4FCD7F868B05A229BFB33
:106F2000F2F302FB13B3B0EE408A13B1AA4839F072
:106F3000F7FB97F8B0A0FE6EBAF1000F08D0012E53
:106F400006D0A64840F21A224FF4447139F0F0FB03
:106F5000F5F7D2FAA24B036097F88450B7F9603086
:106F60007D6297F888503B633D62B7F9643097F8CB
:106F70008C50FB62FD6197F870307D6C7B63BD6166
:106F800097F8A030BD6C7D610446B7F8945097F82F
:106F90007400FB6097F8A43097F87CC097F880E005
:106FA000B7F85810B7F85C20D7F8A890B8623D61E0
:106FB00097F8780097F89C50BB6397F8AC30BB60AB
:106FC0004FF00008D7F8B4307B6084F8B380CDE987
:106FD00004CE0390BB6A02937B6BB6B2CDE900632B
:106FE00004F108001FFA8BF346F0E1F904F15003B5
:106FF0007B63012E14BF00230AF00103CDE9078350
:10700000CDF82480FB6806934FF48073CDE90433F8
:107010003B6A03937B6A0293FB6A01933B6B009389
:10702000C5F58075ABB21A46396804F150000BF013
:1070300063F9FB6984F8B2303B69A4F8AC30BB6BF0
:10704000A4F8AE9083F0010384F8B430BB6884F8F0
:10705000B5301FFA89F94FF47A73B3FBF9F3A4F84A
:10706000B030BB8AFB62C346FB6A9B4537D35D4B9E
:10707000C4F88430FB6BD3B1187943F0C1F8B0B1D8
:1070800000220092BB88F96B04F1840005F030F90E
:10709000002800F08B80544BC4F88430F96B04F165
:1070A000840042F0EAFDFB6B187943F0BEF8B0EEC5
:1070B000480A204603F07CFA4C4991F82A309B0795
:1070C00002D4204642F096FDB96B204642F07EFD88
:1070D0002046BC37BD46BDEC028BBDE8F08FBB69D6
:1070E00003EB0B0898F80150786B0BF0F7F80028C9
:1070F0003AD094F880906BB23B6305F07F05B9F10C
:10710000000F3CD005F1080303F0F803E946ADEBAE
:10711000030D98F800208DF828200AAB6E1C2A4633
:1071200008F102010DF12900BB6249F058FF0096F9
:10713000266EBB6A206D01220021B047CD46786BD8
:1071400045F0B0FF3B6B002B2DDA6E1C023518F8B2
:107150000500FF2808BF4FF4FA701CF0A9FB0BF1E3
:10716000020306EB030B7FE7F9F77CFB204B9B6ADE
:10717000002BB9D01F4840F26F3139F0A7FA012334
:107180000093B5EB0902206D266E434618BF01221D
:107190004946B0470095206D266E08F102034A4625
:1071A0000121B047CBE72E460A20D6E7124BD4F890
:1071B0008800C4F884302DF04DFF94F88C200F49DE
:1071C00002F07F02012393400A5C13430B54D4F86E
:1071D000903069E744290A00FB480900034E090082
:1071E000F8C30900A060090038C309004401012068
:1071F000745D0120374E09009CBC090062690120C2
:10720000F0B58DB002AF07F108030C460193264B91
:10721000009304310223013818F00AFD206823F09E
:1072200043FBD7E902650446062207F11C01284604
:107230001CF082FA94F83A30102B02D01B4839F037
:107240006FFAA28E386ABA8202F00103002103EBC2
:1072500052033961B0EB830F7E8206F10106B961FA
:10726000FE821ED3520901327A607A68FB6992006D
:10727000073222F00702ADEB020D02AA8C467E68AF
:1072800088B2864209D807F1100104F1080046F0DF
:10729000C4F828462C37BD46F0BD42F820C0013165
:1072A000EDE70348CBE700BFAC2A0A000D4909000F
:1072B0001A4B090008B5014839F000FA424B0900A1
:1072C0007FB502AB0C4601932B4B00930431022394
:1072D000013818F0ADFC206823F0E6FA039B044661
:1072E0000298002BCABF4FF47A764FF0FF3696FB18
:1072F000F3F60E2811D04AF091FF4FF47A7595FB02
:10730000F0F594F8B3305BB10023204684F8B43034
:1073100040F01DF93E2004B070BD4FF0FF35F0E79E
:1073200094F8B430002BEFD16B1CEDD054F09BF9E6
:107330002369C31A9E4202D2104839F0BFF9D4F82B
:10734000A020821A9542C4E9280112D3B3FBF5F2BA
:1073500005FB1233ED1A54F086F9D4E92832C01A2D
:1073600061EB0201A84271F10001CDD2F9F77AFA7E
:10737000F1E71E20CFE700BF34290A00724B090055
:1073800038B50D4623F090FA044628461EF098FAC8
:10739000B5EEC00AF1EE10FA06D4B7EE007AB4EEFC
:1073A000C70AF1EE10FA01DD00F00CF8204603F0F8
:1073B000FFF810B9024839F081F90E2038BD00BF3E
:1073C000424B090008B503480123002240F2E321A3
:1073D00039F0AEF90D4E090008B5014839F020F931
:1073E000664C09002DE9F04786B0084611461A465A
:1073F00002AB0193674B0093042349F07DFF40F2F9
:10740000795102983BF006FB40F27C510546039807
:107410003BF000FB604906460C204BF0D9FAFF23F5
:10742000DDF8108083722A7933799A42044603D1B9
:1074300040F2E24018F0EEFB00234360574B1A7A0B
:1074400022B11A7E002A40F0A280012203EB02132F
:1074500063602879012128F0AFFA0121307928F002
:10746000ABFA0A2028F006FC2879002128F0A4FABB
:107470003079002128F0A0FA032028F0FBFB3079B6
:1074800028F0ECFA40B930792EF0E8FE28792EF099
:10749000E5FE434839F012F9287928F0DFFA002890
:1074A000F1D0404B96F804902F79984522D83E4B66
:1074B00098458CBF4FF080684FF0CC786772307978
:1074C000A07201F059FF2879384D01F055FF63682B
:1074D00001221A72666896F804A0342101FB0AF1B1
:1074E0006B1893F82D2042B1204603F00FF90520C8
:1074F00039F0CEF84FF0C868E0E71F2F9A6083F8A4
:10750000302083F82F2083F832205E608ABF07F096
:107510001F033B46264A2748685098BF4FF0A042B9
:1075200003F5E073B9F11F0F40F20C6142F823102C
:107530008CBF09F01F034B4603F5E0738CBF1C4A58
:107540004FF0A04240F20C6142F823103368C3F8B8
:107550000875C3F80C95C3F82485342303FB0AF39C
:10756000EB5853B13068072140F30730F1F7E6FDDF
:10757000306840F307303FF067F9342303FB0A55C6
:107580002046012385F82D3006B0BDE8F0870A4873
:1075900039F0C6F88C2A0A00DCC30900580401201F
:1075A000854509007F1A06008FD00300985C0120F2
:1075B0000003005057CA0800354C0900F0B50C46CE
:1075C0008DB054F8045B0646A87A174641F021FFB7
:1075D000284641F059FF08AB01931D4B009321460B
:1075E0000423701E3A4618F023FB062205A90998C9
:1075F0001CF0A2F89DF81C100022402018F05CFC42
:10760000069B0B99B3FBF0F30446049304AA0A9B70
:10761000039303A850F0CFFE049E40F2E52201211F
:10762000304649F0A8FE039A06FB04F36243039236
:10763000049353B1059928460A44BDF8201003F07D
:10764000E7F810B1404239F023F80E200DB0F0BD3C
:107650006C2A0A00F0B50C468DB054F8045B06465F
:10766000A87A174641F0D5FE284641F00DFF08AB39
:1076700001931A4B0093214604233A46701E18F0DA
:10768000D7FA052205A909981CF056F89DF81C1098
:107690000022402018F010FC069B0B99B3FBF0F37E
:1076A0000446049304AA0A9B039303A850F083FEA4
:1076B000039A049B0121009105996243039263435D
:1076C0000A442846BDF820100493F3F7CBF810B114
:1076D000404238F0DDFF0E200DB0F0BD4C2A0A000C
:1076E0002DE9F0410C4694B054F8046B0546B07A8D
:1076F000174641F08EFE304641F0C6FE0DAB0193B9
:10770000314B00933A4607232146681E18F090FA41
:1077100005220AA90E981CF00FF89DF830100022DF
:10772000402018F0C9FB0B9B1199B3FBF0F3054601
:10773000069306AA109B059305A850F03CFE06226E
:1077400007A90F981BF0F8FF9DF824100022402095
:1077500018F0B2FB089B1399B3FBF0F304460493B3
:1077600004AA129B039303A850F025FE049F40F245
:10777000BF420121384649F0FEFD0598069BBDF841
:107780003480002268436B430092039D0A9A05905F
:10779000654302447C4341463046079F0693039568
:1077A0000494F3F75FF838B94CB123467A1941468F
:1077B000304603F02DF810B1404238F069FF0E203A
:1077C00014B0BDE8F08100BF142A0A00F0B50C46E1
:1077D00087B054F8045B0646687A174641F013FEFA
:1077E000284641F051FE02AB0193184B009321460D
:1077F000701E04233A4618F01BFA40F2EB430122B4
:107800000021039849F0ABFD40F2DB430122002147
:107810000446049849F0A3FD4FF433730646092249
:107820000598082149F09BFDC0B2082802D0052028
:1078300038F02EFF0299F3B2E2B2284642F0E3F9A3
:107840000028F4D00E2007B0F0BD00BF242B0A00A2
:107850002DE9F04F89B0084611461A4604AB019352
:10786000744B0093042349F047FD40F2053104981E
:107870003BF0D0F840F29341074605983BF0D6F82C
:1078800040F28441044606983BF0D0F8064618B909
:1078900014B9694838F044FF68490C204BF098F857
:1078A0009DF81C30FF220546427223B1644840F225
:1078B000F63138F0E1FE4360624BD3F8003513F047
:1078C0000F0305D0604BD3F800351B0711D10123FE
:1078D0005E4A02EB03136B6097F80480D3F808A0AC
:1078E00085F80980404601F047FD24B9FF24AC72B9
:1078F00006E05748CEE72479AC72204601F03CFD03
:107900000EB33679EE72304601F036FDD5F804B08C
:10791000504F9BF80490242303FB09731B7F63B92A
:107920005046F8F7DDFF0290B9F1000F0ED1B0F12B
:10793000206F02D0B0F1A05F0BD1284602F0ACFF5F
:10794000052038F0A5FEFF26EE72DFE7B9F1010F42
:10795000F3D1242202FB09F2B8180021DBF800A0C1
:1079600041604046B95028F05BF8B8F11F0F8BBF5B
:1079700008F01F02424638494FF0A04102F5E0727C
:107980000120FF2C41F822004AD0204628F048F878
:10799000204628F021F8FF2E45D0002130460396DE
:1079A00028F00AF8039A242101FB09F3F91803933C
:1079B00081F82160FF2681F820600221CAF8601555
:1079C000029BCAF80885CAF80C45CAF8102500229F
:1079D0001146CAF82435504650F02DFD039BCAF8D5
:1079E000C065FA5807210AB34022CAF80423CAF82E
:1079F0000015DBF8000040F30730F1F79FFBDBF8E0
:107A0000000040F307303EF01FFF242303FB0977FB
:107A100000237B77284601233B7709B0BDE8F08F30
:107A20004FF0FF34B7E74FF0FF32BCE7CAF800155C
:107A3000EBE700BF442B0A0022460900C0C309003F
:107A4000914E090000F0024000300240501E0A0032
:107A5000244C0900385C01200003005010B5044696
:107A6000407A41F0D0FC63681B68D3F82435B3F149
:107A7000805F23D013D8B3F1006F21D00BD8B3F1BE
:107A8000007F1FD01248B3F1806F18BF0020400064
:107A900040F0010010BD0F48B3F1206FF5E7B3F1DE
:107AA000804F11D006D8B3F1A05F0FD00A48B3F1D0
:107AB000005FEAE70948B3F1004FE6E70848E6E768
:107AC0000848E4E70848E2E70848E0E70848DEE756
:107AD00090D003000024F40080841E0000127A007D
:107AE00040420F0020A1070048E8010000093D00C6
:107AF0000048E801F0B50C468DB054F8045B06462A
:107B0000687A174641F07FFC284641F0BDFC08AB7F
:107B100001931A4B0093214604233A46701E18F035
:107B200087F8062205A908981BF006FE9DF81C1090
:107B30000022402018F0C0F9099B0A9904930446DA
:107B4000069BB3FBF0F303AA04A8039350F033FCA5
:107B50000499039B614303FB04F20491039252B125
:107B600005989DF82C300144284642F06BF810B976
:107B7000052038F08DFD0E200DB0F0BDEC2A0A0076
:107B8000F0B50C468BB054F8045B0646687A17468D
:107B900041F039FC284641F077FC07AB0193194BC3
:107BA0000093214603233A46701E18F041F805223F
:107BB00004A907981BF0C0FD9DF818100022402072
:107BC00018F07AF9089B03930446059B0999B3FBC7
:107BD000F0F302AA03A8029350F0EDFB039B029A74
:107BE000634362430393029242B1049928461944C5
:107BF00002F0F6FE10B9052038F04AFD0E200BB059
:107C0000F0BD00BF0C2B0A00F0B50C4693B054F841
:107C1000046B0546707A174641F0F5FB304641F09B
:107C200033FC0CAB01932B4B009321460623681EBB
:107C30003A4617F0FDFF052209A90C981BF07CFDC0
:107C40009DF82C100022402018F036F90E9B0F9959
:107C5000059304460A9BB3FBF0F304AA05A804931A
:107C600050F0A9FB062206A90D981BF065FD9DF8B2
:107C700020100022402018F01FF9109B1199039347
:107C80000546079BB3FBF0F302AA03A8029350F04A
:107C900092FB049B039A0298059963436A43454308
:107CA0006143AB42059104930392029502D00A48C6
:107CB00038F036FD53B10698024409980144304625
:107CC00002F056FE10B9052038F0E2FC0E2013B089
:107CD000F0BD00BFBC2A0A00903D09002DE9F04F1D
:107CE0002DED028B97B0084611461A460AAB019358
:107CF0005A4B00930C2349F0FFFA40F26D510B9858
:107D00003AF094FE40F2246181460A983AF08EFEE1
:107D100040F26951824612983AF088FE40F23631BC
:107D2000804613983AF082FE40F264510746149858
:107D30003AF07CFE0546BAF1000F05D1B9F1000F0B
:107D40000DD1474838F0ECFCD14518D0C24516D0CB
:107D5000BA4514D0824512D0B9F1000F05D0C14503
:107D60000DD0B9450BD0A94509D0B8F1000F03D00B
:107D7000B84504D0A84502D02FB1AF4203D140F29C
:107D8000E24017F047FF4FF43373092205210D98A5
:107D900049F0E5FA40F21F534FF6FF720646012103
:107DA000119849F0DCFA0E9B2E4A9342834629D063
:107DB0002D4AA3EB020CDCF1000343EB0C035B0048
:107DC000022201210F980293962349F0C8FA1098D5
:107DD0001DF076FDB0EE408A55F051F99DF8543013
:107DE000224903932C204AF0F3FDF6B20C9B079333
:107DF000082E039B044607D01D4808224FF4337118
:107E000038F096FC0123DBE705B913B1194838F0C7
:107E10002BFC4560184D2B68D3F8003513F00F0389
:107E200005D0AB68D3F800351E0714D10123DE005E
:107E300005EBC303636003931FFA8BF3184640F20C
:107E40001F520121069349F082FA029B022B039BE9
:107E500018D10A4876E70A4874E700BF642B0A0085
:107E6000FD30090080640900846409009CC3090096
:107E7000134E0900B343090068020120DF440900E2
:107E8000154C0900BAF1000F00F0E0809AF804B038
:107E9000B9F1000F00F0DD8099F804200492002F62
:107EA00000F0DA803A790592B8F1000F00F0D7803F
:107EB00098F804200392029A1B790893002A18BFAD
:107EC0000E2208990292794A242303FB012393F896
:107ED0002030002B40F0C68047EA0803079809933A
:107EE00010F0A0FABBF1FF3F099005D0584627F0EB
:107EF000C5FD584627F070FD049B581C03D0002197
:107F0000184627F059FDAB59099AC3F82425029B5E
:107F1000AA5947EA0801002918BF43F00103DBB260
:107F2000C2F86C35AB59049AC3F80CB5C3F81425E4
:107F3000B1B1059B591C03D00021184627F03CFD28
:107F4000039B5A1C05D0184627F098FD039827F08C
:107F500043FDAB59039AC3F80825059AC3F81025C9
:107F6000089A5249A8592423534301EB030B504A62
:107F7000CC504FF48871CBF8042050F039FAA8594E
:107F80004FF4907150F034FAA8594FF4927150F0B8
:107F90002FFAA8594FF4A27150F02AFAA8594FF4B9
:107FA000AC7150F025FAAB59424AC3F80423A859E2
:107FB000032140F30730F1F7C1F8A85940F3073027
:107FC0003EF042FCAB590822C3F800250023CBE960
:107FD0000633CBF8143001238BF82030B9F1000FB1
:107FE00045D1BAF1000F55D09AF8040084F8260064
:107FF00001F0C2F9B8F1000F50D098F8040084F8ED
:10800000290001F0B9F9002F4CD0387984F8280004
:1080100001F0B2F9DFED287A079BA36028EE278AEA
:108020000023BCEEC88A84F82530606884ED038A9A
:1080300004F1240128F072F8204B9842024612D134
:10804000204617B0BDEC028BBDE8F08F4FF0FF3B30
:108050001EE74FF0FF3221E74FF0FF3223E74FF0EA
:10806000FF3227E7164A1749174854F00EFE0699C3
:1080700004F1100051F077FD28B9606828F0D4F8B9
:10808000069838F0B7FA99F8040084F8270001F050
:1080900073F9A6E7FF2384F82630ABE7FF2384F8C3
:1080A0002930B0E7FF2384F82830B3E7005D0120D2
:1080B00061CA08001003420000007A440000AD0BC2
:1080C0000500AD0B7D3A0900E44E090010B522F021
:1080D00053FC90F82730FF2B044628D0406828F046
:1080E000A3F894F826002EF0B9F894F827002EF0A3
:1080F000B5F894F829002EF0B1F894F828002EF085
:10810000ADF861680B4A4FF6FF73E3842385914213
:108110004FF00003C4E90433C4E90733A36103D07B
:108120000832914203D10123034A0021D1540E2089
:1081300010BD00BF680201206069012010B522F067
:108140001BFC044690F8270041F057F994ED030A10
:10815000DFED047AB8EE400ABDE8104080EE270A51
:108160001EF05CBC00007A4410B522F005FC044609
:1081700090F8270041F041F96368186840F3073030
:10818000002801DBF0F7CAFF0023C4E90733A3612D
:1081900063681B6843F30733002B08DB590901228E
:1081A00003F01F0302FA03F3024A42F821300E20C3
:1081B00010BD00BF00E100E038B52DED028B0D468B
:1081C00022F0DAFB044690F8270041F016F9284621
:1081D0001DF076FBB0EE408A54F051FFDFED057ADA
:1081E00028EE278A0E20BCEEC88A84ED038ABDECF7
:1081F000028B38BD00007A4407B50A4A40F2931357
:10820000914208BF4FF4A173019340F2ED13009324
:10821000054940F2422340F2EA224AF0EAFD03B067
:1082200000BD00BF806409009C1E09002DE9F047D5
:1082300015460E461F4622F09FFB044690F8270085
:1082400041F0DBF81DB900252846BDE8F0876368DA
:108250001B68D3F81435013304D12E4840F26D5118
:1082600038F066FA53F0FFF9DFF8B0A0804689468F
:10827000A3699D4238D86368186840F30730002826
:1082800044DA2A46314604F1100051F08FFC94F88C
:108290002530054693B1012204F1240104F11000B8
:1082A00051F0ABFC04F12401606827F037FF94F82B
:1082B000290027F0B5FB002384F8253063681B688C
:1082C00043F30733002B08DB5909012203F01F0396
:1082D00002FA03F3104A42F82130002DB4D10B23E7
:1082E0003B604FF0FF35AFE753F0BDF9E368B0EB0B
:1082F000080061EB0901984271F10001BBD2F8F767
:10830000B1FADAF82830002BB2D09CE7F0F706FF7C
:10831000B7E700BFE045090000E100E0745D01201F
:1083200038B50C462046114606221D4617F048FC7B
:108330002CB921460120BDE83840F4F7F5BC296886
:10834000CB0706D411F0030308D10868144A904201
:1083500004D1012C14D0134838F0CEF9124A0A4047
:10836000062A04D03BB90A68104B9A4203D1012C6B
:1083700001D10F48F0E7BDE838400120F4F734BCE4
:10838000084649F04BFF054601462046F4F7CCFC71
:108390002A4604460021C06848F062FE204638BDE7
:1083A000202F0900972F09000F0080FF942D09004E
:1083B000D5310900012807B50B4606D10B6800939B
:1083C00040F61623019302206B4601460022024824
:1083D0001FF01CFC03B000BD942D090001460148AC
:1083E0001CF0DABA485E0900014A1CF01BBB00BF52
:1083F000485E0900014A1CF015BB00BF942D09001E
:1084000008B508460AB117F00DFC21B11946BDE8C0
:10841000084000F005B8014808BD00BFE85E09004B
:1084200070B50646086810F003038EB00D4603D100
:108430000168454A91422AD0444C00EA0402062AC7
:1084400004D043BB0268424B9A4224D1023E012E23
:1084500002D9404838F050F90AA91FF093FB0646AC
:10846000286800EA0403062B13D1000950F0D7FE58
:1084700004460A9D24B92946304650F0A7FE04461A
:10848000314910204AF09DFAC0E9025644600EB00E
:1084900070BD4468EDE7012E01D02F48DAE710F0F7
:1084A000010411D0441002D5002038F039F92146DA
:1084B0000AA855F07AF80C982246002148F0D0FD21
:1084C0000AA81EF007FAE2E701AA40F25F211BF0BA
:1084D000B5FF019B2BB101AA2146204649F055F872
:1084E000D5E72868324603A91BF026F920B1DDE95B
:1084F00003011EF0E7F9CAE728681EF035F90446C3
:10850000B8B91020CDE90A0448F0B1FC8DF8344028
:108510000C90286806A91BF07BF9044620461BF046
:1085200039FB0028CCD049F079FEFF2806D90B484A
:10853000BBE741100AA855F02AF8EAE7C1B20AA839
:1085400054F071FFEAE700BF485E09000F0080FFAA
:10855000942D0900D5310900972F09006D3D0900C0
:10856000F0B585B0054617460C461DF033FA69464E
:10857000064628461FF006FB042F054622D1A30716
:10858000009814D12268104B9A4210D101AA2146BA
:108590004AF079FD10B90D4838F066F8DDE90112AE
:1085A0003046521A29441EF06BFB05B0F0BD01465F
:1085B0000023224630461BF0DDF8285C400040F0E6
:1085C0000100F2E70020F0E7CC5809003734090039
:1085D0002DE9F14F8F0705460C46164613D001F0E2
:1085E0000F03022B19D102F0FD06012E4FEA1111E3
:1085F00004D001B0BDE8F04F06F08EBE01B0BDE87A
:10860000F04F06F097BB4968CBB22D2B00F0878066
:108610000BD8062B0ED02C2B13D0554A21462846BA
:1086200001B0BDE8F04F06F085BE2E2B00F08C8027
:108630009D2BF2D1002EF0D104F10802090A284640
:1086400087E0022A02D0A16806F0CAFBE768002F83
:10865000E3D017F00309E0D17B68DAB28E2AB8467E
:108660000DD1022E4FEA132805D007F1040A08F1B4
:10867000FF3BD94515DB08F1010857F8288098F829
:108680000430312B2BD1022E13D1686A49F011F935
:10869000686A56226FF0020101B0BDE8F04F45F064
:1086A000BDBB5AF8041F284606F09AFB09F10109E0
:1086B000DFE72846D8F8081006F092FB012E686A1A
:1086C00009D15822022145F0A9FB686A01B0BDE832
:1086D000F04F49F018B956226FF00201DCE7322B57
:1086E0009BD1012E686A0AD149F031F8D8F80810F8
:1086F000686A090901B0BDE8F04F48F0D9BF022E01
:1087000001D149F0DAF8D8F80830686A1B09182254
:108710006FF0010101B0BDE8F04F45F0FFBBA2686A
:10872000002A3FF47AAF002E7FF477AF5168090A30
:10873000022907D1D3682BB1980703D11B79AC2B41
:108740003FF46BAF08327AE7002A7FF466AFA16886
:1087500021B901B0BDE8F04F00F00CB88E0703D18D
:108760000B79922B0A46E1D004F10802012166E759
:10877000343D09002DE9F04701F1FF3A05468846EE
:1087800091464FEA0A2700244FF0FF3617F5807F05
:108790000CD1731C05D1686A4346302251460BF058
:1087A00053F8002444451DD1BDE8F08759F8241042
:1087B00071B18A070CD10A79222A09D101360BD16D
:1087C000686A47EA0403312251460BF03DF8264619
:1087D0000134A7F58077D9E72846084ABDE8F04775
:1087E00006F0A8BD59F82410A64208BF89680022E7
:1087F0002846FFF7EDFE0134D4E700BFE635090057
:1088000001F00F03022B2DE9F04707460C4604D177
:10881000BDE8F047090906F02BB900295BD011F03B
:10882000030558D10B792C2B3FD1896806F0D8FA73
:10883000E568002D4FD015F003084CD16E68F2B2F8
:108840008E2A2B4609D1360A05F1040906F1FF3AB2
:10885000C24518DC013655F826301A79312A1AD16A
:108860009968384606F0BCFA7C6A204648F0FBFF5F
:10887000204649F01EF820465622BDE8F0476FF02A
:10888000020145F0CBBA59F8041F384606F0A8FAA1
:1088900008F10108DCE7322A1DD19968786A0222C2
:1088A000BDE8F047090948F0EBBE2D2B13D18C68C9
:1088B0008CB163681B0A022B01D1E36833B9261D12
:1088C0006368B5EB132F0DD3BDE8F0879A07F6D197
:1088D0001B79AC2BF3D121463846064ABDE8F04758
:1088E00006F028BD56F8041F3846FFF789FF01350A
:1088F000E6E700BFD73C090070B5137803F06003CA
:10890000202B5AD12E4B90885C7884420ED093F85D
:108910003D48844251D103F63C0001255478203C67
:10892000032C4AD8DFE804F005050D311846002570
:10893000F4E7012903D10721043037F061F9012060
:1089400070BD012902D137F04BF9F8E70329F6D1C0
:108950005188847FC17001F0010282F001018C42D4
:1089600018BF817752B95B68B3F5966FE7D14FF0C6
:1089700080434E22C3F81C252DF046FC114B1248B3
:1089800001221A70F7F732FFD9E70129DBD003295A
:10899000D5D10E4B1B78002BD1D00D4B1B6801336A
:1089A000CDD0002DCBD15388002BC8D0094B0A4A1B
:1089B0005A6603F15C029A62C1E70020C0E700BF7B
:1089C0005C100120D7670120BC6101208B69012068
:1089D00020020120745D0120AC6309002DE9F047FD
:1089E00041F278020021214848F03AFB1F4B204811
:1089F00000211F464FF0FF094FF4E1380A464FF0BF
:108A0000080E4FF4806540F63C0C012603F23C440E
:108A10001C630CFB01744FF0000A83F80B90C3F841
:108A200004801A725A7283F80AE083F825209D8622
:108A300083F836206287228783F80DA003F13C0A71
:108A4000D862C3F818A09D839E776284228400F1C7
:108A500040045C614C1C022C03F63C0300F18000D6
:108A60004FF00101D2D1BDE8F08700BF5C100120BA
:108A70005C0F01202DE9F84F4B79022B81468A4685
:108A800015D18B79022B12D14D4F97F8266096B1F4
:108A9000BE7B86B197F8623863B197F84A384BB11C
:108AA0004FF0E023D3F8F03DDB0700D500BE0020F7
:108AB000BDE8F88F012640F63C037343F91807F828
:108AC00003909AF802304B709AF800400AEB0208C3
:108AD00054444445627805D223782344984501D311
:108AE000242A18D0052A0CD1204639F065FC00282C
:108AF000D6D040F63C0303FB0673A2789A70237825
:108B00001C446378042B38D163790A2B35D1234672
